:020000040800F2
:1000000000060020A1020008AD0F00082D0F000817
:10001000850F00082D0F0008590F0008A3020008E3
:10002000A3020008A3020008A3020008F9220008A6
:10003000A3020008A3020008A3020008A30200080C
:10004000A3020008A3020008A3020008A3020008FC
:10005000A3020008A302000881370008AD3700089A
:10006000D93700080538000831380008A302000815
:10007000A3020008A3020008A3020008A3020008CC
:10008000A3020008A3020008A3020008A3020008BC
:10009000A3020008A3020008A30200085D380008BC
:1000A000A3020008A3020008A3020008A30200089C
:1000B000A3020008A3020008A3020008A30200088C
:1000C000A3020008A3020008A3020008A30200087C
:1000D000A3020008A3020008A3020008A30200086C
:1000E000C1380008A3020008A3020008A302000808
:1000F000A3020008A3020008A3020008A30200084C
:10010000A3020008A302000835390008A302000872
:10011000A3020008A3020008A3020008A30200082B
:10012000A3020008A3020008A3020008A30200081B
:10013000A3020008A3020008A3020008A30200080B
:10014000A3020008A3020008A3020008A3020008FB
:10015000A3020008A3020008A3020008A3020008EB
:10016000A3020008A3020008A3020008A3020008DB
:10017000A3020008652E0008A3020008A3020008DD
:10018000A3020008A3020008A3020008A3020008BB
:10019000A3020008A3020008A3020008A3020008AB
:1001A000A3020008A3020008A3020008A30200089B
:1001B000A3020008A3020008A3020008A30200088B
:1001C000A3020008A3020008A3020008A30200087B
:1001D000A3020008512E0008A3020008A302000891
:1001E000A3020008A3020008A3020008A30200085B
:1001F000A3020008A3020008A3020008A30200084B
:10020000A3020008A3020008A3020008A30200083A
:10021000A3020008A3020008A3020008A30200082A
:10022000A3020008A3020008A3020008A30200081A
:10023000A3020008A3020008A3020008A30200080A
:10024000A3020008A3020008A3020008A3020008FA
:10025000A3020008A3020008A3020008A3020008EA
:10026000A3020008A3020008A3020008A3020008DA
:10027000A3020008A3020008A3020008A3020008CA
:10028000A3020008A3020008A3020008A3020008BA
:10029000A3020008A3020008A3020008A3020008AA
:1002A00002E000F000F8FEE772B63A4880F30888F2
:1002B000394880F3098839484EF60851CEF20001DA
:1002C000086040F20000CCF200004EF63471CEF22D
:1002D00000010860BFF34F8FBFF36F8F40F2000043
:1002E000C0F2F0004EF68851CEF200010860BFF374
:1002F0004F8FBFF36F8F4FF00000E1EE100A4EF604
:100300003C71CEF200010860062080F31488BFF330
:100310006F8F02F0AFF802F051F802F0EBFF4FF0F0
:1003200055301F491B4A91423CBF41F8040BFAE784
:100330001C49194A91423CBF41F8040BFAE71A499B
:100340001A4A1B4B9A423EBF51F8040B42F8040B69
:10035000F8E700201749184A91423CBF41F8040BC6
:10036000FAE702F069F803F049F8144C144DAC4276
:1003700003DA54F8041B8847F9E700F041F8114C00
:10038000114DAC4203DA54F8041B8847F9E702F038
:1003900051B80000000600200022002000000008E4
:1003A0000000002000060020003D00080022002080
:1003B0005C220020602200207C420020A002000875
:1003C000A0020008A0020008A00200082DE9F04FDA
:1003D0002DED108AC1F80CD0D0F80CD0BDEC108AED
:1003E000BDE8F08F002383F311882846A047002042
:1003F00001F068FBFEE701F0E3FA00DFFEE7000032
:1004000038B500F0CDFC30B1164B00220E211A7227
:100410005A729972DA7201F02FFF054601F062FFFD
:100420000446D0B9104B9D4219D001339D4241F290
:10043000883512BF044600250124002001F026FF64
:100440000CB100F059F800F045FD00F0E3FB284640
:1004500000F004F900F050F8F9E70025EDE7054653
:10046000EBE700BF00220020010007B008B500F054
:10047000A3FBA0F120035842584108BD07B541F243
:100480001203022101A8ADF8043000F0B3FB03B061
:100490005DF804FB202310B583F311881248C3686C
:1004A0000BB101F095FB0023104A4FF47A710E480E
:1004B00001F052FB002383F311880D4C236813B124
:1004C0002368013B2360636813B16368013B636089
:1004D000084B1B7833B9636823B9022000F074FC21
:1004E0003223636010BD00BF602200209504000825
:1004F0007C23002074220020F8B5514B514A1C4641
:100500001968013100F09B8004339342F8D162688E
:100510004D4B9A4240F293804C4B9B6803F1006331
:1005200003F500339A4280F08A80002000F098FBA7
:100530000220474B187000F03DFC464B0021D3F8D9
:10054000E820C3F8E810D3F81021C3F81011D3F84D
:100550001021D3F8EC20C3F8EC10D3F81421C3F821
:100560001411D3F81421D3F8F020C3F8F010D3F805
:100570001821C3F81811D3F81821D3F8802042F0BD
:100580000062C3F88020D3F8802022F00062C3F814
:100590008020D3F88020D3F8802042F00072C3F886
:1005A0008020D3F8802022F00072C3F88020D3F896
:1005B000803072B64FF0E023C3F8084DD4E9000450
:1005C000BFF34F8FBFF36F8F234AC2F88410BFF37E
:1005D0004F8F536923F480335361BFF34F8FD2F8A9
:1005E000803043F6E076C3F3C905C3F34E335B01B5
:1005F00003EA060C29464CEA81770139C2F8747285
:10060000F9D2203B13F1200FF2D1BFF34F8FBFF38C
:100610006F8FBFF34F8FBFF36F8F536923F4003396
:1006200053610023C2F85032BFF34F8FBFF36F8F77
:10063000202383F31188854680F308882047F8BD7E
:100640000000020820000208FFFF0108002200202D
:10065000742200200044025800ED00E02DE9F04F24
:1006600093B0A94B2022FF2100900AA89D6800F0BA
:10067000DBFBA64A1378A3B90121A5481170C3601A
:10068000202383F31188C3680BB101F0A1FA002382
:10069000A04A4FF47A719E4801F05EFA002383F37A
:1006A0001188009B9C4A03B1136000239B49009C66
:1006B00098469B461E469A460B705360012000F0F8
:1006C00079FB24B1944B1B68002B00F016820020AC
:1006D00000F072FA0390039B002BF2DB012000F084
:1006E00061FB039B213B162BE8D801A252F823F0B3
:1006F0004D0700087507000809080008BD06000836
:10070000BD060008BD0600089D0800086F0A000825
:1007100089090008EB090008130A0008390A0008D3
:10072000BD0600084B0A0008BD060008BD0A000807
:10073000ED070008BD060008010B00085907000876
:10074000ED070008BD060008EB0900080220FFF7CE
:100750008DFE002840F0FB81009B022105A8B8F126
:10076000000F08BF1C4641F21233ADF8143000F000
:1007700041FAA3E74FF47A7000F01EFA071EEBDB94
:100780000220FFF773FE0028E6D0013F052F00F29C
:10079000E081DFE807F0030A0D101336052304217A
:1007A00005A8059300F026FA17E004215648F9E75A
:1007B00004215B48F6E704215A48F3E74FF01C098F
:1007C000484609F1040900F04DFA0421059005A8F6
:1007D00000F010FAB9F12C0FF2D101204FF0000A0D
:1007E00000FA07F747EA0B0B5FFA8BFB00F068FB98
:1007F00026B10BF00B030B2B08BF0024FFF73EFEC6
:100800005CE704214848CDE7002EA5D00BF00B0390
:100810000B2BA1D10220FFF729FE074600289BD011
:1008200001203E4E00F01CFA4FF00008022030700C
:1008300000F0C0FA5FFA88F9484600F021FA044651
:1008400090B1484608F1010800F02AFA0028F1D1D9
:10085000B846044641F21213022105A83E46ADF8FF
:10086000143000F0C7F929E7012325460220337030
:1008700000F098FA244B9B68AB4207D9284600F059
:10088000F1F9013040F068810435F3E70025234B8E
:10089000B8463E461D70204B5D60A7E7002E3FF432
:1008A0005BAF0BF00B030B2B7FF456AF02201B4BFF
:1008B000187000F07FFA322000F07EF9B0F10009E4
:1008C000FFF64AAF19F003077FF446AF0E4A09EB73
:1008D0000503926893423FF63FAFB9F5807F3FF73B
:1008E0003BAF124BB945019322DD4FF47A7000F013
:1008F00063F90390039A002AFFF62EAF039A01379B
:10090000019B03F8012BEDE7002200207823002053
:1009100060220020950400087C230020742200201F
:1009200004220020082200200C220020782200202F
:10093000C820FFF79BFD074600283FF40DAF1F2D91
:1009400011D8C5F120020AAB25F0030084494A45BD
:10095000184428BF4A46019200F040FA019AFF214C
:100960007F4800F061FA4FEAA903C9F387027C4986
:100970002846019300F060FA064600283FF46AAF6B
:10098000019B05EB830531E70220FFF76FFD00288F
:100990003FF4E2AE00F0A0F900283FF4DDAE0027FE
:1009A000B946704B9B68BB4218D91F2F11D80A9BC0
:1009B00001330ED027F0030312AA134453F8203C4E
:1009C00005934846042205A9043700F0F1FA814650
:1009D000E7E7384600F046F90590F2E7CDF81490C5
:1009E000042105A800F006F900E70023642104A80B
:1009F000049300F0F5F800287FF4AEAE0220FFF774
:100A000035FD00283FF4A8AE049800F05BF905908E
:100A1000E6E70023642104A8049300F0E1F800282D
:100A20007FF49AAE0220FFF721FD00283FF494AE38
:100A3000049800F049F9EAE70220FFF717FD0028C3
:100A40003FF48AAE00F058F9E1E70220FFF70EFD0F
:100A500000283FF481AE05A9142000F053F90746A1
:100A60000421049004A800F0C5F83946B9E7322003
:100A700000F0A2F8071EFFF66FAEBB077FF46CAE66
:100A8000384A07EB0A03926893423FF665AE0220AC
:100A9000FFF7ECFC00283FF45FAE27F00307574454
:100AA000BA453FF4A3AE50460AF1040A00F0DAF862
:100AB0000421059005A800F09DF8F1E74FF47A7045
:100AC000FFF7D4FC00283FF447AE00F005F90028FA
:100AD00044D00A9B01330BD008220AA9002000F061
:100AE000ABF900283AD02022FF210AA800F09CF997
:100AF000FFF7C4FC1C4800F0EBFF13B0BDE8F08F1B
:100B0000002E3FF429AE0BF00B030B2B7FF424AE29
:100B10000023642105A8059300F062F80746002829
:100B20007FF41AAE0220FFF7A1FC814600283FF4B3
:100B300013AEFFF7A3FC41F2883000F0C9FF05981F
:100B400000F0F2F94E463C4600F0BAF9B6E506462A
:100B50004CE64FF0000AFFE5B8467BE6374679E6FB
:100B60007822002000220020A08601000F4B70B5E3
:100B70001B780C460133DBB2012B11D80C4D4FF41E
:100B80007A732968A2FB033222460E6A0146284680
:100B9000B047844204D1074B002201201A7070BD77
:100BA0004FF4FA7000F094FF0020F8E710220020C4
:100BB00070250020B0230020002307B50246012144
:100BC0000DF107008DF80730FFF7D0FF20B19DF839
:100BD000070003B05DF804FB4FF0FF30F9E70000B9
:100BE0000A46042108B5FFF7C1FF80F00100C0B23A
:100BF000404208BD30B4054C0A46014623682046F1
:100C0000DD69034BAC4630BC604700BF7025002057
:100C1000A086010070B5104C0025104E01F004FABA
:100C200020803068238883420CD800252088013832
:100C300001F0F6F923880544013BB5F5802F2380A8
:100C4000F4D370BD01F0ECF9336805440133B5F518
:100C5000003F3360E5D3E8E7B2230020842300207F
:100C600001F0C0BA00F1006000F500300068704784
:100C700000F10060920000F5003001F037BA00008A
:100C8000054B1A68054B1B889B1A834202D91044F6
:100C900001F0C6B90020704784230020B223002051
:100CA00038B5074D04462868204401F0BFF928B93B
:100CB00028682044BDE8384001F0CAB938BD00BFFB
:100CC000842300200020704700F1FF5000F58F10B2
:100CD000D0F8000870470000064991F8243033B17D
:100CE00000230822086A81F82430FFF7C1BF0120E1
:100CF000704700BF88230020014B1868704700BF71
:100D00000010005C244BF0B51A680446234BC2F374
:100D10000B06120C1F885868BE4293F9085028D061
:100D20009F89BE4206D101200C2505FB003358687F
:100D300093F9085041F201039A421CD041F2030397
:100D40009A421AD042F201039A4218D042F20303A7
:100D50009A4208BF5625621E0B46441E0A4493421F
:100D60000FD214F9016F581C6EB1034600F8016CE4
:100D7000F5E70020D8E75A25EDE75925EBE7582598
:100D8000E9E7184605E02C2482421C7001D9981C22
:100D90005D70401AF0BD00BF0010005C14220020FE
:100DA00000207047022802D1014B04229A6170474B
:100DB00000080258022803D1024B4FF480229A61A6
:100DC000704700BF00080258022804D1024A536944
:100DD00083F004035361704700080258002310B5E4
:100DE000934203D0CC5CC4540133F9E710BD00003A
:100DF000013810B510F9013F3BB191F900409C4218
:100E000003D11AB10131013AF4E71AB191F9002086
:100E1000981A10BD1046FCE703460246D01A12F994
:100E2000011B0029FAD1704702440346934202D0C5
:100E300003F8011BFAE770472DE9F8431F4D1446EC
:100E40000746884695F8242052BBDFF870909CB383
:100E500095F824302BB92022FF2148462F62FFF756
:100E6000E3FF95F824004146C0F1080205EB80003D
:100E7000A24228BF2246D6B29200FFF7AFFF95F8F4
:100E80002430A41B17441E449044E4B2F6B2082E4A
:100E900085F82460DBD1FFF71FFF0028D7D108E0D9
:100EA0002B6A03EB82038342CFD0FFF715FF0028A4
:100EB000CBD10020BDE8F8830120FBE78823002088
:100EC000024B1A78024B1A70704700BFB023002003
:100ED0001022002010B5104C104800F0FBF82146FD
:100EE0000E4800F023F924680D48D4F89020D2F879
:100EF000043843F00203C2F8043800F0E9FD094960
:100F0000204600F021FAD4F89020D2F8043823F0DB
:100F10000203C2F8043810BDE03A00087025002032
:100F200040420F00E83A00087047000000B59BB04F
:100F3000EFF3098168226846FFF750FFEFF305835E
:100F4000044B9A6BDA6A9A6A9A6A9A6A9A6A9A6AF5
:100F50009B6AFEE700ED00E000B59BB0EFF309816E
:100F600068226846FFF73AFFEFF30583044B9A6B5C
:100F70009A6A9A6A9A6A9A6A9A6A9B6AFEE700BFB4
:100F800000ED00E000B59BB0EFF3098168226846F0
:100F9000FFF724FFEFF30583034B5A6B9A6A9A6AB3
:100FA0009A6A9A6A9B6AFEE700ED00E0FEE700009D
:100FB00030B50A44084D91420DD011F8013B58401C
:100FC000082340F30004013B2C4013F0FF0384EAA4
:100FD0005000F6D1EFE730BD2083B8ED02684368DA
:100FE0001143016003B118477047000013B5406B0F
:100FF00000F58054D4F8A4381A681178042914D163
:10100000017C022911D11979012312898B401342E5
:101010000BD101A94C3002F06DF8D4F8A448024677
:10102000019B2179206800F0DFF902B010BD0000BB
:10103000143001F0EFBF00004FF0FF33143001F027
:10104000E9BF00004C3002F0C1B800004FF0FF33A0
:101050004C3002F0BBB80000143001F0BDBF0000FE
:101060004FF0FF31143001F0B7BF00004C3002F0F8
:101070008DB800004FF0FF324C3002F087B800000E
:101080000020704710B500F58054D4F8A4381A68D1
:101090001178042917D1017C022914D1597901232F
:1010A00052898B4013420ED1143001F04FFF02469B
:1010B00048B1D4F8A4484FF4407361792068BDE882
:1010C000104000F07FB910BD406BFFF7DBBF0000A0
:1010D000704700007FB5124B0125042604460360CB
:1010E0000023057400F1840243602946C0E90233FD
:1010F0000C4B0290143001934FF44073009601F0B2
:1011000001FF094B04F69442294604F14C00029475
:10111000CDE900634FF4407301F0C8FF04B070BD27
:101120001C3A0008C9100008ED0F00080A682023C7
:1011300083F311880B790B3342F823004B79133377
:1011400042F823008B7913B10B3342F8230000F5EA
:101150008053C3F8A41802230374002383F3118877
:101160007047000038B5037F044613B190F854303F
:10117000ABB90125201D0221FFF730FF04F1140057
:101180006FF00101257700F0CBFC04F14C0084F8EE
:1011900054506FF00101BDE8384000F0C1BC38BDCB
:1011A00010B5012104460430FFF718FF0023237710
:1011B00084F8543010BD000038B5044600251430C2
:1011C00001F0B8FE04F14C00257701F087FF201DE7
:1011D00084F854500121FFF701FF2046BDE8384054
:1011E000FFF750BF90F8803003F06003202B06D14A
:1011F00090F881200023212A03D81F2A06D8002036
:101200007047222AFBD1C0E91D3303E0034A42673D
:1012100007228267C3670120704700BF2C2200208D
:1012200037B500F58055D5F8A4381A681178042927
:101230001AD1017C022917D11979012312898B4017
:10124000134211D100F14C04204602F007F858B1C6
:1012500001A9204601F04EFFD5F8A4480246019BA3
:101260002179206800F0C0F803B030BD01F10B0314
:10127000F0B550F8236085B004460D46FEB120233A
:1012800083F3118804EB8507301D0821FFF7A6FEC4
:10129000FB6806F14C005B691B681BB1019001F013
:1012A00037FF019803A901F025FF024648B1039BCF
:1012B0002946204600F098F8002383F3118805B0F2
:1012C000F0BDFB685A691268002AF5D01B8A013B01
:1012D0001340F1D104F18002EAE70000133138B580
:1012E00050F82140ECB1202383F3118804F580539A
:1012F000D3F8A4281368527903EB8203DB689B6957
:101300005D6845B104216018FFF768FE294604F1C5
:10131000140001F025FE2046FFF7B4FE002383F3FE
:10132000118838BD7047000001F018B90123402230
:10133000002110B5044600F8303BFFF775FD00238F
:10134000C4E9013310BD000010B52023044683F327
:1013500011882422416000210C30FFF765FD2046F2
:1013600001F01EF902232370002383F3118810BDBE
:1013700070B500EB8103054650690E461446DA60ED
:1013800018B110220021FFF74FFDA06918B11022FB
:101390000021FFF749FD31462846BDE8704001F0C5
:1013A00011BA000083682022002103F0011310B558
:1013B000044683601030FFF737FD2046BDE810403B
:1013C00001F08CBAF0B4012500EB810447898D400F
:1013D000E4683D43A469458123600023A260636003
:1013E000F0BC01F0A9BA0000F0B4012500EB8104C3
:1013F00007898D40E4683D436469058123600023CB
:10140000A2606360F0BC01F01FBB000070B5022356
:1014100000250446242203702946C0F888500C3069
:1014200040F8045CFFF700FD204684F8705001F09E
:101430005DF963681B6823B129462046BDE870400A
:10144000184770BD037880F88C300523037043681B
:101450001B6810B504460BB1042198470023A36014
:1014600010BD000090F88C20436802701B680BB11F
:10147000052118477047000070B590F87030044699
:1014800013B1002380F8703004F18002204601F08F
:1014900049FA63689B68B3B994F8803013F060052B
:1014A00035D00021204601F0F3FC0021204601F058
:1014B000E3FC63681B6813B10621204698470623A6
:1014C00084F8703070BD204698470028E4D0B4F806
:1014D0008630A26F9A4288BFA36794F98030A56FC7
:1014E000002B4FF0200380F20381002D00F0F280EA
:1014F000092284F8702083F3118800212046D4E962
:101500001D23FFF771FF002383F31188DAE794F8B6
:10151000812003F07F0343EA022340F20232934228
:1015200000F0C58021D8B3F5807F48D00DD8012BBD
:101530003FD0022B00F09380002BB2D104F188023F
:1015400062670222A267E367C1E7B3F5817F00F01B
:101550009B80B3F5407FA4D194F88230012BA0D1B9
:10156000B4F8883043F0020332E0B3F5006F4DD099
:1015700017D8B3F5A06F31D0A3F5C063012B90D875
:101580006368204694F882205E6894F88310B4F86B
:101590008430B047002884D0436863670368A3673A
:1015A0001AE0B3F5106F36D040F6024293427FF452
:1015B00078AF5C4B63670223A3670023C3E794F80B
:1015C0008230012B7FF46DAFB4F8883023F0020332
:1015D000A4F88830C4E91D55E56778E7B4F8803091
:1015E000B3F5A06F0ED194F88230204684F88A308B
:1015F00001F0DAF863681B6813B1012120469847AF
:10160000032323700023C4E91D339CE704F18B03FB
:1016100063670123C3E72378042B10D1202383F3CE
:1016200011882046FFF7BEFE85F311880321636809
:1016300084F88B5021701B680BB12046984794F8B2
:101640008230002BDED084F88B3004232370636853
:101650001B68002BD6D0022120469847D2E794F889
:10166000843020461D0603F00F010AD501F04CF925
:10167000012804D002287FF414AF2B4B9AE72B4BA0
:1016800098E701F033F9F3E794F88230002B7FF408
:1016900008AF94F8843013F00F01B3D01A06204637
:1016A00002D501F00DFCADE701F0FEFBAAE794F8CE
:1016B0008230002B7FF4F5AE94F8843013F00F01E4
:1016C000A0D01B06204602D501F0E2FB9AE701F00C
:1016D000D3FB97E7142284F8702083F311882B46FC
:1016E0002A4629462046FFF76DFE85F31188E9E674
:1016F0005DB1152284F8702083F311880021204603
:10170000D4E91D23FFF75EFEFDE60B2284F870206E
:1017100083F311882B462A4629462046FFF764FEAC
:10172000E3E700BF4C3A0008443A0008483A000892
:1017300038B590F870300446002B3ED0063BDAB244
:101740000F2A34D80F2B32D8DFE803F037313108B5
:10175000223231313131313131313737856FB0F8A3
:1017600086309D4214D2C3681B8AB5FBF3F203FB9B
:1017700012556DB9202383F311882B462A4629463A
:10178000FFF732FE85F311880A2384F870300EE0EB
:10179000142384F87030202383F31188002320461B
:1017A0001A461946FFF70EFE002383F3118838BD51
:1017B000C36F03B198470023E7E70021204601F0FB
:1017C00067FB0021204601F057FB63681B6813B1DB
:1017D0000621204698470623D7E7000010B590F869
:1017E00070300446142B29D017D8062B05D001D809
:1017F0001BB110BD093B022BFBD80021204601F094
:1018000047FB0021204601F037FB63681B6813B1DA
:10181000062120469847062319E0152BE9D10B2312
:1018200080F87030202383F3118800231A4619466C
:10183000FFF7DAFD002383F31188DAE7C3689B69B9
:101840005B68002BD5D1C36F03B19847002384F8A0
:101850007030CEE7024B0022C3E900339A60704734
:10186000B4230020002382680374054B1B68996829
:101870009142FBD25A680360426010605860704722
:10188000B423002008B5202383F31188037C032BA5
:1018900005D0042B0DD02BB983F3118808BD436903
:1018A00000221A604FF0FF334361FFF7DBFF002394
:1018B000F2E7D0E9003213605A60F3E70023826850
:1018C0000374054B1B6899689142FBD85A68036002
:1018D0004260106058607047B4230020054B1969BE
:1018E00008741868026853601A6018610123037451
:1018F000FEF76CBDB42300204B1C30B5044687B006
:101900000A4D10D02B6901A8094A00F025F920469C
:10191000FFF7E4FF049B13B101A800F059F92B690C
:10192000586907B030BDFFF7D9FFF8E7B4230020AE
:101930008518000838B50C4D044641612B69816853
:101940009A68914203D8BDE83840FFF78BBF18462C
:10195000FFF7B4FF01232C61014623742046BDE844
:101960003840FEF733BD00BFB4230020044B1A6893
:101970001B6990689B68984294BF002001207047C3
:10198000B423002010B5084C236820691A685460FD
:101990002260012223611A74FFF790FF014620693B
:1019A000BDE81040FEF712BDB423002008B5FFF7D4
:1019B000DDFF18B1BDE80840FFF7E4BF08BD000037
:1019C000FFF7E0BFFEE7000010B50C4CFFF742FF49
:1019D00000F0B4F880220A49204600F03BF80123C9
:1019E00044F8180C037400F097FC002383F311886B
:1019F00062B60448BDE8104000F04CB8DC2300207B
:101A0000503A0008603A000800F01CB9EFF311806A
:101A100020B9EFF30583202282F31188704700007C
:101A200010B530B9EFF30584C4F3080414B180F3A2
:101A3000118810BDFFF7BAFF84F31188F9E70000A1
:101A4000034A516853685B1A9842FBD8704700BF3D
:101A5000001000E082600222028270478368A3F1D6
:101A60007C0243F80C2C026943F83C2C426943F891
:101A7000382C074A43F81C2CC268A3F1180043F81D
:101A8000102C022203F8082C002203F8072C7047C0
:101A9000E503000810B5202383F31188FFF7DEFF6C
:101AA00000210446FFF746FF002383F311882046F8
:101AB00010BD0000024B1B6958610F20FFF70EBFDD
:101AC000B4230020202383F31188FFF7F3BF000025
:101AD00008B50146202383F311880820FFF70CFF87
:101AE000002383F3118808BD49B1064B42681B6986
:101AF00018605A60136043600420FFF7FDBE4FF08A
:101B0000FF307047B42300200368984206D01A685B
:101B10000260506018465961FFF7A4BE704700008C
:101B200038B504460D462068844200D138BD0368AC
:101B300023605C604561FFF795FEF4E7054B4FF0CD
:101B4000FF3103F11402C3E905220022C3E90712A1
:101B5000704700BFB423002070B51C4E05460C46EC
:101B6000C0E9032301F0B0FB334653F8142F9A4227
:101B70000DD130620A2C2CBF00190A302A60C5E949
:101B80000124C6E90555BDE8704001F087BB316A04
:101B9000431AE31838BF1C469368A34202D90819B8
:101BA00001F08CFB73699A6894420CD85A68AC6057
:101BB0002B606A6015609A685D60121B9A604FF036
:101BC000FF33F36170BDA41A1B68ECE7B423002057
:101BD00038B51B4C636998420DD08168D0E900325A
:101BE00013605A600022C2609A680A449A604FF0FB
:101BF000FF33E36138BD03682246002142F8143FF9
:101C000093425A60C16003D1BDE8384001F050BB37
:101C10009A688168256A0A449A6001F055FB6369F5
:101C2000411B9A688A42E5D9AB181D1A206A092D12
:101C300098BF01F10A02BDE83840104401F03EBBF4
:101C4000B42300202DE9F041184C002704F11406BC
:101C5000656901F039FB236AAA68C11A8A4215D85E
:101C60001344D5F80C802362D5E9003213605A6022
:101C70006369EF60B34201D101F01AFB87F3118869
:101C80002869C047202383F31188E1E76169B142E5
:101C900009D013441B1ABDE8F0410A2B2CBFC01811
:101CA0000A3001F00BBBBDE8F08100BFB423002077
:101CB00000207047FEE70000704700004FF0FF3043
:101CC0007047000002290CD0032904D001290748DD
:101CD00018BF00207047032A05D8054800EBC20052
:101CE0007047044870470020704700BF443B00081D
:101CF0003C220020F83A000870B59AB00546084624
:101D0000144601A900F0C2F801A8FFF785F8431CAA
:101D10000022C6B25B001046C5E9003423700323DD
:101D2000023404F8013C01ABD1B202348E4201D836
:101D30001AB070BD13F8011B013204F8010C04F84D
:101D4000021CF1E708B5202383F311880348FFF74D
:101D500067FA002383F3118808BD00BF70250020B7
:101D600090F8803003F01F02012A07D190F88120FB
:101D70000B2A03D10023C0E91D3315E003F06003F3
:101D8000202B08D1B0F884302BB990F88120212A7B
:101D900003D81F2A04D8FFF725BA222AEBD0FAE786
:101DA000034A426707228267C3670120704700BF6A
:101DB0003322002007B5052917D8DFE801F01916EE
:101DC00003191920202383F31188104A012101905F
:101DD000FFF7CEFA019802210D4AFFF7C9FA0D4824
:101DE000FFF7EAF9002383F3118803B05DF804FBE1
:101DF000202383F311880748FFF7B4F9F2E7202383
:101E000083F311880348FFF7CBF9EBE7983A000812
:101E1000BC3A00087025002038B50C4D0C4C2A4601
:101E20000C4904F10800FFF767FF05F1CA0204F14D
:101E300010000949FFF760FF05F5CA7204F11800A8
:101E40000649BDE83840FFF757BF00BF483E0020B5
:101E50003C220020783A0008823A00088D3A0008B7
:101E600070B5044608460D46FEF7D6FFC6B22046BA
:101E7000013403780BB9184670BD32462946FEF787
:101E8000B7FF0028F3D10120F6E700002DE9F04765
:101E900005460C46FEF7C0FF2B49C6B22846FFF7A1
:101EA000DFFF08B10736F6B228492846FFF7D8FF0A
:101EB00008B11036F6B2632E0BD8DFF88C80DFF84D
:101EC0008C90234FDFF894A02E7846B92670BDE899
:101ED000F08729462046BDE8F04701F089BD252E50
:101EE0002ED1072241462846FEF782FF70B9194BD2
:101EF000224603F10C0153F8040B8B4242F8040B09
:101F0000F9D11B8807350E341380DDE708224946D6
:101F10002846FEF76DFF98B9A21C0F4B19780232C4
:101F20000909C95D02F8041C13F8011B01F00F0137
:101F30005345C95D02F8031CF0D118340835C3E7D6
:101F4000013504F8016BBFE7643B00088D3A0008D7
:101F50007B3B00086C3B000800E8F11F0CE8F11F18
:101F6000BFF34F8F044B1A695107FCD1D3F81021EE
:101F70005207F8D1704700BF0020005208B50D4B42
:101F80001B78ABB9FFF7ECFF0B4BDA68D10704D530
:101F90000A4A5A6002F188325A60D3F80C21D207FB
:101FA00006D5064AC3F8042102F18832C3F8042199
:101FB00008BD00BFA6400020002000522301674555
:101FC00008B5114B1B78F3B9104B1A69510703D5AB
:101FD000DA6842F04002DA60D3F81021520705D5E2
:101FE000D3F80C2142F04002C3F80C21FFF7B8FFF0
:101FF000064BDA6842F00102DA60D3F80C2142F0B5
:102000000102C3F80C2108BDA640002000200052A8
:102010000F289ABF00F58060400400207047000040
:102020004FF4003070470000102070470F2808B5AB
:102030000BD8FFF7EDFF00F500330268013204D141
:1020400004308342F9D1012008BD0020FCE70000E4
:102050000F2870B5054645D8FFF7D8FC224CFFF78E
:102060007FFF0646FFF78AFF4FF0FF33072D6361BE
:10207000C4F8143120D82361FFF772FF2B0243F01C
:102080002403E360E36843F08003E36023695A07B5
:10209000FCD42846FFF764FF4FF40031FFF7B8FF88
:1020A00000F002F93046FFF78BFFFFF7B9FC284636
:1020B000BDE87040FFF7BABFC4F81031FFF750FF1A
:1020C000A5F108031B0243F02403C4F80C31D4F833
:1020D0000C3143F08003C4F80C31D4F810315B07A5
:1020E000FBD4D6E7002070BD002000522DE9F84F48
:1020F00040EA020305460C461746D80602D00020E7
:10210000BDE8F88F27F01F07DFF8D4B0FFF736FFE0
:102110002744BC4203D10120FFF752FFF0E7202201
:102120002946204601F054FC10B920352034F0E750
:102130002B4605F120021E68711CE0D104339A423F
:10214000F9D1FFF763FC05F17843234AB3F5801F0B
:10215000224B28BF9A4603F1040338BF9046A2F1F0
:10216000080228BF9846A3F108033ABF9146DA4611
:102170009946FFF7F5FEC8F80060A5EB040CD9F806
:10218000002004F11C0142F00202C9F80020221FC5
:10219000DAF8006016F00506FAD152F8043F8A42D8
:1021A0004CF80230F4D1BFF34F8FFFF7D9FE4FF058
:1021B000FF32C8F80020D9F8002022F00202C9F846
:1021C0000020FFF72DFC20222146284601F000FCCC
:1021D0000028AAD030469FE7142000521021005258
:1021E0001020005210B5084C237828B11BB9FFF716
:1021F000C5FE0123237010BD002BFCD02070BDE86C
:102200001040FFF7DDBE00BFA64000200244074B90
:10221000D2B210B5904200D110BD441C00B253F8A8
:10222000200041F8040BE0B2F4E700BF5040005832
:102230000E4B30B51C6F240405D41C6F1C671C6F3B
:1022400044F400441C670A4C02442368D2B243F4AD
:1022500080732360074B904200D130BD441C51F87D
:10226000045B00B243F82050E0B2F4E700440258A7
:10227000004802585040005807B5012201A900202B
:10228000FFF7C4FF019803B05DF804FB13B50446E3
:10229000FFF7F2FFA04205D0012201A9002001941E
:1022A000FFF7C6FF02B010BD0144BFF34F8F064BCE
:1022B000884204D3BFF34F8FBFF36F8F7047C3F8CB
:1022C0005C022030F4E700BF00ED00E0034B1A6829
:1022D0001AB9034AD2F8D0241A607047A8400020E7
:1022E0000040025808B5FFF7F1FF024B1868C0F331
:1022F000806008BDA8400020EFF3098305496833DA
:102300004A6B22F001024A6383F30988002383F3B6
:102310001188704700EF00E0202080F3118862B63A
:102320000D4B0E4AD96821F4E0610904090C0A43F7
:102330000B49DA60D3F8FC2042F08072C3F8FC202D
:10234000084AC2F8B01F116841F001011160102263
:10235000DA7783F82200704700ED00E00003FA0509
:1023600055CEACC5001000E0202310B583F31188D2
:102370000E4B5B6813F4006314D0F1EE103AEFF3E8
:1023800009844FF08073683CE361094BDB6B236683
:1023900084F30988FFF7EAFA10B1064BA36110BD78
:1023A000054BFBE783F31188F9E700BF00ED00E080
:1023B00000EF00E0F7030008FA03000870B5BFF370
:1023C0004F8FBFF36F8F1A4A0021C2F85012BFF32C
:1023D0004F8FBFF36F8F536943F400335361BFF3E3
:1023E0004F8FBFF36F8FC2F88410BFF34F8FD2F8B7
:1023F000803043F6E074C3F3C900C3F34E335B018E
:1024000003EA0406014646EA81750139C2F86052C2
:10241000F9D2203B13F1200FF2D1BFF34F8F536954
:1024200043F480335361BFF34F8FBFF36F8F70BDA1
:1024300000ED00E0FEE700000A4B0B480B4A90421B
:102440000BD30B4BC11EDA1C121A22F003028B4273
:1024500038BF00220021FEF7E7BC53F8041B40F808
:10246000041BECE75C3D00087C4200207C4200201D
:102470007C4200207047000070B5D0E92443002260
:102480004FF0FF359E6804EB42135101D3F8000969
:10249000002805DAD3F8000940F08040C3F80009AD
:1024A000D3F8000B002805DAD3F8000B40F0804089
:1024B000C3F8000B013263189642C3F80859C3F8F9
:1024C000085BE0D24FF00113C4F81C3870BD000067
:1024D00000EB8103D3F80CC02DE9F043DCF81420A5
:1024E0004E1CD0F89050D2F800E005EB063605EB14
:1024F0004118506870450AD30122D5F8343802FAE1
:1025000001F123EA0101C5F83418BDE8F083AEEB10
:102510000003BCF81040A34228BF2346D8F818494E
:10252000A4B2B3EB840FF0D89468A4F1040959F86D
:10253000047F3760A4EB09071F44042FF7D81C441D
:10254000034494605360D4E7890141F020010161A4
:1025500003699B06FCD41220FFF772BA10B50A4C2F
:102560002046FEF7E3FE094BC4F89030084BC4F850
:102570009430084C2046FEF7D9FE074BC4F8903043
:10258000064BC4F8943010BDAC4000200000084059
:10259000B03B00084841002000000440BC3B00085C
:1025A00070B503780546012B5DD1494BD0F89040BA
:1025B000984259D1474B0E216520D3F8D82042F0DC
:1025C0000062C3F8D820D3F8002142F00062C3F8BB
:1025D0000021D3F80021D3F8802042F00062C3F834
:1025E0008020D3F8802022F00062C3F88020D3F846
:1025F000803000F071FC384BE360384BC4F8003891
:102600000023D5F89060C4F8003EC02323604FF447
:102610000413A3633369002BFCDA01230C2033611C
:10262000FFF70EFA3369DB07FCD41220FFF708FA34
:102630003369002BFCDA00262846A660FFF71CFF52
:102640006B68C4F81068DB68C4F81468C4F81C68C8
:10265000002B3AD1224BA3614FF0FF336361A36893
:1026600043F00103A36070BD1E4B9842C8D1194BC3
:102670000E214D20D3F8D82042F00072C3F8D820A4
:10268000D3F8002142F00072C3F80021D3F80021F2
:10269000D3F8802042F00072C3F88020D3F8802065
:1026A00022F00072C3F88020D3F88020D3F8D8201D
:1026B00022F08062C3F8D820D3F8002122F0806293
:1026C000C3F80021D3F8003193E7074BC3E700BFFD
:1026D000AC40002000440258401400400300200297
:1026E000003C30C048410020083C30C0F8B5D0F86C
:1026F0009040054600214FF000662046FFF724FF7A
:10270000D5F8941000234FF001128F684FF0FF307E
:10271000C4F83438C4F81C2804EB431201339F4238
:10272000C2F80069C2F8006BC2F80809C2F8080BC9
:10273000F2D20B68D5F89020C5F898306362102368
:102740001361166916F01006FBD11220FFF778F915
:10275000D4F8003823F4FE63C4F80038A36943F4C6
:10276000402343F01003A3610923C4F81038C4F8D0
:1027700014380B4BEB604FF0C043C4F8103B094BCF
:10278000C4F8003BC4F81069C4F80039D5F8983093
:1027900003F1100243F48013C5F89820A362F8BD3A
:1027A0008C3B000840800010D0F8902090F88A10F0
:1027B000D2F8003823F4FE6343EA0113C2F800386C
:1027C000704700002DE9F84300EB8103D0F89050EA
:1027D0000C468046DA680FFA81F94801166806F05F
:1027E0000306731E022B05EB41134FF0000194BF4B
:1027F000B604384EC3F8101B4FF0010104F110036A
:1028000098BF06F1805601FA03F3916998BF06F567
:10281000004600293AD0578A04F15801374349014C
:102820006F50D5F81C180B430021C5F81C382B1825
:102830000127C3F81019A7405369611E9BB3138A7F
:10284000928B9B08012A88BF5343D8F89820981888
:1028500042EA034301F140022146C8F898002846A5
:1028600005EB82025360FFF76FFE08EB8900C36837
:102870001B8A43EA845348341E4364012E51D5F821
:102880001C381F43C5F81C78BDE8F88305EB4917D1
:10289000D7F8001B21F40041C7F8001BD5F81C181D
:1028A00021EA0303C0E704F13F030B4A284621460F
:1028B00005EB83035A60FFF747FE05EB4910D0F89C
:1028C000003923F40043C0F80039D5F81C3823EA56
:1028D0000707D7E70080001000040002D0F894201A
:1028E0001268C0F89820FFF7C7BD00005831D0F833
:1028F000903049015B5813F4004004D013F4001FDA
:102900000CBF0220012070474831D0F890304901B7
:102910005B5813F4004004D013F4001F0CBF0220D6
:102920000120704700EB8101CB68196A0B681360C6
:102930004B6853607047000000EB810330B5DD68E1
:10294000AA691368D36019B9402B84BF4023136070
:102950006B8A1468D0F890201C4402EB4110013CB3
:1029600009B2B4FBF3F46343033323F0030343EAF4
:10297000C44343F0C043C0F8103B2B6803F003038B
:10298000012B0ED1D2F8083802EB411013F4807FEE
:10299000D0F8003B14BF43F0805343F00053C0F81D
:1029A000003B02EB4112D2F8003B43F00443C2F873
:1029B000003B30BD2DE9F041D0F8906005460C4653
:1029C00006EB4113D3F8087B3A07C3F8087B08D518
:1029D000D6F814381B0704D500EB8103DB685B686D
:1029E0009847FA071FD5D6F81438DB071BD505EB37
:1029F0008403D968CCB98B69488A5A68B2FBF0F66F
:102A000000FB16228AB91868DA6890420DD2121AB1
:102A1000C3E90024202383F3118821462846FFF7C9
:102A20008BFF84F31188BDE8F081012303FA04F2DF
:102A30006B8923EA02036B81CB68002BF3D021461C
:102A40002846BDE8F041184700EB81034A0170B504
:102A5000DD68D0F890306C692668E66056BB1A4491
:102A60004FF40020C2F810092A6802F00302012A7C
:102A70000AB20ED1D3F8080803EB421410F4807F99
:102A8000D4F8000914BF40F0805040F00050C4F862
:102A9000000903EB4212D2F8000940F00440C2F8EA
:102AA00000090122D3F8340802FA01F10143C3F806
:102AB000341870BD19B9402E84BF402020602068B2
:102AC0001A442E8A8419013CB4FBF6F440EAC4404F
:102AD00040F00050C6E700002DE9F041D0F89060CA
:102AE00004460D4606EB4113D3F80879C3F808797C
:102AF000FB071CD5D6F81038DA0718D500EB810390
:102B0000D3F80CC0DCF81430D3F800E0DA6896454E
:102B10001BD2A2EB0E024FF000081A60C3F804802B
:102B2000202383F31188FFF78FFF88F311883B067A
:102B300018D50123D6F83428AB40134212D02946C9
:102B40002046BDE8F041FFF7C3BC012303FA01F2C0
:102B5000038923EA02030381DCF80830002BE6D066
:102B60009847E4E7BDE8F0812DE9F84FD0F89050A0
:102B700004466E69AB691E4016F480586E6103D03E
:102B8000BDE8F84FFEF742BC002E12DAD5F8003E41
:102B90009F0705D0D5F8003E23F00303C5F8003E9B
:102BA000D5F80438204623F00103C5F80438FEF7B1
:102BB00059FC300505D52046FFF75EFC2046FEF7A0
:102BC00041FCB1040CD5D5F8083813F0060FEB68BA
:102BD00023F470530CBF43F4105343F4A053EB6041
:102BE000320704D56368DB680BB120469847F302CF
:102BF00000F1BA80B70226D5D4F8909000274FF0A4
:102C0000010A09EB4712D2F8003B03F44023B3F565
:102C1000802F11D1D2F8003B002B0DDA62890AFA1D
:102C200007F322EA0303638104EB8703DB68DB68B5
:102C300013B13946204698470137D4F89430FFB293
:102C40009B689F42DDD9F00619D5D4F89000026A3E
:102C5000C2F30A1702F00F0302F4F012B2F5802F4C
:102C600000F0CC80B2F5402F09D104EB83030022A1
:102C700000F58050DB681B6A974240F0B280300359
:102C8000D5F8185835D5E90303D500212046FFF7BC
:102C900091FEAA0303D501212046FFF78BFE6B03AB
:102CA00003D502212046FFF785FE2F0303D503211C
:102CB0002046FFF77FFEE80203D504212046FFF7F8
:102CC00079FEA90203D505212046FFF773FE6A02AB
:102CD00003D506212046FFF76DFE2B0203D5072101
:102CE0002046FFF767FEEF0103D508212046FFF7D6
:102CF00061FE700340F1A980E90703D50021204659
:102D0000FFF7EAFEAA0703D501212046FFF7E4FEFC
:102D10006B0703D502212046FFF7DEFE2F0703D500
:102D200003212046FFF7D8FEEE0603D504212046F6
:102D3000FFF7D2FEA80603D505212046FFF7CCFEFB
:102D4000690603D506212046FFF7C6FE2A0603D5ED
:102D500007212046FFF7C0FEEB0576D52046082167
:102D6000BDE8F84FFFF7B8BED4F8909000274FF0B9
:102D7000010AD4F894305FFA87FB9B689B453FF6C5
:102D800039AF09EB4B13D3F8002902F44022B2F516
:102D9000802F24D1D3F80029002A20DAD3F8002983
:102DA00042F09042C3F80029D3F80029002AFBDB47
:102DB0005946D4F89000FFF7C7FB22890AFA0BF3B3
:102DC00022EA0303238104EB8B03DB689B6813B1C6
:102DD00059462046984759462046FFF779FB013768
:102DE000C7E7910701D1D0F80080072A02F101025C
:102DF0009CBF03F8018B4FEA18283DE704EB8303DF
:102E000000F58050DA68D2F818C0DCF80820DCE958
:102E1000001CA1EB0C0C00218F4208D1DB689B69E0
:102E20009A683A449A605A683A445A6027E711F01F
:102E3000030F01D1D0F800808C4501F1010184BF5E
:102E400002F8018B4FEA1828E6E7BDE8F88F00008A
:102E500008B50348FFF788FEBDE80840FFF784BACD
:102E6000AC40002008B50348FFF77EFEBDE80840EF
:102E7000FFF77ABA48410020D0F8903003EB4111B7
:102E8000D1F8003B43F40013C1F8003B7047000049
:102E9000D0F8903003EB4111D1F8003943F400131E
:102EA000C1F8003970470000D0F8903003EB4111B1
:102EB000D1F8003B23F40013C1F8003B7047000039
:102EC000D0F8903003EB4111D1F8003923F400130E
:102ED000C1F8003970470000090100F16043012288
:102EE00003F56143C9B283F8001300F01F039A4051
:102EF00043099B0003F1604303F56143C3F880215C
:102F00001A60704730B50433039C0172002104FB42
:102F10000325C160C0E90653049B0363059BC0E918
:102F20000000C0E90422C0E90842C0E90A11436375
:102F300030BD00000022416AC260C0E90411C0E94E
:102F40000A226FF00101FEF7EBBD0000D0E9043268
:102F5000934201D1C2680AB9181D7047002070471A
:102F6000036919600021C2680132C260C26913445A
:102F700082699342036124BF436A0361FEF7C4BDC3
:102F800038B504460D46E3683BB162690020131D65
:102F90001268A3621344E36207E0237A33B9294637
:102FA0002046FEF7A1FD0028EDDA38BD6FF00100E4
:102FB000FBE70000C368C269013BC3604369134477
:102FC00082699342436124BF436A43610023836261
:102FD000036B03B11847704770B52023044683F391
:102FE0001188866A3EB9FFF7CBFF054618B186F314
:102FF0001188284670BDA36AE26A13F8015B934208
:10300000A36202D32046FFF7D5FF002383F3118884
:10301000EFE700002DE9F84F04460E4617469846A4
:103020004FF0200989F311880025AA46D4F828B06A
:10303000BBF1000F09D141462046FFF7A1FF20B1A7
:103040008BF311882846BDE8F88FD4E90A12A7EB64
:10305000050B521A934528BF9346BBF1400F1BD96D
:10306000334601F1400251F8040B914243F8040B3E
:10307000F9D1A36A403640354033A362D4E90A232C
:103080009A4202D32046FFF795FF8AF31188BD428A
:10309000D8D289F31188C9E730465A46FDF79EFE1B
:1030A000A36A5E445D445B44A362E7E710B5029CFB
:1030B0000433017204FB0321C460C0E9061300233A
:1030C000C0E90A33039B0363049BC0E90000C0E925
:1030D0000422C0E90842436310BD0000026A6FF099
:1030E0000101C260426AC0E904220022C0E90A224A
:1030F000FEF716BDD0E904239A4201D1C26822B975
:10310000184650F8043B0B607047002070470000E1
:10311000C3680021C2690133C360436913448269F3
:103120009342436124BF436A4361FEF7EDBC000054
:1031300038B504460D46E3683BB1236900201A1DEB
:10314000A262E2691344E36207E0237A33B92946B5
:103150002046FEF7C9FC0028EDDA38BD6FF001000B
:10316000FBE7000003691960C268013AC260C269E6
:10317000134482699342036124BF436A03610023BD
:103180008362036B03B118477047000070B52023BA
:103190000D460446114683F31188866A2EB9FFF75F
:1031A000C7FF10B186F3118870BDA36A1D70A36AB2
:1031B000E26A01339342A36204D3E16920460439F1
:1031C000FFF7D0FF002080F31188EDE72DE9F84FDD
:1031D00004460D46904699464FF0200A8AF311881E
:1031E0000026B346A76A4FB949462046FFF7A0FF1D
:1031F00020B187F311883046BDE8F88FD4E90A077B
:103200003A1AA8EB0607974228BF1746402F1BD94A
:1032100005F1400355F8042B9D4240F8042BF9D1E9
:10322000A36A40364033A362D4E90A239A4204D306
:10323000E16920460439FFF795FF8BF31188464575
:10324000D9D28AF31188CDE729463A46FDF7C6FD63
:10325000A36A3D443E443B44A362E5E7D0E904232E
:103260009A4217D1C3689BB1836A8BB1043B9B1A06
:103270000ED01360C368013BC360C3691A448369FD
:103280009A42026124BF436A0361002383620123DF
:10329000184670470023FBE700F0DAB8034B002222
:1032A00058631A610222DA60704700BF000C0040C8
:1032B000014B0022DA607047000C0040014B58635C
:1032C000704700BF000C0040014B586A704700BFB8
:1032D000000C00404B6843608B688360CB68C36020
:1032E0000B6943614B6903628B6943620B6803603E
:1032F0007047000008B53C4B40F2FF713B48D3F8E3
:1033000088200A43C3F88820D3F8882022F4FF627B
:1033100022F00702C3F88820D3F88820D3F8E020F1
:103320000A43C3F8E020D3F808210A43C3F8082170
:103330002F4AD3F808311146FFF7CCFF00F5806023
:1033400002F11C01FFF7C6FF00F5806002F13801B1
:10335000FFF7C0FF00F5806002F15401FFF7BAFFEC
:1033600000F5806002F17001FFF7B4FF00F58060A6
:1033700002F18C01FFF7AEFF00F5806002F1A801B9
:10338000FFF7A8FF00F5806002F1C401FFF7A2FF7C
:1033900000F5806002F1E001FFF79CFF00F580601E
:1033A00002F1FC01FFF796FF02F58C7100F58060D9
:1033B000FFF790FF00F000F90E4BD3F8902242F097
:1033C0000102C3F89022D3F8942242F00102C3F81C
:1033D00094220522C3F898204FF06052C3F89C2035
:1033E000054AC3F8A02008BD004402580000025856
:1033F000C83B000800ED00E01F00080308B500F01E
:10340000C9FAFEF7E1FA0F4BD3F8DC2042F0400294
:10341000C3F8DC20D3F8042122F04002C3F80421D1
:10342000D3F80431084B1A6842F008021A601A688F
:1034300042F004021A60FEF749FFBDE80840FEF7BB
:10344000EBBC00BF0044025800180248704700005F
:10345000114BD3F8E82042F00802C3F8E820D3F873
:10346000102142F00802C3F810210C4AD3F81031A1
:10347000D36B43F00803D363C722094B9A624FF022
:10348000FF32DA6200229A615A63DA605A600122DE
:103490005A611A60704700BF004402580010005C77
:1034A000000C0040094A08B51169D3680B40D9B235
:1034B0009B076FEA0101116107D5202383F311886F
:1034C000FEF7A2FA002383F3118808BD000C004028
:1034D000384B4FF0FF31D3F88020C3F88010D3F879
:1034E00080200022C3F88020D3F88000D3F8840025
:1034F000C3F88410D3F88400C3F88420D3F8840080
:10350000D86F40F0FF4040F4FF0040F43F5040F0DF
:103510003F00D867D86F20F0FF4020F4FF0020F470
:103520003F5020F03F00D867D86FD3F888006FEA8B
:1035300040506FEA5050C3F88800D3F88800C0F3B9
:103540000A00C3F88800D3F88800D3F89000C3F8C5
:103550009010D3F89000C3F89020D3F89000D3F8DF
:103560009400C3F89410D3F89400C3F89420D3F8CF
:103570009400D3F89800C3F89810D3F89800C3F8D3
:103580009820D3F89800D3F88C00C3F88C10D3F8A7
:103590008C00C3F88C20D3F88C00D3F89C00C3F8BF
:1035A0009C10D3F89C10C3F89C20D3F89C3000F0FA
:1035B000C9B900BF00440258614B0122C3F8082179
:1035C000604BD3F8F42042F00202C3F8F420D3F8A1
:1035D0001C2142F00202C3F81C210222D3F81C3144
:1035E000594BDA605A689104FCD5584A1A60012296
:1035F0009A60574ADA6000221A614FF440429A6199
:10360000514B9A699204FCD51A6842F480721A6090
:103610004C4B1A6F12F4407F04D04FF480321A677B
:1036200000221A671A6842F001021A60454B1A68B4
:103630005007FCD500221A611A6912F03802FBD13A
:10364000012119604FF0804159605A67414ADA629E
:10365000414A1A611A6842F480321A60394B1A687A
:103660009103FCD51A6842F480521A601A689204D9
:10367000FCD53A4A3A499A6200225A631963394999
:10368000DA6399635A64384A1A64384ADA621A6803
:1036900042F0A8521A602B4B1A6802F02852B2F17D
:1036A000285FF9D148229A614FF48862DA6140229A
:1036B0001A622F4ADA644FF080521A652D4A5A6511
:1036C0002D4A9A6532232D4A1360136803F00F03C5
:1036D000022BFAD11B4B1A6942F003021A611A69D4
:1036E00002F03802182AFAD1D3F8DC2042F0005256
:1036F000C3F8DC20D3F8042142F00052C3F80421BF
:10370000D3F80421D3F8DC2042F08042C3F8DC2057
:10371000D3F8042142F08042C3F80421D3F80421F5
:10372000D3F8DC2042F00042C3F8DC20D3F80421B7
:1037300042F00042C3F80421D3F80431704700BFBF
:1037400000800051004402580048025800C000F0B8
:10375000020000010000FF01008890081210200004
:10376000630209012C02040047040508FD0BFF0158
:10377000200000200010E0000001010000200052A5
:103780004FF0B04208B5D2F8883003F00103C2F818
:10379000883023B1044A13680BB150689847BDE8DC
:1037A0000840FEF7E1BD00BFFC4100204FF0B042F1
:1037B00008B5D2F8883003F00203C2F8883023B18C
:1037C000044A93680BB1D0689847BDE80840FEF7FB
:1037D000CBBD00BFFC4100204FF0B04208B5D2F88D
:1037E000883003F00403C2F8883023B1044A136917
:1037F0000BB150699847BDE80840FEF7B5BD00BF62
:10380000FC4100204FF0B04208B5D2F8883003F0F8
:103810000803C2F8883023B1044A93690BB1D06918
:103820009847BDE80840FEF79FBD00BFFC4100205F
:103830004FF0B04208B5D2F8883003F01003C2F858
:10384000883023B1044A136A0BB1506A9847BDE827
:103850000840FEF789BD00BFFC4100204FF0B04397
:1038600010B5D3F8884004F47872C3F88820A30612
:1038700004D5124A936A0BB1D06A9847600604D502
:103880000E4A136B0BB1506B9847210604D50B4AB7
:10389000936B0BB1D06B9847E20504D5074A136CC4
:1038A0000BB1506C9847A30504D5044A936C0BB137
:1038B000D06C9847BDE81040FEF756BDFC41002093
:1038C0004FF0B04310B5D3F8884004F47C42C3F8FD
:1038D0008820620504D5164A136D0BB1506D9847C8
:1038E000230504D5124A936D0BB1D06D9847E004BF
:1038F00004D50F4A136E0BB1506E9847A10404D53E
:103900000B4A936E0BB1D06E9847620404D5084AF7
:10391000136F0BB1506F9847230404D5044A936F7B
:103920000BB1D06F9847BDE81040FEF71DBD00BF3A
:10393000FC41002008B5FFF7B5FDBDE80840FEF7E3
:1039400013BD0000062108B50846FFF7C5FA062199
:103950000720FFF7C1FA06210820FFF7BDFA06216C
:103960000920FFF7B9FA06210A20FFF7B5FA062168
:103970001720FFF7B1FA06212820FFF7ADFA092139
:103980007A20FFF7A9FA07213220BDE80840FFF7A7
:10399000A3BA000008B5FFF79BFD00F00BF8FDF798
:1039A000C3FCFDF795FBFFF751FDBDE80840FFF7AD
:1039B00073BC00000023054A19460133102BC2E9ED
:1039C000001102F10802F8D1704700BFFC4100204D
:1039D00010B501390244904201D1002005E003787E
:1039E00011F8014FA34201D0181B10BD0130F2E7BE
:1039F000034611F8012B03F8012B002AF9D1704777
:103A000053544D333248373F3F3F0053544D3332C8
:103A1000483734332F3735330000000000000000F2
:103A20004D100008391000087510000861100008DA
:103A30006D100008591000084510000831100008EA
:103A400081100008000000000100000000000000DC
:103A50006D61696E0000000069646C650000000023
:103A6000583A0008F82300207025002001000000CB
:103A7000C5190008000000004172647550696C6F40
:103A8000740025424F415244252D424C0025534598
:103A90005249414C250000000200000000000000D7
:103AA0006D120008DD12000840004000183E0020A2
:103AB000283E00200200000000000000030000007B
:103AC00000000000251300080000000010000000A6
:103AD000383E00200000000001000000000000004F
:103AE000AC40002001010200B51D0008C51C000803
:103AF000611D0008451D000843000000003B000850
:103B000009024300020100C0320904000001020260
:103B10000100052400100105240100010424020213
:103B20000524060001070582030800FF09040100BF
:103B3000020A00000007050102400000070581029B
:103B400040000000120000004C3B00081201100170
:103B50000200004009124157000201020301000067
:103B60000403090425424F41524425004B616B7503
:103B7000746548374D696E697632003031323334BE
:103B8000353637383941424344454600000000008D
:103B90007914000831170008DD17000840004000C4
:103BA000E4410020E441002001000000F441002035
:103BB000800000004001000008000000000100003B
:103BC00000040000080000000001802A000000003E
:103BD000AAAAAAAA00010024FFFF0000000000001A
:103BE00000A00A000000400100000000AAAAAAAA42
:103BF00000000001FFFF00000000000000000000C6
:103C00001000000400000000AAAAAAAA00000008F0
:103C1000FBDF0000000000000000000000000000CA
:103C200000000000AAAAAAAA00000000FFFF0000EE
:103C30000000000000000000000100000000000083
:103C4000AAAAAAAA00010000FFFF000000000000CD
:103C5000000000000000000000000000AAAAAAAABC
:103C600000000000FFFF0000000000000000000056
:103C70000000000000000000AAAAAAAA000000009C
:103C8000FFFF000000000000000000000000000036
:103C900000000000AAAAAAAA00000000FFFF00007E
:103CA0000000000000000000000000000000000014
:103CB000AAAAAAAA00000000FFFF0000000000005E
:103CC000000000000000000000000000AAAAAAAA4C
:103CD00000000000FFFF00000000000000000000E6
:103CE0000000000000000000AAAAAAAA000000002C
:103CF000FFFF0000000000000000000000000000C6
:103D0000220400000000000000001A000000000073
:103D1000FF00000000000000003A00083F00000023
:103D2000500400000B3A00083F000000009600001D
:103D300000000800960000000008000004000000D9
:103D4000603B0008000000000000000000000000D0
:103D5000000000000000000000000000FFFFFFFF67
:103D6000FFFFFFFFFFFFFFFFFFFFFFFFFFFFFFFF63
:103D7000FFFFFFFFFFFFFFFFFFFFFFFFFFFFFFFF53
:103D8000FFFFFFFFFFFFFFFFFFFFFFFFFFFFFFFF43
:103D9000FFFFFFFFFFFFFFFFFFFFFFFFFFFFFFFF33
:020000040801F1
:020000040802F0
:10000000000600307D0D020889E00908310302086E
:1000100011E0090809E009080DE009087F0D020850
:100020007F0D02087F0D02087F0D0208DD5C0E08BF
:100030007F0D02087F0D02087F0D02087F0D020868
:100040007F0D02087F0D02087F0D02087F0D020858
:100050007F0D02087F0D02086D6C0E08996C0E086A
:10006000C56C0E08F16C0E081D6D0E08E5140E0827
:100070000D150E0839150E0865150E0891150E0898
:10008000B9150E08E5150E0809110E087F0D0208B6
:100090007F0D02087F0D02087F0D0208496D0E08D2
:1000A0007F0D02087F0D02087F0D02087F0D0208F8
:1000B000996E0E08AD6E0E08C16E0E08DD1B0E089F
:1000C000051D0E087F0D02087F0D020835200E0861
:1000D0004D200E08216E0E08356E0E08496E0E0872
:1000E000AD6D0E087F0D02087F0D0208E96E0E0847
:1000F000F96E0E080D6F0E08116F0E0811160E081E
:100100007F0D02087F0D0208D56E0E087F0D0208D4
:100110005D6E0E087F0D02087F0D02087F0D02083C
:100120003D160E0865160E0891160E08BD160E082F
:10013000E9160E087F0D02087F0D02087F0D0208E8
:100140007F0D02087F0D02087F0D02087F0D020857
:1001500011170E083D170E0869170E08716E0E086C
:100160007F0D02087F0D02087F0D02087F0D020837
:100170007F0D0208C9680E087F0D02087F0D020876
:100180007F0D02087F0D0208856E0E087F0D0208A4
:1001900065200E087F0D02087F0D02087F0D020802
:1001A0007F0D02087F0D02087F0D02087F0D0208F7
:1001B0007F0D02087F0D02087F0D02087F0D0208E7
:1001C0007F0D02087F0D02087F0D02087F0D0208D7
:1001D0007F0D0208B5680E087F0D02087F0D02082A
:1001E0007F0D02087F0D02087F0D02087F0D0208B7
:1001F0007F0D02087F0D02087F0D02087F0D0208A7
:100200007F0D02087F0D02087F0D02087F0D020896
:100210007F0D02087F0D02087F0D02087F0D020886
:100220007F0D02087F0D02087F0D02087F0D020876
:100230007F0D02087F0D02087F0D020829110E08AC
:100240007F0D0208B1120E08D9120E0805130E0810
:1002500031130E085D130E0889130E08B5130E082E
:10026000E1130E087F0D02087F0D02087F0D0208C2
:100270007F0D02087F0D02087F0D02087F0D020826
:100280007F0D02087F0D02087F0D02087F0D020816
:100290007F0D02087F0D02087F0D02087F0D020806
:1002A0007F0D02087F0D02087F0D02087F0D0208F6
:1002B0007F0D02087F0D02087F0D02087F0D0208E6
:1002C0007F0D02087F0D02087F0D02087F0D0208D6
:1002D0007F0D02087F0D02087F0D02087F0D0208C6
:1002E000F52C0208FDBF02084989040839BA06083E
:1002F000B1E00608C14907083153070881560708CD
:1003000045DC0708D5E20708650208082DB2080891
:1003100051D90908E1F109080D600C08D1060D0852
:10032000592E0D08A1450D0829780D08ED7D0D0801
:10033000EFF30383EFF30982EFF30881DFF814D0C2
:100340002DE9FE4F684600F0E3FFBDE8FE4F8D4605
:10035000704700009C2B0030F1EE101AA0EC200A30
:1003600001607047A0EC108A704700BF81F0004127
:1003700002E000BF83F0004330B54FEA41044FEA8A
:10038000430594EA050F08BF90EA020F1FBF54EA25
:10039000000C55EA020C7FEA645C7FEA655C00F0C1
:1003A000E2804FEA5454D4EB5555B8BF6D420CDD92
:1003B0002C4480EA020281EA030382EA000083EA15
:1003C000010180EA020281EA0303362D88BF30BDB5
:1003D00011F0004F4FEA01314FF4801C4CEA11310B
:1003E00002D0404261EB410113F0004F4FEA03336A
:1003F0004CEA133302D0524263EB430394EA050FF5
:1004000000F0A780A4F10104D5F1200E0DDB02FA63
:100410000EFC22FA05F2801841F1000103FA0EF2F7
:10042000801843FA05F359410EE0A5F120050EF1BD
:10043000200E012A03FA0EFC28BF4CF0020C43FAEE
:1004400005F3C01851EBE37101F0004507D54FF0FB
:10045000000EDCF1000C7EEB00006EEB0101B1F54B
:10046000801F1BD3B1F5001F0CD349085FEA300091
:100470004FEA3C0C04F101044FEA445212F5800F9C
:1004800080F09A80BCF1004F08BF5FEA500C50F139
:10049000000041EB045141EA050130BD5FEA4C0C1C
:1004A000404141EB0101013C28BFB1F5801FE9D279
:1004B00091F0000F04BF01460020B1FA81F308BF9C
:1004C0002033A3F10B03B3F120020CDA0C3208DD68
:1004D00002F1140CC2F10C0201FA0CF021FA02F143
:1004E0000CE002F11402D8BFC2F1200C01FA02F1B3
:1004F00020FA0CFCDCBF41EA0C019040E41AA2BFD8
:1005000001EB0451294330BD6FEA04041F3C1CDA9F
:100510000C340EDC04F11404C4F1200220FA04F0BF
:1005200001FA02F340EA030021FA04F345EA030169
:1005300030BDC4F10C04C4F1200220FA02F001FA2B
:1005400004F340EA0300294630BD21FA04F02946AD
:1005500030BD94F0000F83F4801306BF81F4801146
:100560000134013D4EE77FEA645C18BF7FEA655CB9
:1005700029D094EA050F08BF90EA020F05D054EA8B
:10058000000C04BF1946104630BD91EA030F1EBF90
:100590000021002030BD5FEA545C05D14000494194
:1005A00028BF41F0004130BD14F580043CBF01F587
:1005B000801130BD01F0004545F0FE4141F470016D
:1005C0004FF0000030BD7FEA645C1ABF1946104648
:1005D0007FEA655C1CBF0B46024650EA013406BF49
:1005E00052EA033591EA030F41F4002130BD00BF08
:1005F00090F0000F04BF0021704730B54FF48064C5
:1006000004F132044FF000054FF0000150E700BF45
:1006100090F0000F04BF0021704730B54FF48064A4
:1006200004F1320410F0004548BF40424FF0000191
:100630003EE700BF42004FEAE2014FEA31014FEAD4
:1006400002701FBF12F07F4393F07F4F81F0605123
:10065000704732F07F4208BF704793F07F4F04BF6E
:1006600041F40021704730B54FF4607401F000454B
:1006700021F000411CE700BF50EA010208BF7047AB
:1006800030B54FF000050AE050EA010208BF70479C
:1006900030B511F0004502D5404261EB41014FF405
:1006A000806404F132045FEA915C3FF4D8AE4FF00D
:1006B00003025FEADC0C18BF03325FEADC0C18BFF0
:1006C000033202EBDC02C2F1200300FA03FC20FA41
:1006D00002F001FA03FE40EA0E0021FA02F114448E
:1006E000BDE600BF80F0004002E000BF81F00041A5
:1006F00042001FBF5FEA410392EA030F7FEA226CC8
:100700007FEA236C6AD04FEA1262D2EB1363C1BF57
:10071000D218414048404140B8BF5B42192B88BFC6
:10072000704710F0004F40F4000020F07F4018BFE9
:10073000404211F0004F41F4000121F07F4118BF09
:10074000494292EA030F3FD0A2F1010241FA03FCB1
:1007500010EB0C00C3F1200301FA03F100F0004399
:1007600002D5494260EB4000B0F5000F13D3B0F161
:10077000807F06D340084FEA310102F10102FE2AD0
:1007800051D2B1F1004F40EBC25008BF20F0010040
:1007900040EA03007047490040EB0000013A28BFDF
:1007A000B0F5000FEDD2B0FA80FCACF1080CB2EB62
:1007B0000C0200FA0CF0AABF00EBC25052421843E0
:1007C000BCBFD0401843704792F0000F81F4000185
:1007D00006BF80F400000132013BB5E74FEA410358
:1007E0007FEA226C18BF7FEA236C21D092EA030FC4
:1007F00004D092F0000F08BF0846704790EA010F3E
:100800001CBF0020704712F07F4F04D1400028BF6A
:1008100040F00040704712F100723CBF00F500004C
:10082000704700F0004343F0FE4040F40000704782
:100830007FEA226216BF08467FEA2363014642022E
:1008400006BF5FEA412390EA010F40F48000704741
:100850004FF0000304E000BF10F0004348BF4042E7
:100860005FEA000C08BF704743F0964301464FF023
:1008700000001CE050EA010208BF70474FF000037F
:100880000AE000BF50EA010208BF704711F00043C0
:1008900002D5404261EB41015FEA010C02BF844690
:1008A0000146002043F0B64308BFA3F18053A3F5EF
:1008B0000003BCFA8CF2083AA3EBC25310DB01FA36
:1008C00002FC634400FA02FCC2F12002BCF1004FBA
:1008D00020FA02F243EB020008BF20F0010070474B
:1008E00002F1200201FA02FCC2F1200250EA4C009F
:1008F00021FA02F243EB020008BF20EADC707047E5
:100900007BB972B90029BEBF00204FF0004106E05C
:1009100008BF00281CBF6FF000414FF0FF3000F00F
:100920002BBAADF1080C6DE904CE002909DB002BD0
:100930001ADB00F0B9F8DDF804E0DDE9022304B0C9
:100940007047404261EB4101002B1BDB00F0ACF82B
:10095000DDF804E0DDE9022304B0404261EB41012F
:10096000524263EB43037047524263EB430300F090
:100970009BF8DDF804E0DDE9022304B0404261EBBE
:1009800041017047524263EB430300F08DF8DDF8FC
:1009900004E0DDE9022304B0524263EB43037047F5
:1009A00053B94AB9002908BF00281CBF4FF0FF31D6
:1009B0004FF0FF3000F0E0B9ADF1080C6DE904CE66
:1009C00000F072F8DDF804E0DDE9022304B07047BE
:1009D000430803F05533C01A830803F0333300F0A3
:1009E0003330184400EB101000F00F3000EB002003
:1009F00000EB0040000E704708B502460B4643EC82
:100A0000172BB5EEC07BF1EE10FA03D4BDE8084019
:100A100000F02AB8B1EE477B51EC170B00F024F838
:100A2000404261EB410108BD9FED0B6B07EE900A60
:100A30009FED0B5BB7EEE77A27EE066BBCEEC66B5D
:100A4000B8EE464BA4EE457BFCEEC77B16EE101AC3
:100A500017EE900A704700BF000000000000F03D54
:100A6000000000000000F0419FED0B6B41EC170B04
:100A70009FED0B5B27EE066BBCEEC66BB8EE464BEC
:100A8000A4EE457BFCEEC77B16EE101A17EE900A1B
:100A9000704700BFAFF30080000000000000F03D91
:100AA000000000000000F0412DE9F047089D0446D9
:100AB0008E46002B4DD18A42944669D9B2FA82F211
:100AC00052B101FA02F3C2F1200120FA01F10CFA4D
:100AD00002FC41EA030E94404FEA1C48210CBEFB85
:100AE000F8F61FFA8CF708FB16E341EA034306FB0E
:100AF00007F199420AD91CEB030306F1FF3080F09D
:100B00001F81994240F21C81023E63445B1AA4B2E9
:100B1000B3FBF8F008FB103344EA034400FB07F78B
:100B2000A7420AD91CEB040400F1FF3380F00A81CC
:100B3000A74240F207816444023840EA0640E41BC1
:100B400000261DB1D4400023C5E900433146BDE86D
:100B5000F0878B4209D9002D00F0EF800026C5E90F
:100B6000000130463146BDE8F087B3FA83F6002E27
:100B70004AD18B4202D3824200F2F980841A61EB9F
:100B8000030301209E46002DE0D0C5E9004EDDE7BD
:100B900002B9FFDEB2FA82F2002A40F09280A1EBA5
:100BA0000C014FEA1C471FFA8CFE0126200CB1FBFA
:100BB000F7F307FB131140EA01410EFB03F08842F3
:100BC00008D91CEB010103F1FF3802D2884200F280
:100BD000CB804346091AA4B2B1FBF7F007FB101112
:100BE00044EA01440EFB00FEA64508D91CEB0404B0
:100BF00000F1FF3102D2A64500F2BB800846A4EB0B
:100C00000E0440EA03409CE7C6F12007B34022FAF5
:100C100007FC4CEA030C20FA07F401FA06F31C4324
:100C2000F9404FEA1C4900FA06F3B1FBF9F8200C31
:100C30001FFA8CFE09FB181140EA014108FB0EF077
:100C4000884202FA06F20BD91CEB010108F1FF3AC7
:100C500080F08880884240F28580A8F102086144D3
:100C6000091AA4B2B1FBF9F009FB101144EA0141E1
:100C700000FB0EFE8E4508D91CEB010100F1FF348C
:100C80006CD28E456AD90238614440EA0840A0FB24
:100C90000294A1EB0E01A142C846A64656D353D0FA
:100CA0005DB1B3EB080261EB0E0101FA07F722FA1E
:100CB00006F3F1401F43C5E9007100263146BDE847
:100CC000F087C2F12003D8400CFA02FC21FA03F3AA
:100CD000914001434FEA1C471FFA8CFEB3FBF7F02B
:100CE00007FB10360B0C43EA064300FB0EF69E4250
:100CF00004FA02F408D91CEB030300F1FF382FD2E9
:100D00009E422DD9023863449B1B89B2B3FBF7F690
:100D100007FB163341EA034106FB0EF38B4208D969
:100D20001CEB010106F1FF3816D28B4214D9023EAA
:100D30006144C91A46EA004638E72E46284605E7C8
:100D40000646E3E61846F8E64B45A9D2B9EB020899
:100D500064EB0C0E0138A3E74646EAE7204694E729
:100D60004046D1E7D0467BE7023B614432E730465C
:100D700009E76444023842E7704700BF02E000F030
:100D800000F8FEE772B6374880F30888364880F3EB
:100D9000098836483649086040F20000CCF200006D
:100DA0004EF63471CEF200010860BFF34F8FBFF3EF
:100DB0006F8F40F20000C0F2F0004EF68851CEF284
:100DC00000010860BFF34F8FBFF36F8F4FF000003B
:100DD000E1EE100A4EF63C71CEF2000108600620EA
:100DE00080F31488BFF36F8FC4F0DAFFC6F072FB94
:100DF0004FF055301F491B4A91423CBF41F8040B4C
:100E0000FAE71D49184A91423CBF41F8040BFAE742
:100E10001A491B4A1B4B9A423EBF51F8040B42F839
:100E2000040BF8E700201849184A91423CBF41F8EA
:100E3000040BFAE7C4F0F2FFC6F0D0FB144C154DDA
:100E4000AC4203DA54F8041B8847F9E701F0C0FE0E
:100E5000114C124DAC4203DA54F8041B8847F9E7F1
:100E6000C4F0DABF000600300022003000000208A3
:100E700008ED00E0000000300006003040AC110832
:100E800000220030A4290030A82900309CB5013090
:100E9000E0020208300302083003020830030208AF
:100EA0002DE9F04F2DED108AC1F80CD0D0F80CD000
:100EB000BDEC108ABDE8F08F002383F3118828462B
:100EC000A0470020C3F0F0FCFEE7C3F059FB00DFB1
:100ED000FEE7000070B54FF0FF0C4CF4E06C1CEA2C
:100EE00011541DBF1CEA135594EA0C0F95EA0C0F20
:100EF00000F0DEF82C4481EA030621EA4C5123EA93
:100F00004C5350EA013518BF52EA033541F48011C1
:100F100043F4801338D0A0FB02CE4FF00005E1FB74
:100F200002E506F00042E0FB03E54FF00006E1FBBE
:100F300003569CF0000F18BF4EF0010EA4F1FF0401
:100F4000B6F5007F64F5407404D25FEA4E0E6D4141
:100F500046EB060642EAC62141EA55514FEAC52052
:100F600040EA5E504FEACE2EB4F1FD0C88BFBCF5CE
:100F7000E06F1ED8BEF1004F08BF5FEA500E50F17F
:100F8000000041EB045170BD06F0004646EA010145
:100F900040EA020081EA0301B4EB5C04C2BFD4EB77
:100FA0000C0541EA045170BD41F480114FF0000E70
:100FB000013C00F3AB8014F1360FDEBF002001F0DE
:100FC000004170BDC4F10004203C35DA0C341BDC58
:100FD00004F11404C4F1200500FA05F320FA04F02A
:100FE00001FA05F240EA020001F0004221F000415E
:100FF00010EBD37021FA04F642EB06015EEA430ED1
:1010000008BF20EAD37070BDC4F10C04C4F1200500
:1010100000FA04F320FA05F001FA04F240EA0200B3
:1010200001F0004110EBD37041F100015EEA430E84
:1010300008BF20EAD37070BDC4F1200500FA05F2A4
:101040004EEA020E20FA04F301FA05F243EA020323
:1010500021FA04F001F0004121FA04F220EA020032
:1010600000EBD3705EEA430E08BF20EAD37070BD78
:1010700094F0000F0FD101F00046400041EB010158
:1010800011F4801F08BF013CF7D041EA060195F03A
:10109000000F18BF704703F00046520043EB0303F4
:1010A00013F4801F08BF013DF7D043EA06037047E1
:1010B00094EA0C0F0CEA135518BF95EA0C0F0CD0EC
:1010C00050EA410618BF52EA4306D1D181EA030132
:1010D00001F000414FF0000070BD50EA410606BF2C
:1010E0001046194652EA430619D094EA0C0F02D171
:1010F00050EA013613D195EA0C0F05D152EA0336B6
:101100001CBF104619460AD181EA030101F00041D3
:1011100041F0FE4141F470014FF0000070BD41F01C
:10112000FE4141F4780170BD4FEA410212F5001210
:1011300015D211D56FF47873B3EB625212D94FEA1E
:10114000C12343F0004343EA505311F0004F23FA08
:1011500002F018BF404270474FF00000704750EA5D
:10116000013005D111F0004008BF6FF0004070471A
:101170004FF00000704700BF4FEA4102B2F1E04378
:1011800024BFB3F5001CDCF1FE5C0DD901F0004C6E
:101190004FEAC0024CEA5070B2F1004F40EB8300BE
:1011A00008BF20F00100704711F0804F21D113F1EA
:1011B0003872BCBF01F00040704741F480114FEA23
:1011C0005252C2F11802C2F1200C10FA0CF320FAAC
:1011D00002F018BF40F001004FEAC1234FEAD323C9
:1011E00003FA0CFC40EA0C0023FA02F34FEA430333
:1011F000CCE77FEA625307D150EA01331EBF4FF0BC
:10120000FE4040F44000704701F0004040F0FE40D6
:1012100040F40000704700BF01F0FF01102A2BDBF3
:1012200010F0070F08D010F8013B013A8B422DD087
:1012300010F0070F42B3F6D1F0B441EA012141EAC0
:10124000014122F007047FF000070023F0E8025676
:10125000083C85EA010586EA010685FA47F5A3FA06
:1012600087F586FA47F6A5FA87F68EB9EED1F0BC77
:1012700001F0FF0102F0070232B110F8013B013A20
:1012800083EA010313B1F8D1002070470138704799
:10129000002D06BF35460338073815F0010F07D17A
:1012A000013015F4807F02BF013015F4C03F0130DA
:1012B000F0BC0138704700BF10F8012B11F8013B5A
:1012C000012A28BF9A42F7D0D01A7047034613F874
:1012D000012B002AFBD1181A0138704710B50446BB
:1012E00020461CB154F80C3B013300D110BD08223C
:1012F000012100F071FB54F80C0C54F8082C14F880
:10130000041C121AB2FBF1F200F066FBE8E70000E1
:10131000C26AD0E9003112F0040F2DE9F04118BF84
:101320000B46A6B00021594C042601270291CDE9B5
:101330000003D0064CBF03F1200203F168020392C0
:10134000DA690399D2099B6902F004021B880A43F7
:1013500003F47F4303924FF0E022A3F53E41D2F81D
:10136000882D02F4A002B2F5A00F04BF0122029260
:101370004B424B410493464D03A82C6000F02AFADF
:1013800004220121434800F027FB0422012102A886
:1013900000F022FB10220121019800F01DFB0098B3
:1013A000202201210C3000F017FB019804220121BA
:1013B000103000F011FB0422012103A800F00CFB07
:1013C00001980C220121143000F006FB0C220121AF
:1013D000009800F001FB029BDA071FD5009BDB6A37
:1013E000DB064ED415A8FEF7BDFFDDF804C00DF1F5
:1013F000140E0CF120030CF160081868083353F840
:10140000041C7246434503C29646F6D1DCF86030B0
:1014100025938422012105A800F0DEFA00F0C0F82F
:10142000FFF75CFF4FF0E023D3F8003D03F4702397
:10143000B3F5402F0ED0184B05A88DF81C6005930E
:1014400014338DF8287006934FF0FF33CDE908333D
:10145000FFF744FF2B68A34206D0104B0422012162
:1014600005A8059300F0B8FA00F02AFA002882D007
:10147000049B1BB1019A93690233936126B0BDE8C6
:10148000F08105A8FEF768FFC3E700BFED55CEACBD
:10149000A8290030E0FA0E0828ED00E0ACCE55EDAA
:1014A00037B50E4D2A78202A15D10D4C0D482368EA
:1014B0000D4918440192C3F02FFE23680021019AC0
:1014C0002033094829702360C9F054FF03B0BDE8F8
:1014D0003040C4F017BB03B030BD00BF9C2B0030C0
:1014E000C42B003000B411089E2B003008B5262014
:1014F000C1F0CCFC144BD3F8902042F40032C3F876
:101500009020D3F8902022F40032C3F89020D3F832
:101510009020D3F8E82042F40032C3F8E820D3F852
:10152000102142F40032C3F810216D22D3F810319B
:10153000064BDA604FF0FF321A620D221A60012268
:10154000034B1A7008BD00BF00440258004400401D
:10155000D42B0030014B1868704700BFFCFF1B08FC
:10156000014B0248C01A704700B4110800001C0863
:101570000048704700B4110807490022074B5B1A66
:101580009A4201D30120704751F8040B013001D178
:101590000432F5E70020704700B4110800001C0871
:1015A0005E4B2DE9F74F1A6802255D4B02F56A582C
:1015B000DFF894911A7808F118085A4F5A4C904461
:1015C000DFF888A1C2F0F2FEA9EB070B06460EB1C8
:1015D0004E2D49D9A9EB0702B2EB080700F1928022
:1015E0004E2D00F28F80DFF868C16B1C4F4E0C212E
:1015F000DBB2ACEB06006943B84273DD60184FF014
:10160000010C665090463E4480F808C04660B2EB3C
:10161000080213D44F2B11D0454E19464548AB1C38
:10162000351ADBB295424FF00C0505FB01F163DD85
:1016300065180126024460502E726A600C22012156
:101640005343E21811724FF0FF31E15051603A4BB1
:101650001B782BB1394B1B682360394B1B686360C7
:10166000314803B0BDE8F08F336AF06953450ABFD3
:10167000344BF31AA3EB0A0380B10193C3F03AFF92
:10168000019B58B12A460C2101354A430121EDB294
:10169000A0180172F169A1500D3141600C200121A7
:1016A000984400FB05FCD84504EB0C0244F80C60A0
:1016B00006F13C0C1172C2F804C005EB010205F101
:1016C0000205D2B2EDB200FB02F204EB020001729D
:1016D000316AA1501944416014D23046C2F076FEFE
:1016E000064674E767184FF0010E8044665087F88D
:1016F00008E0C7F804C08AE7621801256050157237
:1017000056609BE74F2D01D82B4697E7012384F8BD
:10171000BC334FF0FF33C4E9ED3398E7C42B0030FE
:101720009C2B003000B4110804220030A82900309E
:1017300000000430A0B5013000220030C82B00307A
:10174000C02B00300022003000001C0800060030D2
:101750009CB501300C4B1B7810B50BB9FFF7C6FEDA
:1017600000230A490A48CA699206FCD54A6A1C5CE9
:10177000D2B2944205D10133DBB20E2BF3D100205B
:1017800010BD0023EFE700BFD42B00300044004021
:10179000E4FA0E0838B5084B04461B780BB9FFF77E
:1017A000A5FEE4B2054DAC62EB695B0600D538BD21
:1017B000C4F0A8F9F8E700BFD42B00300044004083
:1017C00010B5441E14F8010F00B910BDFFF7E2FF79
:1017D000F8E7000070B502680446EFF30581D920F0
:1017E0005369C9B27CF016FC294B1B78A3B1294B75
:1017F00094E8030083E803002748FFF7E1FF6368EC
:10180000B3B12648FFF7DCFF2548FFF7D9FFFFF704
:10181000A1FF2448FFF7D4FF234D2B783BB1246868
:101820001CB12046C3F066FE20B900232B7070BDAA
:101830001E48E7E720461E4EC3F070FE00F214502B
:1018400084421FD22046C3F069FE30602046194E04
:10185000C3F078FE04F5E053834217D92046C3F065
:1018600071FE30600023144A1360144A1370FFF7AE
:1018700083FE0028D9D0C4F045F90120BDE87040AE
:10188000C3F0D2BCA4F214533360DFE73360E9E75E
:101890009D2B0030CC2B0030F4FA0E08F9FA0E081C
:1018A0000AFB0E08D4C80F080022003004FB0E0803
:1018B000C82B0030C02B0030C42B00309C2B0030D4
:1018C000284B1A7870B542B12748FFF779FF274BAC
:1018D0005868003818BF012070BD254A10780028CC
:1018E0003CD0244E244C33682448254D1A1D2178C1
:1018F0002D1A0A44AA4205D3224A4FF0FF31D16182
:10190000202222702278D2B103F120018D4205D825
:101910001F2A9FBF1B4AD36120222270202219490F
:101920001844C3F0F9FB32682378002115481344AA
:10193000202221703360C9F01DFDC4F0E3F8336844
:101940009D4207D90F4920220F48CB61C3F0E4FB29
:10195000C4F0D8F80020C3F067FCB8E701221A7081
:10196000BAE700BF9D2B003050FB0E08CC2B003097
:1019700000220030C42B00309C2B003000B4110832
:1019800000001C089E2B0030E0FF1B082DE9F843E7
:1019900007460E460024DFF83890DFF83880B4425E
:1019A00001D1BDE8F88324B1230702D14846FFF7EF
:1019B00007FF3D5D01342B0905F00F0518F8030002
:1019C000FFF7E8FE18F80500FFF7E4FEE7E700BFC1
:1019D000D4C80F0860FB0E08474B1B782DE9F74F62
:1019E00007460E4690465BB1022925D0042938D01F
:1019F000012902D11146FFF7C9FF4048FFF7E0FE79
:101A00003F4B1B78002B4ED03E4A00253E4BA2EBAD
:101A1000030938E037F81430ADF8043024B1620718
:101A200002D12846FFF7CCFE0134022101A8FFF7BE
:101A3000ADFFA045EED1E0E70024304DF9E757F8BF
:101A40002430019324B1A30702D12846FFF7B8FE42
:101A5000042101340DEB0100FFF798FFA045EED102
:101A6000CBE70024254DF9E7FFF71AFD022E1DD024
:101A7000042E2CD0012E06D12378795D5A1C2270B9
:101A8000224AD1540135A8450DD0214B214C1B6869
:101A90002278043313444B45E6D31C4B4FF0FF32FE
:101AA000DA612023237003B0BDE8F08F2378DFF8DC
:101AB0005CA05A1C22703A780AF80320FFF7F0FC69
:101AC00023785A1C227000220AF80320DAE74FF02C
:101AD000000ADFF838B022783B78511C23FA0AF369
:101AE0000AF1080A21700BF80230FFF7D9FCBAF1AD
:101AF000200FF0D1C6E700BF9D2B0030D4C80F08DF
:101B00000022003000001C0800B411089E2B003099
:101B1000C42B00309C2B0030036800221B68184740
:101B20000120704737B501912021044679F06AFE03
:101B3000E0B10F4B93F9B61EB1B1B3F9B81E03F57E
:101B40008053019AD3F85838B3F90C5001F10A03C5
:101B50009D4203DD40F28D33994205DC2046054B62
:101B6000202179F055FE002003B030BD0120FBE7B5
:101B7000D85B003074FB0E0808B505F0CBFF0121DF
:101B8000BDE8084005F03AB82DE9F04300278FB0D2
:101B90000E46054605F0BEFF80462E22394602A8B5
:101BA0000197C9F0E7FB322301AA3946404605F008
:101BB000F3F9044648B901AB174A314628467AF092
:101BC00019F820460FB0BDE8F083DFF85890D9F837
:101BD000800503689B6898470028F2D0A9F5A040CB
:101BE00003F0F8FD814630B90C4A314628464C4690
:101BF0007AF000F8E5E76946404604F0F1FF002876
:101C0000DFD09DF801305B06DBD5054A314628461A
:101C10003C4679F0EFFFD4E788FB0E0891FB0E08F5
:101C2000A8FB0E08D87B003008B5064B93F8C93ADC
:101C30009B0704D5044A79F0DDFF002008BD012090
:101C4000FCE700BFD86B0030B8FB0E0870B50C4C39
:101C500005460E46D4F880050368DB68984710B146
:101C60000124204670BDA4F5A04003F0D1FD044638
:101C70000028F5D1034A3146284679F0BBFFF0E74A
:101C8000D87B0030C8FB0E08284B2DE97043D3F8F1
:101C9000CC3A814688461D7B5DB9254B1B68986A06
:101CA00003685B6B984738B9224A4146484679F049
:101CB000A1FF2846BDE870835CF06CFA20215DF03E
:101CC00001FD38B15CF066FA1F215DF0FBFC08B144
:101CD000194AEAE7484679F08DFD38B9D9F800305D
:101CE000414648469B6BBDE870431847414648460D
:101CF000FFF718FF0646414648467AF033FD064096
:101D000020214846F5B279F07DFD41464846FFF76F
:101D10008BFF054041464846FFF798FF0540414686
:101D200048467AF097FF0540C3E700BFD86B003004
:101D300060820030DCFB0E08F3FB0E0808B5FFF7ED
:101D4000A3FF054A92F8B81A60F3410182F8B81A65
:101D5000024A907108BD00BFD86B00300D8300307F
:101D60002DE9F04106460F4679F082FD044668B33E
:101D70000221304679F046FD40B305F0CBFE4FF42A
:101D80008071804604F03AFF0546F8B94FF40071BF
:101D9000404604F033FFC8B10E487BF0A9F90E4B62
:101DA000D3ED277AF8EEE77A30EE670ADFED0B7AAB
:101DB000B0EEC00AB4EEE70AF1EE10FA06DD2C46EA
:101DC000074B3A460221304679F022FD2046BDE815
:101DD000F08100BF6C7D0030D87B00300000C8422D
:101DE00010FC0E08F8B504460F467AF0AFF8102143
:101DF0000546204679F006FD58B12046FFF7BCFEA7
:101E0000064630B93546044B3A461021204679F053
:101E1000FFFC2846F8BD00BF24FC0E0870B505463F
:101E20000E4679F047FC044678B18021284679F0C7
:101E3000E9FC50B1094B93F8993043B10024084BA9
:101E400032468021284679F0E3FC204670BD3146B9
:101E50002846BDE870407AF05BBA00BFD87B0030FE
:101E600038FC0E082DE9F04180460E461B4FFFF767
:101E70008BFE044610B90024FC710AE0184D05F5EC
:101E8000A043D3F8800503689B68984720B90123D5
:101E9000FB712046BDE8F0810821404679F0B2FC94
:101EA0000028F4D095F81434B02202FB035305F552
:101EB0004055B3F81E22B5F9B43E9A4206DD094BEF
:101EC00032460821404679F0A3FCD4E7314640462B
:101ED00079F0BEFD0028DAD1CDE700BF0D830030D8
:101EE000D82B00304CFC0E087AF010BB70B50546BC
:101EF0000E46FFF749FE084B04463146D871284686
:101F0000FFF7A4FE00283146284608BF00247AF0D7
:101F100001FE204070BD00BF0D8300302DE9F84365
:101F2000414F81463B78002B7BD1404C0126D4F8B1
:101F3000CC5A3E702D7B1DB13B702846BDE8F8831E
:101F40007AF062FF054630B9394A3870137843F0A9
:101F500001031370F1E7DFF8F4804EF015F9314614
:101F60004DF03CFA88F804600B26013E45F06AF912
:101F700045F086F816F0FF06F7D12E4948467AF06C
:101F80001BFE05F0C7FDD0F80C22C4F8DC2A90F83F
:101F90009432DA0733D405F06DF84EF0F5F83C21B1
:101FA0004EF02EF804F6C42300221A60224B0121C1
:101FB0001B68D86A03681B689847D4F8CC2A137B3F
:101FC0001BB90123137388F804304EF0DDF894F840
:101FD000BD2A94F8BC1A4DF0F1FB4AF0C3FD4AF05B
:101FE000F3F800233B707CF081F8144BC3F87405C0
:101FF00094F8B93A43F0200384F8B93A9DE79B0777
:10200000D4D431460E4802F07FFA0E487BF070F8C7
:10201000DFED0D7A04F6C42320EE270A83ED000AD3
:10202000C4E7002589E700BFD52B0030D86B00300E
:102030002C8300305CFC0E0860820030D87B0030BE
:10204000D82B00306C7D00300AD7233C0D83003044
:102050002DE9F043364D87B006460C46D5F8CC3A0C
:102060001B7B002B61D000294BD0214630467AF0F3
:102070008FFF0446002853D02E4930467AF09CFD4D
:1020800005F048FD07460AF08FFD8046384604F00B
:10209000EDF9D8B198F92830022B17D100264FF06E
:1020A0000009F1B203AA3846CDF80C900191CDF8A1
:1020B0001090CDF8149004F00BFE019918B103AA0A
:1020C00040460AF07DFA0136032EEAD1D5F8CC2A33
:1020D000137B1BB100231373174A13714EF054F88E
:1020E00000214DF07BF9154B00211B68D86A03686D
:1020F0001B68984795F8B93A6FF3451385F8B93AD4
:102100000FE005F580530192D3F880050368DB6882
:102110009847019A0028A8D195F8B83ADB06A4D4CC
:102120000024204607B0BDE8F0830124F9E700BF92
:10213000D86B00306CFC0E080D83003060820030DC
:1021400000F5804008B590F8B83AC3F380028A429F
:102150000BD061F3820380F8B83A31B14EF014F835
:102160000F21BDE808404DF04BBF08BD00F580428F
:1021700010B592F8C93A0C4603F00101A14209D00A
:1021800064F3000382F8C93ADB0704D402F00EFCC2
:10219000024B9C7210BD02F0BDFCF9E70D830030CC
:1021A00000F5804090F8C93A61F3410380F8C93ADC
:1021B000014B1973704700BF0D830030002070473A
:1021C00000207047002070470020704700207047B3
:1021D00000207047002070470020704700207047A3
:1021E00000207047002070470020704770470000B3
:1021F00070470000002070470020704700207047A3
:102200000020704700207047002070470020704772
:102210000020704700207047704700000020704782
:102220000020704700207047002070470020704752
:102230000020704700207047002070470020704742
:102240000020704700207047002070470020704732
:1022500000207047704700007047000000F57B5079
:102260000430704700487047002D0F0800F580408B
:1022700090F8BC0A70470000034808601C211170E8
:1022800008221A60704700BF44000F084AF0B6BB2E
:102290001CF026BF4DF020BA5BF058BB59F01AB8BD
:1022A00002F0A4BB02F0D6BA02F0FCB944F0E8BEDA
:1022B00061F07CBC5BF020BE13F02CBB02F010B9C7
:1022C00002F0DEBD02F08EBA02F02CBD03F0A8B819
:1022D0001DF0A8BB03F0B2BA02F0BCBB02F076BCA2
:1022E000684B70B5044640F8043B5FF073FF00256F
:1022F00004F1100004F5795609F00EF904F16800B4
:102300004AF00AF904F5907011F0F2FC04F5AA60A5
:1023100007F02EFD04F5DF6009F0B6FE04F5246039
:102320001CF008FD04F668705FF0CAFE04F58150E9
:102330000C36183049F038FD04F59B504CF09EFFE8
:1023400004F5A050183067F0BFFA04F5A15014301E
:102350005EF006FC04F5A350103070F09DFD04F50E
:10236000D85077F0F9FF04F5D8501C304AF08EFCB5
:1023700004F5E050103061F019F904F5805304F5CC
:10238000E250414A83F8345C04F5E15304301433DD
:10239000136044F07DFC04F5E4502946183003F046
:1023A0004DFD04F50C50303063F096FD04F50D50F2
:1023B00020306DF0BDFF04F533502C306EF014FD6D
:1023C00004F54950303075F01DF804F54E500830D2
:1023D00077F01CF904F54F502C3077F051FD04F5DF
:1023E000515004306CF0BAFE04F553502C3007F015
:1023F000F3FA04F5595010306EF052FE04F55B50BC
:10240000103079F045F904F568502049243048F03F
:1024100081FB04F568503C3067F056FE04F56D50C2
:102420000C3079F009F804F56E5024307BF06AFE28
:1024300004F5715010305DF0E3FF04F5405383F86C
:10244000B85C04F573550C3528460C3550F0D6F8B9
:10245000AE42F9D104F579500D4D183079F06CF891
:1024600004F579503C304FF033FF2B6813B1094825
:102470007BF00EFE2046084948F04CFB20462C60BD
:1024800070BD00BF1CD70F08788F0030689210080D
:1024900000840030C4FC0E08C4D50F0810B503F04A
:1024A00099F85BF077FE0368BDE810405B68184759
:1024B000FFF7F4BF38B500F595450446603528466A
:1024C00008F0F4FE0AF070FB90F92530D3B190F8D3
:1024D0004433BBB12846002108F07EFCDFED0A7AC8
:1024E00004F6541304F5DF6020EE270ADFED077AC7
:1024F00093ED287AA7EE270A83ED280ABDE8384035
:102500000AF062BA38BD00BFCDCCCC3D6666663FEE
:10251000FFF7D0BF10B50121044603F0B3F910B1A5
:10252000204601F0A5F94FF48051204603F0AAF9A6
:1025300020B12046BDE8104001F05CB910BD00009C
:10254000FFF7E8BF13B50221044603F09BF938B149
:102550000121204603F096F910B9204601F088F9D0
:102560000221204603F08EF950B3204601F08EF987
:102570004021204603F086F960B104F59B5001909C
:102580004CF04CF904F58053019893F934340BB1B5
:102590004CF010FB4FF48061204603F073F918B142
:1025A00004F59B504CF0DCF98021204603F06AF9D9
:1025B00068B11EF0DFF902B0BDE810401CF0FAB9B6
:1025C0000121204603F05EF90028CED1D0E74FF478
:1025D0008021204603F056F90028EAD14FF400216B
:1025E000204603F04FF90028E3D102B010BD0000EF
:1025F000FFF7A8BF10B50121044603F043F910B15D
:10260000204601F043F98021204603F03BF928B130
:102610001EF0B0F9BDE810401CF0A8B910BD0000D4
:10262000FFF7E8BF38B504464FF6FF7103F02AF90B
:1026300004F5804528B1D5F8B82A0721204601F0D5
:102640002DF95DF009FE5DF0FBFA95F8B83A074AFE
:1026500083F01003C3F3001353714AF083FA49F077
:10266000D5FE0348BDE838406BF0F2BF0D83003063
:1026700058800030FFF7D6BF30B500F5E45405466A
:10268000012118342DED028B20469FB005F0B4F9DE
:1026900005F5A14120463C3105F01CF805F5A141A6
:1026A0002046543104F008F805F5FF5104F54B704D
:1026B00005F5A044083122F09DFE05F5A140D4F8AF
:1026C000BC201CA9D4F8C030683084ED380A1C92B4
:1026D0001D9350F035FC05F5A14105F5A240B0EE83
:1026E000608AF0EE408A44312C3050F0BDFA05F596
:1026F000A14105F5A240C4ED328A603184ED338AF0
:10270000603084ED340A50F0AFFA84ED390A4DF0B0
:102710003BFD05467BF0F2FC2A4B2B4A93ED007AF9
:102720002A4BB7EEC77A8DED187B94ED377AB7EE6A
:10273000C77A8DED167B94ED367AB7EEC77A8DEDBC
:10274000147B94ED357AB7EEC77A8DED127B94ED5C
:10275000397AB7EEC77A8DED107B94ED387AB7EE03
:10276000C77A8DED0E7B94ED347AB7EEC77A8DED96
:102770000C7B94ED317AB7EEC77A8DED0A7B94ED40
:10278000337AB7EEC77A8DED087B94ED307AB7EEE9
:10279000C77A8DED067B94ED327AB7EEC77A8DED70
:1027A000047B94ED2F7AB7EEC77ACDE90001084992
:1027B00028468DED027B4DF059FA1FB0BDEC028B1F
:1027C00030BD00BF884A0030E6FC0E08D8FC0E0879
:1027D00013FD0E08FFF750BF10B5044602F084FF4A
:1027E0001021204603F04EF850B11EF0C3F81CF043
:1027F000AFF904F5A350BDE8104010306FF080BD74
:1028000010BD0000FFF7E8BF00F5E450D1ED017AFC
:1028100091ED006AD0EDA05AD0EDA36A26EEE77ADA
:1028200067EEA57AA6EE257AE6EE267A81ED007AA5
:10283000C1ED017A7047000000F5E450D1ED017A56
:1028400091ED006AD0EDA05AD0EDA36A27EEA67AEA
:1028500067EEA57AA6EE257AE6EE667A81ED007A35
:10286000C1ED017A704700002DE9F04105464FF0B7
:1028700001082DED028B86B005F58044FFF730FD91
:10288000B94B05F57B5005F590462B6004AF383009
:10289000683601F0F3FC05F57A5330463C33C4F852
:1028A0006038062384F8643878F010FFAF4B301D91
:1028B00005F591463946C4F8683864368DF81080BD
:1028C00049F03EF9AA4B06F10C00C4F8E4387AF05E
:1028D00063FD1E234FF4E16084F8488AC4F8503A3F
:1028E0000023A4F8543A09F095FBC4F84C0A05F506
:1028F000944058307AF050FD05F595401C307AF040
:102900004BFD9C4B1A6802B91E609B49304648F04B
:1029100001F99A4B05F59540F7EE008AC4F8E438C2
:1029200001233E309FED968AA4F8BC3A05F5A044F9
:102930007AF072FB934B05F595404FF400710593C7
:10294000914B603004950093904E97E80C0008F08E
:1029500085F805F5A14003A9CDED038A20301427A1
:102960004FF0D2FE05F5A1402C3008F0EFFE05F542
:10297000E453B0EE083A9FED862A183305F5A340DC
:10298000F0EE420A84ED2F8AC4F8AC31F0EE432A0F
:10299000B0EE430A3030F0EE481A84ED308AB0EEE3
:1029A000481A84ED318A84ED328A84ED338A84EDCD
:1029B000348A84ED358A84ED368A84ED378A84ED55
:1029C000438A84ED448A84ED458A84ED468A84ED09
:1029D000478A84ED488A84ED498A84ED4A8A84EDE9
:1029E000658A84ED668A84ED678A84ED688A84ED61
:1029F000698A84ED6A8A6CF063F8B0EE083A05F5EE
:102A0000A440B0EE682AF0EE481AF0EE432A643093
:102A1000B0EE481AF7EE080AB1EE0C0A6CF0FEF9B7
:102A2000B0EE083A05F5A540F0EE481AB0EE481AA7
:102A30009FED572AF0EE432ADFED560AB0EE430A27
:102A40005C306CF0EBF9B0EE083A05F5A640F0EE1C
:102A5000481AB0EE481A9FED502AF0EE432ADFEDF7
:102A60004F0AB0EE680A54306CF02AF8B0EE083A1B
:102A700005F5A840B0EE482AF0EE481A9FED480A46
:102A8000F0EE432A0830B0EE481AF0EE480A6CF037
:102A9000C5F9F0EE083AB0EE485A9FED420AF0EE62
:102AA000684A05F5A940B0EE484AB0EE633AF0EE48
:102AB000632AB0EE002AF0EE481AB0EE481AF6EE9D
:102AC000000A6BF075FD384B05F5AA421E60002325
:102AD0007C3298B2013307FB0061097C0029F8D1F0
:102AE000324B1880324B1880324B196811B1324882
:102AF0007BF0CEFA05F5AB401A600430C4F88005CF
:102B000002F076F92D4B05F5AB40C4F8843534302E
:102B100002F06EF92A4B05F5AB40C4F8B4356430C9
:102B200002F066F9274B05F5AC40C4F8E4351430E3
:102B300002F05EF9244B05F5AC40C4F8143604F2FB
:102B40004463543083ED008A83ED018A83ED028A69
:102B500002F04EF91D4B2846C4F8543606B0BDECC1
:102B6000028BBDE8F08100BF80020F0888FC0E08D0
:102B700024FC0F0878880030A8F70F08A8030F0876
:102B800000000000DD22020874020F08DC3F0F087D
:102B9000CDCC4C3ECDCCCC3ECDCCCC3DCDCC4C3DAB
:102BA0003333333F9A99993FC4830030C283003056
:102BB000988300306C83003018FD0E0814490F080C
:102BC0005C480F08C8490F08B4480F0864490F084B
:102BD00038B5054B0A4601461C68236820461D6827
:102BE000024BA847002038BD60820030D82B00304F
:102BF00038B5037904463BB905682DB128461BF06A
:102C00004FF8284609F008FA204638BD2B4B70B51E
:102C10000360044600F56750043008F079FD04F5C0
:102C2000405393F8E02342B9D3F8DC532DB1284642
:102C30001BF036F8284609F0EFF904F5D85004F6F1
:102C4000EC7577F09DFB04F5B45004F68C760430F7
:102C5000FFF7CEFF04F5B3501C30FFF7C9FF04F5B2
:102C6000B3501430FFF7C4FF04F5A15014305DF0E9
:102C70008FFFB54204D0183D28461AF00FFCF8E744
:102C80000F4B04F63C50C4F8403AFFF7B1FF04F68E
:102C90003450FFF7ADFF04F62C50FFF7A9FF04F501
:102CA0003D6050F053FC04F63C3050F04FFC04F60D
:102CB000A82050F04BFC204670BD00BF1CD70F0869
:102CC00070A30F08094B0A4A10B5036000F5804352
:102CD0000446D3F84C0AC3F8E42808B109F0A0F977
:102CE0002046FFF793FF204610BD00BF80020F086B
:102CF00024FC0F0810B57AF027FE064C064B18602E
:102D00002046FFF7B1FD2046044A0549BDE81040C2
:102D1000C4F0ACBCD82B0030608200309C2C013059
:102D2000C52C020810B504460180024947F0F2FEA6
:102D3000204610BD70030F0800234FF07C524FF067
:102D40007E5110B5264C0365C0F88030C0F8903035
:102D5000C0F8A030C0F8C0304365C0F88430C0F877
:102D60009430C0F8A430C0F8C43083668367C0F8DC
:102D70009830C0F8A830C0F8B830C366C367C0F850
:102D80009C30C0F8AC30C0F8BC304FF03F43026715
:102D9000C0F8B0204267C0F8B420C0F88820C0F85E
:102DA000C820C0F88C20016644668465C1654FF474
:102DB0007A71C0F8CC3021205CF0B4FE4FF47A7107
:102DC00022205CF0AFFE4FF47A7123205CF0AAFE63
:102DD0004FF47A712420BDE810405CF0A3BE00BF20
:102DE000000080BF70B52DED068B037B82B00446DA
:102DF0009FED8A8A3BB980ED358A80ED368A80ED79
:102E0000388A80ED378AD4ED371A04F1100594ED35
:102E1000381AB7EE009AD4ED360A212694ED350A19
:102E20007F4800F07BFCB7EE001AFFEE000A582046
:102E300094ED350A1EF006FBB7EE001AFFEE000A0D
:102E4000592084ED350A94ED360A1EF0FBFAB7EEF0
:102E5000001AFFEE000A5A2084ED360A94ED380A73
:102E60001EF0F0FAB7EE001AFFEE000A5B2084EDC8
:102E7000380A94ED370A1EF0E5FA84ED370A7BF044
:102E80002DF907EE900A9FED677A2946F8EE677AEA
:102E9000DFED659A67EE877AC4ED027AD4ED353AB4
:102EA00094ED384AD4ED367A95ED105AD5ED145A92
:102EB00095ED186A23EE855A67EEA55AD4ED374A88
:102EC00024EE066AD5ED1C6A88FE055AB5EEC05A96
:102ED000C8FE255A64EEA66AB0EEC66A35EE257ABB
:102EE000F0EEE66AF1EE10FA37EE067AF5EEC05A29
:102EF000CCBF0123002337EE267AF1EE10FAB5EEAF
:102F0000C06AA5EC017A95ED233A85ED079A67EE44
:102F1000837A95ED1F3AE3EE837AD5ED273AE4EE16
:102F2000237A95ED2B4AE4EE847AC5ED037A84F892
:102F3000D030C2BF94F8D030013384F8D030F1EEF5
:102F400010FAF5EEC06AC2BF94F8D030013384F8AD
:102F5000D030F1EE10FAC2BF94F8D030013384F8CB
:102F6000D03094F9D030002BC1BF06EE903AF8EE85
:102F7000E66A87EEA66A85ED036AD5ED038AF0EE70
:102F8000E87A37EE277AB4EEC97AF1EE10FAC4BFC8
:102F900039EE677A05ED017A94F9E83015ED01AA6A
:102FA00073B1B4EEE9AAF1EE10FA09D89FED1F7AD9
:102FB000F4EEC77AF1EE10FAA4BF4FF08043EB6154
:102FC00094ED390AD5ED077A019120EE270AD4ED68
:102FD000027A20EE270ADFED167A30EE000A20EEA4
:102FE000270AC4F049FBEAEE008A30B201369FEDB1
:102FF000110AB6B228EE800AC5ED0B8A5CF06EFDB0
:10300000252E01997FF44AAF04F12002044802B052
:10301000BDEC068BBDE8704000F0B2BB00000000C4
:10302000D82B0030BD3786359A99193FCDCCCC3E90
:10303000DB0F494000007A440022C0F8D420C0F8D9
:10304000D820C0F8E020C0F8DC20FFF7CBBE00009D
:1030500000207047002070470120704790F8303002
:103060008B4286BF00EB8100406B00207047000060
:1030700090F830308B4286BF00EB8100406B00201F
:1030800070470000FA207047D0E9093242F4E0525C
:1030900043F4F8438262C26A436242F4E052C2627D
:1030A00070470000014802F007BC00BFD82B003079
:1030B00013B54FF45E70019108F0A6FF044620B1ED
:1030C000019959F0F1FB024B2360204602B010BD7C
:1030D000F0030F08704700007047000000207047A1
:1030E00070470000002070470020704700207047A4
:1030F00000207047002070477047000070470000B4
:103100000320704708207047064BD3F8CC3A3BB1F8
:103110001B7B002B0CBF5020D02040F001007047DB
:103120005020FAE7D86B003070470000704700006D
:10313000114BD3F8CC0AF0B1D0ED387A90ED367A55
:10314000F0EEE77AD0ED376AB0EEC77AF0EEE66AD5
:10315000C7FE877A90ED357AB0EEC77A87FE267A79
:10316000C7FE877A9FED057A67EE877AFDEEE77AEC
:1031700017EE903A18B27047D86B00300000C84282
:1031800053F076B810B5044654F08EFC054802F0B2
:1031900093FB054A034606212046BDE8104054F043
:1031A0006BBC00BFD82B0030DC030F0853F05EBBB4
:1031B000084608B508F0ECFB00280CBF04200020EE
:1031C00008BD0000162A01D053F088B80322012060
:1031D0000A70704759F074B808B553F0E1FA40F43A
:1031E0001C6040F00D0008BD10B5044608F014FF47
:1031F000204610BD08B5094B93F8B82AD2060BD467
:1032000003F58053D3F880050368DB6A98470028EC
:103210000CBF0220042008BD0120FCE7D86B003061
:10322000044B187820B9044B93F8B90AC0F3801006
:10323000704700BFB8820030D86B003000B5002363
:1032400089B002930393049304F064FC02A904F090
:103250001DFAA0B104F05EFC00F5607005AB07C874
:1032600083E80700184622F067FCF1EE047A20EEAE
:10327000270AFCEEC07ACDED017A9DF8040009B072
:103280005DF804FB7FB5002303930493059304F0DA
:1032900041FC03A904F0FAF9D8B104F03BFCD0EDED
:1032A000E00A90EDE10AF1EE600AB1EE400AC5F0E5
:1032B000BBF9DFED097A20EE270A1EF01FF8F6EEC3
:1032C000007A20EE270AFCEEC07ACDED017A9DF857
:1032D000040007B05DF804FBE02E65421FB5002333
:1032E00001930293039304F015FC01A904F0CEF9B5
:1032F00028B101A822F020FC05B05DF804FB12F013
:1033000047FBB02290F8F43202FB030090ED3B0A39
:10331000F2E700000C4B93F899208AB9A3F580538B
:1033200093F8C92A51070BD193F8B82AD20609D4C9
:1033300093F8B93A13F0020F14BF0420012070472C
:103340000520704703207047D87B00302DE9F04FEF
:10335000374E8DB0044696F8BC3A012B56D9A6F5E7
:103360008058344F082506F5A95617F901BBB8F95E
:10337000D03E0BF1FF3A43FA0AF3D90742D594F84D
:10338000280051F063F9814694F8280052F056F96C
:1033900000F12103994506D294F828000DB0BDE84C
:1033A000F04F52F015BEBAF1070F2BD8DFE80AF044
:1033B0003D0431333537393B1F4B5A69D868196999
:1033C000D3F804E0D3F818C0D3F800A008925A6AE2
:1033D0001B6ACDF825206222CDF8293021230690E2
:1033E0000791C22194F82800CDF80CA0CDF810E088
:1033F000CDF814C08DF824B0CDE90032192303AA0A
:1034000051F0A2F9013D15F0FF05AED10DB0BDE8B8
:10341000F08F0A4BD1E70A4BCFE70A4BCDE70A4BB7
:10342000CBE70A4BC9E73346C7E7094BC5E700BFFF
:10343000D86B0030D0040F08F47D00306C7E003073
:10344000E47E00306C7F0030987F003010800030C8
:10345000C87D0030084BD3F8FC2E920701D452F0FF
:1034600031BF03F50053DFED057A93ED2C0AB8EE7A
:10347000C00A20EE270A7047D85B00300AD7233CE9
:1034800010B594B0044603A808F060F91A4B03A9DC
:10349000D3F8800503685B6B984758B394F82840CD
:1034A0007AF024FE059B9622DDED047A57210893DD
:1034B000069BF8EEE77A9FED117A0993002367EEF9
:1034C000877A07900B9320460C930D930E930F93DE
:1034D0001093119312934FF6F853CDED0A7AADF88D
:1034E0004C3000238DF84E303323CDE9003207AA4B
:1034F00051F02AF914B010BDD87B00300AD7233C14
:10350000F0B5254D95B00E46074603AC0FCD0FC460
:103510002B682360731EDBB2042B2AD814AA02EB9B
:10352000830353F8445C2B6828461B6A98472B6832
:10353000044628469B6A98470023052297F828509E
:10354000089009938DF828208DF829608DF82A308D
:1035500094B9232221460DF12B00C7F00BFF8622E0
:103560002E2340F2B3112846CDE9003208AA51F0CB
:10357000EBF8052015B0F0BD20460DF12B0304F14A
:10358000200250F8041B904243F8041BF9D1028832
:103590001A8082789A70E2E7ECF80E08014802F08F
:1035A00089B900BFD82B0030014B93F8BC0A704793
:1035B000D86B0030024B93F8B90AC0F34000704753
:1035C000D86B0030164B30B505460C462DED028BFE
:1035D000D3F8800585B091ED018A0368DB699847CF
:1035E00028B9BDEEC88A18EE103ADB0712D5D4E927
:1035F00004011EF0E5F968B1684608F0A7F86A46CC
:103600002146284657F05EFF20B10649684608F07B
:10361000CBF900B1022005B0BDEC028B30BD00BF7C
:10362000D87B0030847C00308B8B162B05D0C02BD0
:1036300001D1FFF7C7BF59F01DBE00207047000041
:1036400030B5002305462DED028B8DB00393049316
:10365000059304F05FFA03A904F018F860B304F0CE
:1036600059FA00F5607306AC95F8285093E8070006
:1036700084E80700DDED060A9DED070AF1EE600A19
:10368000B1EE400AC4F0D0FF2046B0EE408A22F0EE
:1036900053FA089B0122DFED0A7AA8210B930C2331
:1036A00028EE278A28468DED0A0ACDE9003209AABC
:1036B0008DED098A51F048F80DB0BDEC028B30BD9C
:1036C000E02E6542242938B5054605D040290DD0A5
:1036D000BDE8384058F070BA0C2152F08BFC04461B
:1036E00010B12846FFF7ACFF204638BD0124FBE7A8
:1036F000F6EE007A08B591ED007AB4EEE77AF1EED5
:1037000010FA06DD012205210348FEF7A1FC002086
:1037100008BD0420FCE700BF407400302DE9F041F3
:1037200088B080461B22002101A810EE107A10EE0E
:10373000906A11EE105A11EE904AC7F01BFEA323B7
:103740008DF8043095238DF805300B238DF8063065
:103750007AF0D4FC1B22CDF80700CDF80B1008F549
:103760009B5001A9CDF80F70CDF81360CDF817501C
:10377000CDF81B404BF04AFE08B0BDE8F0810000D8
:1037800070B58CB00D46144606462B22002101A8C8
:10379000C7F0F0FDA3238DF8043095238DF8053094
:1037A0000C238DF806307AF0A9FC2B682B22CDF87B
:1037B000070006F59B50CDF80F302368CDF80B10AD
:1037C00001A9CDF813306B68CDF817306368CDF8D8
:1037D0001B30AB68CDF81F30A368CDF82330EB6801
:1037E000CDF82730E368CDF82B304BF00FFE0CB04E
:1037F00070BD000070B500F59B5500F5A34604466A
:103800000E2106F1700228464BF0C8FC06F19C021E
:1038100028460F214BF0C2FC04F5A5422846102192
:10382000143204F5A6464BF0B9FC04F5A64228462E
:1038300011210C324BF0B2FC06F1940228466C21A7
:103840004BF0ACFC06F1C00228466D214BF0A6FC03
:1038500004F5A84228460D2138324BF09FFC04F5B0
:10386000AA42284669212032BDE870404BF096BC40
:103870001FB500F5E450002301A91830019302930D
:10388000039302F0D9F905B05DF804FB08B504F024
:1038900041F9BDE8084003F0CBBD00007FB50E46FE
:1038A0004FF6FF710446154601F0ECFFE0B110221F
:1038B00000216846C7F05EFDA3238DF800309523F4
:1038C0008DF8013004238DF802307AF017FC1022B5
:1038D000CDF80300CDF8071004F59B5069468DF82C
:1038E0000B6003954BF012FE04B070BDB020704722
:1038F00038B500F59B55044601F0DEFF0C49024641
:1039000028464BF01FFF04F58043284693F8BD2A54
:1039100093F8BC1A4BF052FF04F5E450183004F051
:10392000B1FA04F59070BDE8384010F061BF00BFF7
:10393000DC030F0837B5069D044600B92C7801B9A1
:10394000697802B9AA7803B9EB78002064F307001C
:1039500061F30F2062F3174063F31F6003B030BDC3
:103960002DE9F04FE44CF7EE006ADFEDE45A9246A1
:1039700005460E46DFF8B4832DED0C8B9DB00D93FC
:10398000D4ED379A04F5804490ED006AD4F8CC3A2F
:10399000D3ED367A93ED387AF0EEE77AB0EEC77A67
:1039A00077EE877AF4EEE67AF1EE10FAC8BF86EE8B
:1039B000A78ADFEDD37AD8BFB0EE668A28EE277AE1
:1039C000A6EE257A80ED007AD4F8CC3A93ED357ADC
:1039D00093ED376AB0EEC77AB0EEC66A37EE067A74
:1039E000B4EEE67AF1EE10FAC8BFC6EE878A90ED23
:1039F000017AD8BFF7EE008A68EEA77AE7EE257A5B
:103A0000C0ED017A4CF0C0FB07467AF077FBB7EEC9
:103A1000E87AB7EEC88ABB4BBB4A8DED087B8DEDCB
:103A2000068B95ED017AB7EEC77A8DED047B95EDA7
:103A3000007AB7EEC77ACDE900018DED027B3846FA
:103A4000B249B34F4CF012F9B249304697ED00AA93
:103A500021F03EFC8DED160A9AED000ACDED170A15
:103A600030EE4A0A8DED181A1DF0C0FC9DED167A55
:103A700008F56F63B0EEC77AD3ED007AA7F56B63F4
:103A8000B4EEE77A0B93F1EE10FA00F11582D4F858
:103A9000CC3A1B7B002B00F00F82B8F8EE9EC9F3E6
:103AA00040099DED177AB0EEC77AF4EEC77AF1EED1
:103AB00010FA00F30482D4F8CC3A1B7B002B00F000
:103AC000FE81B8F8EE3E03F001039DED187A0A93EB
:103AD000B0EEC77AF4EEC77AF1EE10FA00F3F18196
:103AE000D4F8CC3A1B7B002B00F0EB81B8F8EE3E0B
:103AF000C3F38007B0EEC00AF4EEC07AF1EE10FA1C
:103B000000F3E181D4F8CC3A1B7B002B00F0DB8181
:103B1000B8F8EE3EC3F3C00B0DAB3A460A994846DF
:103B200000935B46FFF706FF9FED7B8AC3B20F90C1
:103B30000BEE103AC0F307230AEE903AC0F30743A6
:103B40000CEE903A030E0DEE103A9DF83430002B37
:103B500040F0BC819DF83530002B40F0B781F8EE85
:103B60004B7A6C4AB0EE690A19AB314602F5207007
:103B7000CDED197AF8EE6A7ACDED1A7AF8EE6C7A14
:103B8000CDED1B7A6BF028F9B0EE409A8DED140A5A
:103B9000F0EE608ACDED150A9DF836305F4C002BB3
:103BA00040F09981B0EE691A1CEE901AD4ED370AF4
:103BB00004F5816096ED020A6BF02CFAB0EE40CA73
:103BC0009DF83730002B40F089819AED000A30EEE5
:103BD0004A0A1DF00BFC5248F0EE690A1DEE101A5D
:103BE0006AF02EFFF0EE40BADAF800304C48C0F828
:103BF000A03080ED29AA08F6D463B0EE490A472028
:103C000093ED001A0C93F1EE410A1DF01BFC0C9B86
:103C1000B0EE40AA482093ED001AB0EE680AF1EE2B
:103C2000410A1DF00FFC08F6D86308F6DC68B0EE18
:103C3000409A93ED001A4920B0EE4C0AF1EE410A89
:103C40001DF000FC98ED001AF0EE408A4A20B0EE1C
:103C50006B0AF1EE410A1DF0F5FB95ED007AD5ED0A
:103C6000017AF0EE40BA6AEE076A9DF834308DEDC5
:103C7000148A8DED158ACDED106A69EE276ACDEDB7
:103C8000116AD4ED326A27EE267AD4ED336A67EEF4
:103C9000A67A8DED127ACDED137AB3B99DF8353051
:103CA0009BB9B0EE690A19ABB8EE4BBA12AAF8EE9E
:103CB0006AAA10A91B488DED19BACDED1AAA6AF0AF
:103CC00077FF8DED140ACDED150A9DF83630002BE7
:103CD00040F0078195ED000AB0EE691AD4ED340A80
:103CE0001CEE901A104860EE200A28EE800A6BF055
:103CF00091F9F0EE40AA1BE0D82B0030A4707D3F74
:103D000000D7233C120B0F08D03C0F08E93C0F08EA
:103D1000884A0030AC7C003000000000D87B0030C6
:103D200058800030887D00303C7E0030D85B003009
:103D300014A98448FEF780FD9DF83730002B40F031
:103D4000D38095ED010AB0EE691AD4ED390A1DEE63
:103D5000101A7D4860EE200A20EE2B0A6BF05AF90B
:103D6000F0EE409A794DD5F8CC3A1B7B83BB19A96C
:103D700077488DED198A8DED1A8A6BF043F89FED27
:103D8000750A75486BF062F99FED720A05F5A4504B
:103D90006AF082FE19A971488DED198A8DED1A8A93
:103DA0006BF030F89FED6B0A6D486BF04FF9664889
:103DB0009FED680A6BF04AF904F1D40393E8070019
:103DC0000B9B03F56B6386E807001B68CAF800309D
:103DD000B9F1000F00F08B80D5F8CC3A83ED368A2C
:103DE0000A9B002B00F08E80D5F8CC3A83ED358A03
:103DF000002F00F09280D5F8CC3A83ED388ABBF1E1
:103E0000000F00F09480D5F8CC3A83ED378A9FED0F
:103E1000558A9FED504AD4ED322A2AEE082A94EDB5
:103E2000351AF0EE443AD6ED000AB0EE443A62EEAE
:103E3000882AF0EE441A21EE081A60EE880AB0EEE5
:103E4000440A79F011FA9FED434AD4ED332A29EE62
:103E5000082A94ED361AF0EE443AD6ED010AB0EE97
:103E6000443A62EE882AF0EE441A21EE081A60EE17
:103E7000880AB0EE440A79F0FBF99FED364AD4ED9A
:103E8000342A28EEC82A94ED371AF0EE443AD6EDDB
:103E9000020AB0EE443A62EEC82AF0EE441A21EE6D
:103EA000481A60EEC80AB0EE440A79F0E5F91DB090
:103EB000BDEC0C8BBDE8F08F4FF00109F1E501235B
:103EC00003E6012716E64FF0010B25E6F0EE488ADF
:103ED000B0EE489A60E69FED1FCA71E6DFED1DBAAD
:103EE00089E6DFED1CAA23E7DFED1A9A3AE79DF891
:103EF0003430002B7FF474AFD5F8CC3A149AC3F861
:103F0000D8206DE79DF83530002B7FF471AFD5F8E0
:103F1000CC3A159AC3F8D4206AE79DF83630002BC6
:103F20007FF46DAFD5F8CC3AC3ED38AA67E79DF8BA
:103F30003730002B7FF46BAFD5F8CC3AC3ED379A0E
:103F400065E700BFD82B0030B47E0030D86B00305E
:103F50002C7F003000000000E07F0030887D0030C2
:103F60003C7E00300000C8422DE9F04F2DED068B5D
:103F700091B080460D460593B84B039203F58046F9
:103F8000D3ED37AAD6F8CC2A127B002A00F035816F
:103F900003F54053B3F8EE4EC4F3400B04F0010AAE
:103FA000C4F3800914F0080400D0012405ABAC4F21
:103FB00051464A46009358462346FFF7BBFC97ED0F
:103FC000001A95ED000AF1EE410A07909A201DF0C3
:103FD00039FA3A46F0EE409A9B20B2EC011A95ED80
:103FE000010AF1EE410A04921DF02CFA049AB0EE97
:103FF000409A9C2092ED001A95ED020AF1EE410ADA
:10400000984D1DF01FFA97ED021A039BF0EE408ABF
:10401000F1EE410A9D2093ED000A00271DF012FAEF
:1040200098ED007AD8ED017AB0EE408A69EE876AA1
:104030009DF814300C970D97CDED086A69EE276A4C
:10404000CDED096AD5ED326A27EE267AD5ED336AD1
:1040500067EEA67A8DED0A7ACDED0B7AFBB99DF865
:104060001530E3B99DF81C30B0EE6A0A0AAA08A917
:1040700007EE103A9DF81D3005F5D87007EE903A1E
:10408000B8EE477A0EABF8EE677A8DED0E7ACDED8D
:104090000F7A6AF08DFD8DED0C0ACDED0D0A9DF8BD
:1040A0001630002B40F0AE8098ED000AB0EE6A1A90
:1040B000D5ED340A9DF81E1060EE200A6A4828EEFD
:1040C000800A6AF0A7FFB0EE40AA0CA96348FEF789
:1040D000B3FB9DF81730002B40F0978098ED010A54
:1040E000B0EE6A1AD5ED390A9DF81F1060EE200A6D
:1040F0005E4820EE080A6AF08DFFB0EE408AD6F8DE
:10410000CC3A1B7B7BB90EA959480E970F976AF0E2
:1041100079FE9FED580A54486AF098FF9FED550AC2
:1041200052486AF093FFBBF1000F71D0D6F8CC3A39
:10413000C3F8D870BAF1000F74D0D6F8CC3AC3F8EF
:10414000D470B9F1000F77D0D6F8CC3AC3F8E0704C
:10415000002C7AD0D6F8CC3AC3F8DC709FED468AB2
:104160009FED444AD5ED322A29EE882A95ED351A7D
:10417000F0EE443AB0EE443A62EE882AF0EE441A89
:1041800021EE081AF0EE440AB0EE440A79F06CF819
:104190009FED384AD5ED332A29EE082A95ED361AD7
:1041A000F0EE443AB0EE443A62EE882AF0EE441A59
:1041B00021EE081AF0EE440AB0EE440A79F058F8FD
:1041C0009FED2C4AD5ED342A28EEC82A95ED371AF2
:1041D000F0EE443AB0EE443A62EEC82AF0EE441AE9
:1041E00021EE481AF0EE440AB0EE440A79F044F8A1
:1041F00011B0BDEC068BBDE8F08F4FF00109CA4647
:10420000CB46D2E69FED1BAA5FE79FED1A8A76E7C1
:104210009DF81430002B8DD1D6F8CC3A0C9AC3F807
:10422000D82087E79DF81530002B8AD1D6F8CC3AF4
:104230000D9AC3F8D42084E79DF81630002B87D15F
:10424000D6F8CC3A83ED38AA82E79DF81730002BD8
:1042500084D1D6F8CC3A83ED378A7FE7D82B00306B
:10426000AC6A0030D87B00303C7E0030B47E003039
:10427000887D0030000000000000C84270B5044690
:10428000103059F083FDA0250A4B0B4E23616019B5
:104290005AF056F866513035B5F5687FF7D104F518
:1042A00068705BF01DFE2046044946F033FC204652
:1042B00070BD00BF2C460F0818460F084C3F0F0872
:1042C00037B500F57A5101220446283149F096FAB3
:1042D0001E4A1368D9070AD404F559531C491033F0
:1042E0000B6004F56E532433CB600123136004F597
:1042F0007B50022216490125383045F0DFFF0023AC
:10430000144A04F59B51FD20CDE9005345F068FFA8
:10431000114B1A68D20705D404F5D8540F4A1D6012
:104320001C34146001210D4845F0E4FF46F0E4FD23
:104330000B4A04210B48138843F0400313800022EA
:1043400003B0BDE8304045F047BF00BF6482003095
:10435000C425003014DE0F0868820030DC250030F0
:10436000A48300303C440F080069C0F3401070473C
:104370000F299DBF302303FB0100903000207047C0
:10438000014B93F9C20E7047D85B0030024B93F893
:10439000C90A00F001007047D86B0030014BD3F818
:1043A0005C087047D86B0030002910B517DB104C43
:1043B000CBB294F864289A4211D3D4F86038012221
:1043C000A4F58040595C00F083FD94F8B93A38B9FF
:1043D0009A0704D5074A137843F00403137010BDFD
:1043E0009B07FCD5034A137843F00203F6E700BFAE
:1043F000D86B00302C830030022A10B50F4C12D13C
:104400003522A4F5804000F063FD94F8B93A9B078B
:1044100005D50B4B1A7818B142F002021A7010BD84
:1044200042F00402FAE794F8BC2A8A42F7D159F024
:10443000B1FEBDE8104059F09BBD00BFD86B003005
:104440002C830030064A92F8C93A92F8C82A03F041
:104450000103134301D159F085BC0020704700BF10
:10446000D86B0030332901D05AF026BF70470000C6
:1044700008B50A68332A07D0382A08D10A790321F7
:10448000FFF7BAFF012008BD0A790121F8E7BDE86E
:1044900008405AF089BB000030B5044689B004F5E5
:1044A000E455684607F052F904A8183507F04EF9AC
:1044B0006946284603F060F878B104A9284603F05D
:1044C000FDF850B104A9684607F06EF92368002290
:1044D0006946D3F8B8302046984709B030BD00008F
:1044E00000F5805292F82C2FD2070BD400F58042B1
:1044F000D2F8CC2A117B09B1FFF7CEBF0368D3F8FD
:10450000B43018477047000010B586B0044602A8C2
:10451000019107F01BF904F5E45002A9183003F0EB
:104520002BF830B1236802A9019A2046D3F8B8309D
:10453000984706B010BD0000F0B5044685B00F46A0
:10454000154604F5E456684607F000F96946183642
:10455000304603F0B3F810B9002005B0F0BD39467D
:10456000304602F03BFE0028F6D0002DF5D004F5D1
:104570008054284694F82C3F43F0020384F82C3FE3
:10458000EBE7000010B500F57B548AB00023D4EDB2
:10459000037A0C34F5EEC07AF1EE10FA44D90793A1
:1045A00000F5E450089303AA099306AB04A9183058
:1045B000019307AB009305AB02F0AEFEDDED087A88
:1045C0009DED077A87FE277ADDED097A87FE277A47
:1045D000D4ED007AB4EEE77A9DED047A77EEA76A1F
:1045E000F1EE10FAF4EEC76AACBF01200020F1EE44
:1045F00010FA0CD802309DED037AF4EEC77AF1EE92
:1046000010FA0CD8003818BF01200AB010BDF4EE23
:10461000C77AF1EE10FA9CBF0130C0B2EBE7012877
:1046200094BF00200120F0E70020EEE700F5804273
:1046300010B592F8C93A044659071CD443F0040354
:1046400082F8C93A4BF0A0FD012211214BF0F8FC91
:10465000094BD3F8800503689B68984728B904F58F
:10466000405393F9C93E032B05D120460621BDE8EE
:10467000104000F029BD10BDD87B003000F580400F
:1046800008B590F8C93A5A070BD56FF3820380F842
:10469000C93A4BF079FD00221121BDE808404BF0EA
:1046A000CFBC08BD2DE9F043054685B005F5E458BB
:1046B000684607F04BF8694608F11808404602F0D2
:1046C000FDFFD8B105F58043434C444FD3F8CC3AB5
:1046D0001B7B43B105F57B53D3ED037AF5EEC07A2E
:1046E000F1EE10FA0DD82388284623F4FF7323F047
:1046F000010323800023FB73FFF7C0FF05B0BDE873
:10470000F083284601F07CF8064618B9284601F0E7
:104710003BF806462846FFF735FF814640B93EB1D3
:104720002378002B41D1637803F00103FB73E5E7A5
:104730006378DB07F7D423780133DBB2082B2370CF
:1047400006D12846FFF71EFF10B1404602F064FE76
:104750002378092B02D1404602F056FE2378092B1C
:10476000E1D9238823F4FF7323F0010343F4857315
:1047700023804BF009FD022210214BF061FC79F0FF
:10478000B5FC6368C01A47F23053984209D905F561
:104790009140134A0221643051F0CAF979F0A6FC25
:1047A00060602846FFF742FFBDE7013B2370238886
:1047B000C3F30803B3F5807FB5D1637860F30003DA
:1047C00063704BF0E1FC4A4610214BF039FC28465F
:1047D000FFF754FFA7E700BF6C8200300D83003065
:1047E00048460F0837B5044600F5E45001A904F522
:1047F0008045183002F036FCD5F8D038834206D018
:10480000C5F8D0084BF0C0FC3E214BF0F9FB04F595
:10481000805395F9D41893F8C02F93F9C03F99426B
:1048200013D0FF2A11D085F8D4384BF0ADFC95F8A1
:10483000D42818214BF004FC04F5914095F9D438A4
:104840000421034A643051F073F903B030BD00BF56
:1048500058460F082DE9F043064695B079F046FC1E
:10486000002403AB06F5E45805460BAA019308F1B2
:10487000180802AB08A94046089400930EAB0994AF
:104880000A940B940C940D940E940F94109402F0CF
:1048900031FDDFED437A07469DED0A7AB4EEE77A03
:1048A000F1EE10FA37DB9DED0D7AB4EEE77AF1EE1A
:1048B00010FAACBF4FF001094FF0000907AB11949B
:1048C000129404AA019311AB139406F5804400934B
:1048D00005A906AB404602F01FFD94F944380028B4
:1048E00008BF002783B17FB1D4F8CC3A1B7B5BB102
:1048F000B9F1000F08D0F7EE007A9DED057AB4EE1D
:10490000E77AF1EE10FA09D594F8D83873B9002394
:10491000C4F8DC380FE04FF00009CFE7D4F8DC082A
:1049200020BBC4F8DC58C4F8E00804E0D4F8E00880
:1049300020B9C4F8E05815B0BDE8F083281A43F652
:1049400098239842E3D9002584F8D858C4F8E05851
:104950004BF01AFC2A461D214BF072FB06F59140E4
:10496000104A0221643051F0E3F8D0E72D1AB5F572
:104970007A7FE0D994F8D838002BDCD1012584F86F
:10498000D8584BF001FC2A461D214BF059FB06F587
:104990009140054A0221643051F0CAF8CBE700BFCC
:1049A0000000003470460F088B460F0810B504460F
:1049B0004BF0EAFB002205214BF042FB04F591404D
:1049C000034A04216430BDE8104051F0B1B800BF83
:1049D000A8460F0800F5804090F8B93A9B065ABFE8
:1049E00090F8B80AC0F300100120704738B50446AB
:1049F00003F090F84FF4804102F000F904F5804292
:104A0000054692F8B93AC3F3001181421CD060F315
:104A1000041304F5914482F8B93A643460B14BF060
:104A2000B3FB02220B214BF00BFB084A204602216C
:104A3000BDE8384051F07CB84BF0A6FB2A460B216C
:104A40004BF0FEFA024AF1E738BD00BFC0460F083E
:104A5000CB460F0800F5405370B593F9B23E0446BB
:104A6000C3B300F58045D5F8446A9EB379F03EFBA8
:104A700005F64C03DFED187A861B93ED000A6920DA
:104A80009FED161A20EE270ADFED150A1CF0DAFC5E
:104A9000BCEEC00A10EE103A9E4209D295F8C93A0F
:104AA0009A0717D520460021BDE87040FDF778BB76
:104AB00010D995F8C93A9B070CD420460121FDF77F
:104AC0006FFB04F59040012212216830BDE8704070
:104AD000FDF7BEBA70BD00BF00007A440000804FF1
:104AE000000000000B461146012B10B404D0052B2A
:104AF00006D05DF8044B70475DF8044B00F0E4BA53
:104B000000F59040012214215DF8044B6830FDF758
:104B10009FBA0000F8B504464BF036FB0122052190
:104B20004BF08EFA04F5405304F59146204693F974
:104B3000B65E6436003D18BF0125FFF74BFF98B104
:104B40001E4A04213046002550F0F2FF04F5904043
:104B5000012210216830FDF77BFA29462046032206
:104B6000BDE8F840FFF7BEBF04F5A047D7F88005C1
:104B70000368DB6A984768B197F8993053B197F9A1
:104B80009830012B06DC0E4A04213046012550F0F6
:104B9000CFFFE2E7D7F880050368DB6A984728B1C2
:104BA00004F58043D3F848381B0705D4054A04218F
:104BB000304650F0BDFFD0E7034AE5E7E0460F0876
:104BC000FB460F0829470F0838470F0870B5044601
:104BD00015464BF0D9FA0122062104F591464BF017
:104BE0002FFA20466436FFF7F5FE98B104F59040A1
:104BF0000122072100256830FDF72AFA144A042112
:104C0000304650F095FF294620460422BDE870400A
:104C1000FFF768BF04F5A043EDB2D3F88005036841
:104C2000DB6A984768B104F58043D3F848381B071E
:104C300007D535B1074A04213046012550F078FFE9
:104C4000E1E7054A0421304650F072FFDBE700BF80
:104C50005C470F0803470F0879470F08F8B504466B
:104C600079F03CFA284B0546B4F8BE201988274E47
:104C700091420ED01A80264B18603378A3B10024DD
:104C800034704BF081FA22461321BDE8F8404BF016
:104C9000D7B933781F4FC3B93B782BB11C4B1E4A91
:104CA0001B68C31A934200D8F8BD0123337004F582
:104CB0008043D3F8CC0A037B0BB1FEF7BDF94BF070
:104CC00063FA012213214BF0BBF93B78002BEBD0A8
:104CD0003378002BE8D00E4A10491368EB1A8B4248
:104CE000E2D904F580441560D4F8CC2A137B002B5C
:104CF000DAD0002313730A4AD4F8CC0A1371BDE842
:104D0000F840FEF76FB800BF768200307482003042
:104D1000788200307582003080841E0040420F008F
:104D20000D8300307FB5044600F5A34500F58043B0
:104D3000143504F5E45693F8D8182846183678F058
:104D400085F9684606F002FD6946304602F014FC1B
:104D500004F5A043029A20213046C3F8B420039AF8
:104D6000C3F8B82001F04AFFD0B1284604F5A145A8
:104D700078F0BEF9FDEEC07A2C3504F5805402229D
:104D800017EE901A284617EE906A06F0E3FC94F8A6
:104D90002C3FDB0706D401223146284606F0DAFC18
:104DA00004B070BD0121284606F0AEFD0028F2D007
:104DB000F6E7000001207047002070470020704790
:104DC0000020704700207047002070470020704787
:104DD000002070479FED010A704700BF00000000EF
:104DE0009FED010A704700BF0000000070470000FF
:104DF0000F4A02600F4A02F15001426081600E4981
:104E0000C1600E49016102F62441416102F6284168
:104E1000816102F6A811C16102F6AC11016202F5CE
:104E20001B6102F6B41241628262054AC262704797
:104E300004480F08806A00306C7D003070480030F4
:104E4000F02C0030042918D8DFE801F003070B0F1D
:104E5000130000F5AB403430704700F5AB40043030
:104E6000704700F5AB406430704700F5AC4014303B
:104E7000704700F5AC405430704700207047000088
:104E800000F5A040D0F8800503685B681847000073
:104E900038B500F5A0450446D5F8800503685B6980
:104EA00098470A4B04F58042187492F8BC2AD5F84A
:104EB0008005DA7003685B6A9847014604F5E250A2
:104EC000BDE83840043042F071B900BF0D830030B6
:104ED0002DE9F84F00F5804A06460F4691469AF8AC
:104EE000BC3A8B4205D101258AF8BD2A2846BDE887
:104EF000F88FFFF7A7FF044620B93046254648F053
:104F000039FEF3E7DAF8CC3A06F591481B7B08F155
:104F1000640883F0010BE3B92368594620461B68F7
:104F20009847054678B306F5A0434A46394606F544
:104F30009B50C3F880458AF8BC7A8AF8BD9A4AF03B
:104F40003DFC4046002158F045F93046FFF7A0FFF0
:104F5000CCE703689B689847E0B11C4800F03AFC36
:104F60000546B8B9236820461B6A9847184A034685
:104F70000421404650F0DCFD4BF006F93A460A2188
:104F80004BF05EF8B2E7236820461B6A9847114A47
:104F90000346EDE70D4800F03BFC0028BCD106F5C8
:104FA000A043D3F880050368DB6898470028B3D096
:104FB00023682046DB68984705460028ACD1236863
:104FC00020461B6A9847044A0346D1E7D82B003095
:104FD0008C470F08DE470F08B5470F080148FFF759
:104FE00077BF00BFD82B0030234B70B593F8C93A78
:104FF00005460C461646DB0705D500236360236093
:10500000A360336070BD59F0C5F8037F002BF4D066
:10501000EB699FED1A7A1B68B3F90A3007EE903AF4
:10502000F8EEE77AC7EE876AC4ED016A2B6A1B685F
:10503000B3F90A3007EE903AF8EEE77AC7EE876ADE
:10504000C4ED006A6B6A1B68B3F90A305B4207EE75
:10505000903AF8EEE77AC7EE876AC4ED026AAB6A67
:105060001B68B3F90A3007EE903AF8EEE77AC7EE1C
:10507000876AC6ED006AC5E7D86B003000007A4445
:1050800000207047012070470020704700207047C3
:1050900000487047ECAD0F08004870474C480F08B7
:1050A0000020704743691A680023C2F8D43042696F
:1050B0001268C2F8D83042691268C2F8DC3042691E
:1050C0001268C2F8E03070470A46002108B5FFF7C1
:1050D000FFFE034A137843F00803137008BD00BFB6
:1050E0002C8300300120704700207047012070475A
:1050F00000207047004870472003100800487047A0
:10510000A4480F0803207047084B03F5A14203F59C
:10511000F5535432103330B5044600F1300507CA58
:1051200085E807001B680120E36330BDD82B003001
:1051300030B52DED028B87B000230446564D01AAF1
:1051400003A995ED378A039304930593FFF74CFF6A
:1051500063689DED037AD3ED0E7A68EE277A27EE29
:10516000277A8DED037A9DED047A67EE277ACDEDEF
:10517000047AD3ED0F7A28EE277ADDED057A67EE13
:10518000877ACDED057AD3ED107A93F9443028EE85
:10519000278ADDED017A27EE888A8DED018A1BB919
:1051A00003A92846FDF730FB3C4A94ED0C7AD2ED7A
:1051B000357A636877EE677A94ED0F0AD3ED0E6A5D
:1051C000F0EEE77AF4EEE67AF1EE10FA44BFDDEDA8
:1051D000037A77EE877A94ED0D7A48BFC4ED0C7AA6
:1051E000D2ED367AD3ED0E6A77EE677AF0EEE77A93
:1051F000F4EEE67AF1EE10FA44BFDDED047A77EED4
:10520000877A94ED0E7A48BFC4ED0D7AD2ED377AE5
:10521000D3ED0F6A77EE677A2369F0EEE77AF4EE62
:10522000E67AF1EE10FA42BFDDED057A77EE877A85
:10523000C4ED0E7AD3ED867A30EE670A1CF0D6F80C
:105240006368B0EEC00AD3ED107AB4EEE70AF1EE6F
:1052500010FA09D594ED0F0ADDED017A30EE270A38
:105260001CF0C4F884ED0F0A00230D4804F13C0241
:1052700004F130018DF808308DF809308DF80A30CE
:105280008DF80B30029BD0F8D00AFEF769FB07B00F
:10529000BDEC028B30BD00BFD82B0030D87B003076
:1052A000D86B003000207047012070470120704704
:1052B0000020704700487047FC480F0800487047BE
:1052C00004490F08012070471FB5044600236A46B1
:1052D00001A9019302930393FFF786FE6369029A83
:1052E0001B68C3F8D4206369019A1B68C3F8D820EF
:1052F0006369009A1B68C3F8DC206369039A1B6822
:10530000C3F8E02004B010BD0120704700207047B2
:1053100001207047002070470048704720110F0897
:105320000048704720110F08042070470120704783
:105330007FB500230B4801AA03A9039304930593A7
:1053400001930023D0F8D00A8DF808308DF8093089
:105350008DF80A308DF80B30029BFEF701FB07B089
:105360005DF804FBD86B00300120704700207047C7
:10537000012070470020704700487047AC490F0873
:1053800000487047B8490F080220704710B586B032
:105390000023044601AA03A9039304930593FFF78E
:1053A00023FE63689DED037AD3ED0B6ADDED047A8D
:1053B00027EE267A93F9443067EEA67A8DED037ACC
:1053C000CDED047A1BB903A91348FDF71DFA6368F4
:1053D00001AADDED057A03A993ED0C7A0F4867EE7B
:1053E000877A93ED0D7A0023D0F8D00ACDED057AB7
:1053F000DDED017A8DF8083067EE877A8DF8093097
:105400008DF80A308DF80B30029BCDED017AFEF756
:10541000ABFD06B010BD00BFD82B0030D86B0030FC
:1054200038B504465AF0C8FD5AF016FF054604F593
:1054300080445AF0A3FE5AF047FAD4F8CC0AFDF79C
:10544000D1FC2846BDE838405AF0A0BE10B500F5A2
:1054500080441421D4F8500858F086FFD4F854083A
:10546000142158F081FFD4F858081E2158F07CFF11
:10547000D4F85C081421BDE8104058F075BF000056
:1054800038B5054658F086FE58F0D2FD05F5804443
:10549000C4F8500858F07EFE58F0D4FDC4F8540803
:1054A00058F078FE58F0D8FDC4F8580858F072FE4D
:1054B00058F0DCFD4FF47A71C4F85C08D4F8500859
:1054C00058F04EFF4FF47A71D4F8540858F048FF62
:1054D0004FF47A71D4F85C0858F042FF4FF47A71B7
:1054E000D4F8580858F03CFF2846FFF7AFFF94F86F
:1054F000B93A43F0080384F8B93A38BD08B55AF010
:10550000ABFE5AF09DFBBDE808405AF04FBB0000CF
:1055100000F58040D0F8CC0AFDF78EBD38B500F517
:105520004053054693F9B62E2AB900212846BDE816
:105530003840FCF71BBEB3F8B83E00F580448B4200
:1055400019D994F8C93ADA070FD458F023FE037F2B
:105550001BB9D4F8CC3A1B7B3BB194F8C83A013361
:105560005BB2022B02DC84F8C83A38BD0323012168
:1055700084F8C83ADAE794F8C83A013B5BB2002BEA
:10558000F1DC002384F8C83A94F8C93ADB07CCD49C
:10559000EBE7000038B50D46044678F0A7FD0C4B4C
:1055A000002D09DD04F58044186094F8B93A6FF3D2
:1055B000C30384F8B93A38BD1B68C01AB0F5C87F78
:1055C000F9D904F5804494F8B93A43F00803F0E7B8
:1055D0007C820030F7B5044678F088FD064658F026
:1055E000D9FD04F5804558F0A7FDB0B395F8B83A59
:1055F000204604F5A04743F0200385F8B83AD5F8D3
:1056000058381989FFF78AFFD5F858382046B3F97A
:105610000A10FFF7BFFFD7F878359FED307A04F511
:10562000A140F31A6A4601A9203007EE903AD5F856
:105630005838F8EE677AB3F90A3067EE877ACDED1D
:10564000007A07EE903AF8EEE77ACDED017A4DF068
:1056500069F8C7F8786503B0F0BD95F8C93ADB077B
:10566000F9D404F5A043D3F87805361A58F032FC83
:1056700088BB58F08FFD9FED1A7AD0ED067A67EE61
:10568000877A9FED187AF4EEC77AF1EE10FA77FE7A
:10569000877AFCEEE77A17EE903AB342DBD804F54E
:1056A000405393F9B63E002BD5D058F073FD037FDD
:1056B00023B9D5F8CC3A1B7B002BCCD04AF064FD43
:1056C000022211464AF0BCFC0121204603B0BDE88D
:1056D000F040FCF74BBD4FF47A73DEE76F12833A6C
:1056E00000007A440000C84238B500F5AA650446B7
:1056F000284604F0F9FD94F8610550229FED077AE1
:1057000004F5A04302FB0055D5ED0B7A67EE877ACE
:10571000FDEEE77AC3ED277A38BD00BF0000C8422E
:10572000FEF7E6B80148FFF799BA00BFD82B003062
:1057300010B5838F044643B948F04EFF92224FF4D0
:10574000801148F001FF638FA387A08F10BD000078
:1057500038B500F5E45504461835284600F0E6FC57
:1057600004F58053022204F1680083F8B82EFFF795
:10577000DFFF014604F524601BF062F92846BDE80E
:10578000384000F0D9BD000038B500F5E4540546B6
:105790001834204600F020FF08B9002038BD05F578
:1057A0008045D5F8CC3A1B7B63B91021204601F027
:1057B00025FA0028F2D14FF400712046BDE83840A8
:1057C00001F01CBA8021204601F018FA0028E4D12B
:1057D0001021F2E738B500F58043054693F8C93A41
:1057E0005B070AD4FFF7D0FF044620B905F5E45063
:1057F000183000F0F1FE204638BD0024FBE7000021
:1058000000F5E45008B5183000F0E6FE002008BDB1
:1058100010B500F5E4541834204600F0DDFE50B118
:105820000421204601F0EAF928B120462021BDE8F4
:10583000104001F0E3B9002010BD000038B500F5BC
:105840008045044695F8B83A590719D5D5F8CC3AA9
:105850001B7B2BB920460021BDE83840FCF770BC0B
:1058600000F5A043D3F880050368DB68984738B19A
:1058700095F8B93A1A0703D595F8C93ADB07E9D57F
:1058800038BD000037B5044600F59B55019104F57D
:105890008044284649F0DAFE019994F8B83A60F35A
:1058A000C303284684F8B83A03B0BDE830404AF054
:1058B00035BC00000720704700487047104A0F08A9
:1058C00037B505461148FFF733FF0190EC2006F08D
:1058D0009BFB044610B10199FDF724FA05F58043BE
:1058E000C3F8CC4A34B905F54055094895F9041F69
:1058F00005F0E4FE0749204645F006FB012044F090
:10590000A3FF03B0BDE8304045F0F6BA402C0030AC
:10591000184A0F0870030F0873B5044600F5E250EB
:10592000043004F5AA6641F0A9FB2046FFF7B0FA5F
:1059300004F59540603005F0C7F804F5A150143027
:105940005BF02EF9304604F055FB04F591406430CD
:1059500053F0C2F82046FFF793FD2046FFF7B0FF53
:105960006048FFF7E5FE082006F04EFB18B14FF047
:105970007E530360436004F58045C5F8D00A58F0B3
:1059800009FC9922292159F0DFFE58F003FC58F058
:105990000DFB2046FFF7B2FD95F8B93A04F5E0504B
:1059A00043F04003103085F8B93A5DF0E3FF4E4B09
:1059B0004FF47A724D491B68986A0368DB6A98470E
:1059C000042304F59070C4F8A4310EF02BFA07F00C
:1059D000EBF84FF40053436307F0E6F807F012FECC
:1059E000802301213046C4F8643504F09DFD404B0E
:1059F00004F59B5000933F4B019302AB13E9060063
:105A000049F0D0FC2046FFF7A3FE4FF40023C4F872
:105A1000503ED5F8CC0AFDF78FF904F590400121EE
:105A20006830FCF77DF810B12046FFF771FD04F1F6
:105A300068063046FFF77CFED5F8CC3A07EE900AB0
:105A400004F5A140D3ED390AF2EE0E1AB8EE670A5A
:105A50006830B6EE001A4DF05BFB3046FFF768FE8B
:105A6000D5F8CC3A07EE900A04F5A240D3ED390AF6
:105A7000F2EE0E1AB8EE670A2C30B7EE001A4DF0AF
:105A800071F93046FFF754FED5F8CC3A07EE900A8C
:105A900004F5A240D3ED390AF2EE0E1A6030B1EEF1
:105AA000041AB8EE670A4DF05DF904F540531A2266
:105AB000204693F8C31EFFF70BFA60B9212201219B
:105AC0002046FFF705FA95F8B93A43F0020385F846
:105AD000B93A02B070BD084A137843F00803137056
:105AE000F1E700BF402C00306082003025570208EB
:105AF000D82B0030215702082C830030836833B93B
:105B0000C36823B94068003818BF012070470120DE
:105B1000704700002DE9F0412DED048B92B0044652
:105B200002AD284605F012FE94F8D433002B70D055
:105B300004F58063D4EDF28A94EDF38A94EDF49A3F
:105B40000FCB85E80F0094F81034002B61D094F847
:105B5000E833002B5DD02846D4F8D883D4F8DC7322
:105B6000D4F8E063D4F8E443FFF7C8FF002855D128
:105B70002E4B01932D22002106A8C5F0FBFBA32389
:105B80008DF8183095238DF8193046238DF81A308A
:105B900078F0B4FA9FED260ADFED267A68EE808A67
:105BA000CDF81F1028EE008ACDF81B0029EE000A60
:105BB00068EEA78A28EE278A20EE270AFDEEE88AFB
:105BC000BDEEC88A18EE903AADF8233018EE103AC0
:105BD000ADF825301BF0C6FBBCEEC00ACDF8358011
:105BE000CDF83970CDF83D6010EE103ACDF8414057
:105BF000ADF82730019BCDF82930049BCDF82D302E
:105C0000059BCDF831304AF0BFFA2D2206A949F0A4
:105C1000FDFB12B0BDEC048BBDE8F08101AA0021B0
:105C2000284605F081FE0028A2D0A3E75241C07F9C
:105C3000E02E65420000C84230B52DED028B8BB0DE
:105C4000044624220D4601A80021C5F093FBA3239E
:105C50009FED228A8DF8043095238DF80530482376
:105C60008DF8063078F04AFAD4ED847A2B6867EE26
:105C7000887A95ED020ACDF80F30CDF80B1017EEAB
:105C8000903AD4ED857ACDF8070067EE887ACDF8A2
:105C900013306B68CDF8173017EE903ACDF81B3003
:105CA0001BF02CFB10EE103A94ED860A20EE080A49
:105CB000CDF81F301BF022FB10EE103ACDF8233048
:105CC00094F824338DF827304AF05EFA242201A993
:105CD00049F09CFB0BB0BDEC028B30BDE02E654261
:105CE00030B5104689B00D461446FFF707FF28BBB4
:105CF000002301931822002102A8C5F03BFBA32337
:105D00008DF8083095238DF8093049238DF80A3035
:105D100078F0F4F9A368CDF80F100593E368CDF897
:105D20000B000693019B8DF8135007934AF02CFA51
:105D3000182202A949F06AFB09B030BD01AA00216E
:105D4000204605F053FD0028D2D0D3E710B590B01F
:105D5000044604A805F0FAFC04A9204601F00CFC56
:105D6000002846D001F0D6FE01A901F0DBF902A916
:105D7000204600F0FBFC00283DD0DDED027AF1EE7C
:105D8000677A03AA002104A8CDED027A05F0CCFDC4
:105D900008B91A4B03931F22002108A8C5F0EAFA9C
:105DA000A3238DF8203095238DF821304A238DF8D8
:105DB000223078F0A3F9069BDDED017ACDF82B3087
:105DC000079BF1EE677ACDF82710CDF82F30039BB3
:105DD000CDF82300CDF8333017EE903ACDF83730B8
:105DE000029BCDF83B304AF0CFF91F2208A949F0B9
:105DF0000DFB10B010BDDFED027AC2E75241C07F4B
:105E00005241C07F0023036043608360C36003612D
:105E100043618361C361036270470000B02290F860
:105E2000F43202FB030390F8892393F8D13012B1C6
:105E3000012B28BF01231846704700002DE9F04FC1
:105E400004464FF0000A8BB00D4623F0D1FE04F556
:105E5000097084F820A24FF07E5777F09DFA4FF436
:105E60007A7304F5217084F88052A4F87A32002500
:105E7000C4F8607204F53179C4F8647204F53A76B6
:105E8000C4F8687204F54E7B05F060FC03234846B5
:105E9000C4F8AC52C4F8983204F27C48C4F8B0524A
:105EA000C4F8B452C4F8B852C4F8BC52C4F8C052D2
:105EB000FFF7A8FF3046FFF7A5FF5846C4F82C535C
:105EC000C4F83053C4F83453FFF79CFF04F57B70DB
:105ED000C4F85C53C4F86053C4F86453C4F86853FE
:105EE000C4F86C53C4F87053C4F87453C4F87853AE
:105EF000C4F87C53C4F88053C4F88453C4F888535E
:105F0000C4F8A453C4F8A853C4F8AC53C4F8C0539D
:105F1000C4F8BC53C4F8B853C4F8C853C4F8CC533D
:105F2000C4F8D053C4F8E453C4F8E053C4F8DC53C5
:105F3000C4F8B473C4F8D87305F008FC04F58060A5
:105F400005F004FC04F2144304F586601D605D60F6
:105F500004F584631D605D609D6005F0F7FB04F24D
:105F60004443404604F254421D605D609D606C4BAA
:105F7000C4F8543404F51073C4F8583404F511739C
:105F8000C4F85C3404F51273C4F8603404F5137378
:105F9000C4F8643404F25123C4F8683404F514736B
:105FA000C4F86C3404F58E631D605D609D60FFF77E
:105FB00029FF04F59460FFF725FF04F59A6304F2C6
:105FC000BC501D605D609D6004F2DC431D605D603F
:105FD0009D6004F59D631D605D609D6004F2F44367
:105FE0001D605D609D6004F204531D605D609D60F6
:105FF00004F214531D605D609D6004F5A763C2F850
:10600000D470C2F8D8701D605D609D6004F2445386
:106010001D605D609D6004F5AC631F605D6004F20F
:1060200084531D605D609D6004F5B2631D605D601A
:106030009D6004F5B5631D605D609D6005F086FBA5
:1060400004F2CC53242251461D6040465D6004F2A8
:10605000D4531D605D6004F2DC531D605D60C5F0CB
:1060600089F904F5C060C8F82070C8F81070C8F845
:106070000070FFF7C7FE04F2246304F27C601F6027
:106080009D605D60DD6004F234631D605D609D6055
:1060900004F5C8631D605D609D6004F24C631D6083
:1060A0005D609D6004F5CB631D605D609D6004F2E2
:1060B00064631D605D609D60354605F047FB194BCC
:1060C000204619491C6044F025FD514624225846BB
:1060D0006E46C5F04FF904F52B7204F52E73C4F823
:1060E0005873C4F84873C4F8387307CA83E80700C4
:1060F000484694EDB01AD4EDAF0A94EDAE0A1BF009
:1061000049FE494668461BF06DFD0FCE0FC50FCE08
:106110000FC5204633682B600BB0BDE8F08F00BF81
:10612000F84C0F0880820030944B0F0810B50446DD
:1061300088B001F05BFD94F93E32012B02D1274873
:1061400005F0DAFA022B0AD1032304A904F11100A5
:1061500084F83E3201238DF8103045F0E1FC94F8CC
:106160003E3204F2544084F8A83201F0FBFC94F96A
:106170003D32642B30D1652304A904F23D208DF813
:10618000103045F00BFD04A9204643F0AFFD18B3D5
:1061900004238DF818300023CDE9013303930F2336
:1061A0000593694604A843F021FF059B28B108AA7E
:1061B000009902EB830242F8581C0133112B05931E
:1061C000EFD975F055FA9DED031ADDED020A652150
:1061D0009DED010A75F00AFA08B010BD284A0F08B3
:1061E00070B500F52B7600F52E758CB0044631465F
:1061F00028461FF00DF8E0B996E8070085E807008B
:1062000004F5317194EDB01AD4EDAF0A02AD94EDFE
:10621000AE0A084601911BF0BDFD019902A81BF0D2
:10622000E1FC04F53A740FCD0FC40FCD0FC42B68F9
:1062300023600CB070BD000084B000F54E7004B057
:106240001BF0E4BB84B000F54E7004B01BF00CBC36
:1062500013B5044600F5097140F2751201A817F054
:106260007BFA04F2544001F071FE204623F0FAFE5E
:1062700001A817F093FA02B010BD0000F8B54B6802
:1062800001F1100607460C46C0F8103200F54E75B5
:106290008B68C0F81432CB68C0F818320FCE0FC527
:1062A0000FCE0FC504F1440233682B6007F54B7322
:1062B00007CA83E8070004F1500207F5577307CABD
:1062C00083E8070004F15C0207F55A73683407CAD3
:1062D00083E8070007F55D7394E8070083E807008B
:1062E000384601F097FD3846BDE8F84001F07ABD28
:1062F00013B5044600F25440019003F071FA04F51E
:10630000BE610198009102F059FE0099204602B04A
:10631000BDE81040FFF7B2BF4A78064BC2F3401207
:106320001A754A78C2F380125A750A78C2F30012BD
:106330009A7570470D83003013B5044600F5097156
:1063400040F24D3201A817F007FA002104F2544040
:1063500002F02AF894F8783223B1204624F028FD80
:1063600084F8780201A817F019FA02B010BD0000F5
:1063700038B590F8243305460C462BB1032B0BD0CF
:1063800095F88032DB070CD405F27C630FCB84E8F0
:106390000F0095F88C0603E023F0E6FE0028EFD00E
:1063A00038BD0020FCE7000000F2544090ED350AB3
:1063B0007047000000F2544090ED360A704700002C
:1063C00010B490F824230C462AB1032A0AD00020E6
:1063D0005DF8044B704700F5B56007C884E8070016
:1063E0000120F5E75DF8044B23F07ABE90F89C039A
:1063F000431E58425841704738B590F824330D4633
:106400008BB900F2544001F009FE044610B9002493
:10641000204638BD01F056FDD5ED007A27EE800A02
:1064200085ED000AF4E7D0EDE67AC1ED007A90F848
:106430009443002CEBD090EDE47ADFED076AB4EEE4
:10644000E67AF7EE006AF1EE10FA27FE267A67EE9A
:10645000877AC1ED007ADBE70000003490F824333E
:10646000032B01D123F0B8BD0020704790F82423FE
:10647000032A01D123F082BF00F2544002F0E6B9B2
:1064800030B5054685B00C469AB1032A1BD005F5F8
:106490002B701EF0F7FE01A920468DED010ACDED0F
:1064A000020A8DED031A1DF095FF0123184605B071
:1064B00030BD90F8F035002BF8D000F224630FCBFC
:1064C00084E80F00E3E790F87832002BEED023F059
:1064D0001FFFDCE790F82423FFF7D2BF7FB590F8C9
:1064E000242332B1032A4FF0000309D0039304930D
:1064F0000CE000F2544007B05DF804EB01F0D8BDA9
:1065000003A903930493059323F05CFD9DED030A17
:10651000DDED040A07B05DF804FB000037B5044662
:106520000D4640F2C75200F5097101A817F014F9A1
:106530002046294623F042FE94F82433032B0CBF57
:106540000446002401A817F029F9204603B030BD05
:1065500010B52DED028BB0F8903682B004461B07C3
:1065600030D5D0F8383401A99FED188A00F51570A0
:1065700007EE903AB8EEE77A27EE087A8DED017AC9
:1065800045F0BAFAD4F83C3401A904F5167007EEC8
:10659000903AF8EEE77A67EE887ACDED017A45F029
:1065A000ABFAD4F8343401A99FED097A04F51770D9
:1065B00007EE903AF8EEE77A67EE877ACDED017A4A
:1065C00045F09AFA02B0BDEC028B10BD95BFD633F0
:1065D0000AD7233C23F026BE90F82403003818BFC6
:1065E0000120704738B590F824230C46032A04D1C3
:1065F000012523F0E7FC284638BD90F87056002DA1
:10660000F9D000F2646393E8070084E80700F2E73A
:1066100010B590F8242303460C461AB1032A0BD078
:10662000002010BD90F878060028FAD003F5BE636C
:10663000D3F884300B60F4E723F0DAFC012084ED1A
:10664000000AEEE790F82433032B01D123F020BE9B
:106650000020704730B590F8243387B005460C46CB
:1066600023B1032B09D0002007B030BD00F2544005
:1066700007B0BDE8304002F095BB0022002302A91C
:10668000CDE90223CDE9042323F084FC0028EAD0DD
:106690006946284623F08AFC0028E4D0DDE902237D
:1066A000C4E90023DDE90423C4E90223DDE9002372
:1066B000C4E90423D8E7000010B586B00022002307
:1066C0000C466946CDE90023CDE90223CDE9042338
:1066D000FFF7C0FF88B19DED027B9DED005BF7EEFB
:1066E000C76BB7EEC55B9DED047B84ED005AC4ED2E
:1066F000016AB7EEC77B84ED027A06B010BD0000D8
:1067000090F824231AB1032A05D00020704700F224
:10671000544002F083BB23F03DBC00001FB50022B3
:1067200000230C466946CDE90023CDE90223FFF79B
:10673000E7FF58B19DED027B9DED006BB7EEC77B87
:10674000B7EEC66B84ED017A84ED006A04B010BD2B
:1067500090F824231AB1032A05D00020704700F2D4
:10676000544002F045BB23F021BC000013B50C4699
:106770006946FFF7EDFF28B19DED007BB7EEC77BC3
:1067800084ED007A02B010BD90F93E323BB990F82A
:10679000803213F0010F14BF032000207047032044
:1067A00070470000F7B50446FFF7EEFF05460028E6
:1067B00062D0032839D194F878326BB394F88032E0
:1067C000D8072BD501A9204623F0E0FEBDF8043000
:1067D000002B18BF002594F8206206F0FD06012E5C
:1067E0004AD10023032D019307D101A9204623F0AC
:1067F000D9FE204623F0F2FD064604F2544002F092
:1068000023FC08B994F821039DF80430D90703D577
:106810005A0701D59F0632D400252DE0204623F0EB
:106820001BFB002808BF0025D5E70025D3E713F0A0
:10683000020F2EE094F9503223B99DF80430DB09A1
:106840002FD0E9E7002EF8D00FF0A2F8FFF7E6FA14
:10685000022807D99DF805309806DDD59DF804304B
:10686000D906D9D5FB6A93F89C30002BE5D118E006
:10687000DA0601D41B0718D5284603B0F0BD00285E
:10688000FAD094F82123B4F99036002ACFD013F02F
:10689000010FF1D1154B1F68FB6A93F89C30002B58
:1068A000C8D19DF804309C07E2D406F07DF906F0CB
:1068B00079F80028B0D10FF06BF8FFF7AFFA022893
:1068C000AAD90FF065F8B02290F8F432F0EE007A11
:1068D00002FB030090ED3B7AB4EEE77AF1EE10FA9A
:1068E0009AD59DF80530DB09C6D195E76082003066
:1068F0002DE9F04790F8783292B00446002B00F072
:106900009380204623F0C4FF2046FFF74BFF032867
:106910007AD104F54E78002720464FF00C0A414604
:1069200000970197029723F0C9FC6946204623F09F
:10693000BBFC009B2046C4F81032019BC4F8143203
:10694000029BC4F8183201F065FA204601F04AFAB9
:106950001AF010F80546204623F00EFB002803AA83
:106960004FF0FF31AEBFC6B295F80A9495F80B64AC
:106970002046A8BFB14603970497059723F046FB2E
:1069800003A804F55D771EF07DFC0AFB09500AFBA5
:10699000065504F5577184EDD70A00F55170C4ED22
:1069A000D80A05F5077584EDD91A06AE1EF07AFCF3
:1069B0003A4684EDCB0A4FF0FF31C4EDCC0A2046B5
:1069C00084EDCD1A23F036FB95E8070086E8070032
:1069D000394630461EF0CCFC04F53172414609A818
:1069E0001BF092F8314609A81BF010F809A92046BF
:1069F00084EDDA0AC4EDDB0A84EDDC1A23F0D2FD63
:106A000009A92046FFF788FC94F89236002B3AD16A
:106A100009A804F09BFE09A9204623F0B1FB90B31E
:106A2000012384F892362EE0D0F87C321BB977F03F
:106A30005DFBC4F87C02154B1B68D86A03685B6871
:106A4000984788B177F052FBD4F87C32C01AB4F87A
:106A50007A32984204D9204624F0AAF984F87802C0
:106A600094F878327BB14CE777F040FBD4F87C3275
:106A7000C01A41F287339842E4D849F085FB49F0C7
:106A800069FB0028DED112B0BDE8F08760820030DB
:106A900090F8243323B1032B4FF0000007D0704748
:106AA00090F93E22032A04D10A7001207047087031
:106AB000FBE718467047000073B50D460DF107015E
:106AC0000446FFF7E5FF064628B19DF807302BB1D5
:106AD000032B09D00026304602B070BD04F27C635F
:106AE0000FCB85E80F00F6E72946204623F03CFB54
:106AF00094F87862EFE7000037B50D460DF1070115
:106B00000446FFF7C5FF28B19DF807202946204617
:106B1000FFF7B6FC03B030BD37B50D460DF10701E8
:106B20000446FFF7B5FF28B19DF8073023B1032BCA
:106B300011D0002003B030BD04F2F4531B682B6069
:106B400004F5BF631B686B6004F2FC531B68AB6009
:106B500094F8F005EEE72046294623F0A5FB94F8CB
:106B60007802E7E710B50446FFF70EFE18B10328D8
:106B700007D0002010BD04F25440BDE8104001F0E1
:106B800021BA94F87832002BF3D0204623F064F930
:106B90000028EED094F8203203F0FD03012BE9D158
:106BA00094F82403C31E58425841E3E710B5044645
:106BB000FFF7EAFD80B1032810D194F8780250B1B4
:106BC00077F094FAD4F87C32C01A44F620639842E5
:106BD00094BF0020012010BD0120FCE70020FAE74F
:106BE00008B50246FFF7D0FD032804D1104623F074
:106BF000D9FC012008BD0020FCE7000013B50C46BD
:106C000001A9FFF7EDFF20B1019B1C4214BF012039
:106C1000002002B010BD000030B585B004460191DF
:106C200002F0F2FE0199054610B9002005B030BD12
:106C3000019102F0B9FE01990028F6D0284602F031
:106C4000B7FE0028F1D0B4F890365907EED494F886
:106C50002133002BEAD00B4A1268D26A92F89C507A
:106C60006DB103A92046FFF7BBFF30B19DF80E3090
:106C70009A07DBD5C3F38000D8E72846D6E7184645
:106C8000D4E700BF6082003010B4BDF80440019426
:106C90005DF8044B23F01ABC10B4BDF80440019415
:106CA0005DF8044B23F0AEBB23F0E6BB90F8402424
:106CB0005AB100F234439FED057AD3ED007AF8EE35
:106CC000E77AA7EEC70A23F03BBC70470AD7233CFC
:106CD00010B50446FFF758FD032804D12046BDE84F
:106CE000104023F015BA002010BD00002DE9F0413E
:106CF00090F824338CB000270646032B0C4615462B
:106D000000970197029719D123F036F96A46804619
:106D10004FF0FF31304623F08DF9B8F1FF3FA76007
:106D2000676027600DD119F025FE2B46224690F8AA
:106D30000B1418F061FD0CB0BDE8F0814FF0FF3886
:106D4000EBE719F017FE2B4622465FFA88F118F0A0
:106D500053FD95ED000A68461EF0D0FA03A92046BF
:106D60008DED051A8DED030ACDED040A1EF000FB32
:106D700006F5317206F54E7103A81AF0C5FE2146DC
:106D800003A81AF043FEDFED077A84ED021A84EDC2
:106D9000000AC4ED010A95ED007AA7EE271A84EDEA
:106DA000021AC8E70AE81C41DFED0B7A20EE270A39
:106DB0001FB50C461946094BBDEEC00A1868084BB2
:106DC0008DED020ACDE900429DF81820C06A16F048
:106DD000B9FE04B010BD00BFE02E654260820030F5
:106DE0003C4A0F082DE9F0472DED028B92B00025AB
:106DF0004FF07E5A04460F4600F54E7106A89046A5
:106E0000CDF818A00995089507951CF0A3FD05F08D
:106E1000CBFE05F0C7FD81462046FFF7B5FC0328F1
:106E200003D094F82433032B4FD100269FED548ACE
:106E3000DFED548A2379F2B2934247D90AAA71B29C
:106E40002046CDF828A00D950C950B9523F040FA1F
:106E50000AA906A81DF0EEFAB4EEC80AF1EE10FA7F
:106E60000DDD3B46484ACDF8008048492046FFF7F3
:106E70009BFF002012B0BDEC028BBDE8F0870AA991
:106E800006A80395049505951DF0BEFA03A90EA862
:106E90008DED0E0ACDED0F0A8DED101ACDED111A04
:106EA0001DF026F8B9F1000F0DD09DED050AB0EEEA
:106EB000C00AB4EEE80AF1EE10FA04DD3B46344AAB
:106EC000CDF80080D1E70136B4E7002394F8806262
:106ED00016F0010001D0012BCCD104F5C0610AA845
:106EE000CDF828A00D950C950B951CF033FD0AA943
:106EF00006A81DF09FFADFED227AB4EEE70AF1EE64
:106F000010FA05DD3B46204ACDF800802149ADE767
:106F10002046FFF739FC03282DD1204623F03AFA0A
:106F200094F88032DB0728D438BB0AA906A8039559
:106F3000049505951DF068FA03A90EA88DED0E0ABB
:106F4000CDED0F0A8DED101ACDED111A1CF0D0FF0A
:106F5000B9F1000F11D09DED050ADFED0A7AB0EE10
:106F6000C00AB4EEE70AF1EE10FA06DD3B46084A25
:106F7000CDF80080CAE70020D2E701207AE700BF01
:106F8000C2B8323EC2B8B23E684A0F08734A0F0810
:106F90000FFD0E08784A0F082DE9F7431546044601
:106FA00088460193FFF7DEFD019A074638B9284865
:106FB0002946284B0068C06A16F0C4FD019A29468C
:106FC00020460192FFF70EFF064668B32046FFF702
:106FD000DBFB94F93E1243B2019A994207D01E4B53
:106FE0001B4829460068C06A16F0ACFD1CE094F806
:106FF0002433834207D0019205F0D6FD05F0D2FC80
:10700000019A0028EBD12046FFF7BEFB18B10328F8
:107010000FD0124BE4E7134641462A4604F254408F
:1070200000F0E4FF00B107B90026304603B0BDE828
:10703000F08394F87892B9F1000F01D1084BCFE7B3
:10704000134641462A46204622F016FFEAE700BFD3
:10705000608200307C4A0F08884A0F08B84A0F083F
:10706000A74A0F0890F82433032B01D123F0B0BABC
:107070000020704713B5044600F5097140F67832D8
:1070800001A816F069FB204623F006F801A816F0C7
:1070900085FB02B010BD000008B50246FFF774FB87
:1070A00010B1032806D008BD02F25440BDE80840E4
:1070B00000F05CBF1046BDE8084023F07FBA000036
:1070C0000B46114610B42BB1032B09D000205DF8FC
:1070D000044B704700F254405DF8044B00F052BF7F
:1070E0005DF8044B23F04CB813B504460A46FFF78D
:1070F0004BFB014620460192FFF7E2FF70B9084BB7
:10710000019A1B68DB6A93F89C0038B194F8241349
:10711000204602B0BDE81040FFF7D2BF02B010BD5C
:107120006082003070B590F8943286B004460D4607
:10713000DB070CD403F04EFB5022437C02FB030020
:10714000D0ED0B7AF1EE677AC5ED007A41E002A846
:1071500004F0FCFA69462046FFF7FAFAE8B90EF0A7
:1071600017FC94F950320646022BE3D1FEF756FE87
:107170000228DFD9B02396F8F4029FED177A03FBBB
:107180000066D4F88832D6F8E0209B1A07EE903AD1
:10719000F8EEE77A67EE877AD6E702A92046FFF78E
:1071A000A3FF0028DBD0D4F88822039BDFED0A7A06
:1071B0009B1A07EE103AB8EEC77A9DED006B27EEEA
:1071C000277AB7EEC77A36EE477BB7EEC77B85EDF9
:1071D000007A06B070BD00BF0AD7233CF0B587B077
:1071E0000C46064600F5097140F6DD3201A816F09E
:1071F000B3FAA36853B9E36843B9636833B90027A6
:1072000001A816F0CBFA384607B0F0BD204604F0CE
:10721000BFFB0028F3D002AD94E80F0085E80F0013
:107220000021284604F070FB07460028E7D096F8B6
:107230009432DB0704D448F0A7FF192148F0E0FEA0
:1072400006F5217C95E80F008CE80F0096F8943243
:10725000304643F0010386F8943200F013FE54F0F8
:1072600069FB462155F0B6FF54F064FB452155F00B
:10727000B1FF084BA2681B68DB6A1A61E2685A61B9
:1072800062689A6121F054FB0028B9D01EF078FFA3
:10729000B6E700BF6082003038B5144B04461B6867
:1072A000DD6A2B6828465B689847F0B12B690BB9FB
:1072B0006A69D2B1C4F88C3200226B6904F521707E
:1072C000C4F89032A96904F045FA94F8943223F096
:1072D000030343F0030384F8943254F02BFB044A75
:1072E0000621BDE838404EF023BC38BD6082003036
:1072F000CC4A0F0813B504460193FFF745FA03285B
:10730000019B05D1204602B0BDE8104023F00AB829
:10731000002002B010BD000010B588B004460593EF
:10732000FFF732FA0328059B4FF000000AD10690C0
:10733000079006A802900B9801900A9800902046AA
:1073400022F0FEFF08B010BD13B504460193FFF70D
:107350001BFA0328019B05D1204602B0BDE810406E
:1073600022F0FCBF002002B010BD000038B504467A
:1073700002F04AFB0546D0B194F82433032B03D026
:1073800095F84E41204638BD204622F0B5FEFF2834
:107390000446F5D00146284602F00AFB0028EFD04B
:1073A0002146284602F000FB0028E9D0EAE704461F
:1073B000E8E7000008B590F82433032B05D019F056
:1073C000D9FA90F90A04C0B208BD22F0D5FD431CD9
:1073D000F9D1F4E708B590F8243383B1032B03D136
:1073E000BDE8084022F0C0BD47F0F6F840F64C5228
:1073F0004FF4801147F0A8F84FF0FF3008BD184651
:10740000FCE70000FFF7D6BF90F82433032B01D12F
:1074100023F0A8BB7047000090F82433032B01D160
:1074200022F09ABC7047000022F0FEBC22F016BE8B
:1074300010B5044626F09AF82046FEF76BFB20466E
:10744000BDE81040FEF782BC90F824330BB1032B4B
:1074500001D122F0ABBF00207047000090F8242338
:107460001AB1032A07D00120704790F95002003862
:1074700018BF0120704722F0A5BF000010B590F89A
:1074800040348AB00446002B62D1B0F89036DB0657
:107490005ED590ED957ADFED2F7AB0EEC77AB4EE37
:1074A000E77AF1EE10FA11D590ED967AB0EEC77A40
:1074B000B4EEE77AF1EE10FA08D590ED977AB0EED7
:1074C000C77AB4EEE77AF1EE10FA41D42046FFF71E
:1074D000C5FF00283CD1D4ED976ADFED1F7A9FED00
:1074E0001F6A66EEA76A94ED967AD4ED957A27EE38
:1074F000067A009067EE867A06A8FDEEE66ABDEE93
:10750000C77AFDEEE77A16EE903A17EE102A17EEDC
:10751000901A04F039F906A92046FEF7FFFFB8B12A
:1075200054F008FA94ED977A0D4A0621B7EEC77A1F
:107530008DED047B94ED967AB7EEC77A8DED027BE4
:1075400094ED957AB7EEC77A8DED007B4EF0F0FAA8
:107550000AB010BD000000340000C8428096184BED
:10756000E44A0F0890F824330BB1032B01D123F028
:1075700061BB00207047000000F57B7330B5044606
:107580000D460FCB85E80F0094F8FC0330BD0000DA
:107590007FB5064668460D4604F0D8F896F8943252
:1075A000DB0703D40024204604B070BD6946304692
:1075B000FFF7E2FF04460028F4D0694606F5217083
:1075C00004F0D2FA85ED000AC5ED010A85ED021A34
:1075D000E9E7000000F56072034610B50C4607CAE3
:1075E00084E8070093F88C0310BD000000B52DED72
:1075F000028B85B0B0EE408A9FED120A01A98DED95
:10760000010A8DED020A8DED030AFFF7E3FFA0B139
:10761000DDED010A9DED020AF1EE600AB1EE400ACD
:10762000C1F002F8DFED087AA8EE670A05B0BDECFC
:10763000028B5DF804EBC0F01FB805B0BDEC028B07
:107640005DF804FB0000000035FA8E3C10B52DED0E
:10765000028B90ED800A0446FFF7C8FFB0EE408A27
:1076600004F560701DF0CAFC20EE080ABDEC028B28
:1076700010BD0000D0F898330B6090F89403704769
:10768000D0F8A0330B6090F89D03704700F5697245
:10769000034610B50C4607CA84E8070093F8B00308
:1076A00010BD000000F56D7330B504460D460FCBDC
:1076B00085E80F0094F8C40330BD000000F5866330
:1076C00030B504460D460FCB85E80F0094F8400412
:1076D00030BD000000F24442034610B50C4607CA14
:1076E00084E8070093F8500410BD00002DE9F04332
:1076F00005460E4617462DED028B8BB0FFF736FE82
:10770000014680462846FFF787FA0446002846D0FF
:1077100002F07AF9414602F04DF986ED000A95F93A
:107720003C32002B38DD0EF033F9FEF777FB0128F1
:1077300032D90EF02DF9B02290F8F432B7EE008A6B
:10774000D5EDE47ADFED598A02FB030095F93C326E
:10775000F4EEE87AD0ED3B0A07EE103A96ED000A17
:1077600040F20E40F1EE10FAB8EEC77A67FE887A62
:1077700020EE270A37EE201A70EEC70A19F062FED3
:10778000D5EDE47AF4EEE87AF1EE10FA67FE887A45
:1077900080EE277A86ED007A01233B7003E095F8AE
:1077A000203333B9387020460BB0BDEC028BBDE8F6
:1077B000F0834FF0000995F82433CDF80490CDF80C
:1077C0000890CDF80C9043B1032B10D0CDF8109059
:1077D000CDF81490CDF818907CB90223324641467A
:1077E00005F254403B7001F073FB0446DBE701A94E
:1077F000284622F075FC0446E8E795F82433002B70
:10780000EBD004A92846FFF765FF04460028E4D022
:1078100001A904A81DF05CFD07A8CDED080A8DEDB7
:10782000091A8DED070A1EF087F904A8B0EE408A08
:107830001EF082F995F93C32002B2EDD07EE903ACE
:1078400040F25440F8EEE77A70EE670A37EE801A9D
:10785000B0EE480AF5EEC00AF1EE10FA48BFDFEDCF
:10786000140AF4EE410AF1EE10FA30FE811A19F012
:10787000E9FDB0EE408AD5EDE47A03239FED0B7A63
:10788000F4EEC77AB7EE007AF1EE10FA67FE877A67
:1078900088EE277A86ED007A7FE7B5EEC08AF1EEB2
:1078A00010FA48BF9FED028AE5E700BF00000034F0
:1078B0000000000038B50446FFF77CFD054694F84B
:1078C0002633834204D019F055F8294617F05CFEA0
:1078D0002046FFF76FFD84F8265384F825032046E1
:1078E000FFF768FD84F827032046FFF773FD04F5D2
:1078F000607184F828032046FEF762FD84F88C034B
:1079000000F0E0FA04F5677284EDE40A04F56671AC
:107910002046FFF7EBFE04F5687184F894032046D7
:10792000FEF76AFD04F5697184F89D032046FEF7B1
:1079300095FD04F56D7184F8B0032046FEF7CAFD8D
:1079400004F5727184F8C4032046FFF7E5F804F5E6
:10795000767184F8D4032046FFF7CEF804F57B71E6
:1079600084F8E8032046FEF703FD04F5806184F8FF
:10797000FC032046FFF7A0F884F810042046FEF729
:10798000ADFD04F2144004F5836380ED000AC3EDFD
:10799000000A1DF033FB04F21C4304F58461204609
:1079A00004F22C4283ED000AFFF7A0F904F586618A
:1079B0002046FFF799FB80B194F840349BB901232E
:1079C000204684F8403400F05DFA53F0B3FF4521BF
:1079D00055F000FC2046FEF7BBFD94F8403413B987
:1079E0002046FFF74BFD04F244412046FEF7FAFD26
:1079F00084F8500438BD000037B50D46044600F049
:107A0000F5F81DB918F0B6FF18F00CF84FF4EA724B
:107A100004F5097101A815F09FFE94F881322BB985
:107A20002046FFF739FC012384F88132224B1D6880
:107A3000A86A03689B6998472046FEF7D1FB204659
:107A4000FEF756FC204600F059FA2046FEF750FF9C
:107A5000286B30B10368D4EDD80ADB6894EDD70AFF
:107A60009847D4F81C0208B18EF01CFF204600F0A5
:107A700079F82046FEF796FE94F8A83284F824039D
:107A800083420ED084F8A80298B10C4D0C4B032809
:107A900008BF1D4653F04EFF2B460A4A06214EF002
:107AA00047F82046FFF706FF01A815F077FE03B060
:107AB00030BD054DEEE700BF60820030E8160F08CC
:107AC000734A0F08104B0F08784A0F08D0EDE47A7C
:107AD000B7EE000A9FED047AF4EEC77AF1EE10FAE1
:107AE00027FE800A704700BF00000034D0EDE47A22
:107AF000B7EE000A9FED067AF4EEC77AF1EE10FABF
:107B000067FE807A67EEA77A80EE270A704700BF8B
:107B100000000034014B1868704700BF80820030BD
:107B20007047000070470000704700000020704759
:107B3000002070470120704703681B6E1847000043
:107B400000207047002070470020704700207047D9
:107B500070470000002070470020704700207047E9
:107B6000704700007047000008B518F003FF90F858
:107B70000A0408BD30B59FED1B1A0C46DFED1A0A4A
:107B800005462D202DED028B87B091ED000A8DED7D
:107B9000011ACDED000A19F055FC9DED011AF0EE29
:107BA000408ADDED000A2E2094ED010A19F04AFC0E
:107BB0009DED011AB0EE408ADDED000A2F2094ED14
:107BC000020A19F03FFC03A905F52B70CDED038ADD
:107BD0008DED048A8DED050A44F0C4F807B0BDECC4
:107BE000028B30BDC2B8323EC2B832BE10B50446B8
:107BF00076F07CFAD4F80C331BB1C21AB2F57A7F56
:107C000012D30A4A1268D26A92F89C2002B15BB978
:107C1000C4F80C0394F83D4218F0ACFE80F805441B
:107C200004F0C2FF80F8294010BD00BF6082003020
:107C30002DE9F0432DED028B87B091ED007AD1ED67
:107C4000037A0C468DED047AB0EEC77A15461E46CF
:107C5000DDF84C90B5EEC07ACDED057ADDE9108700
:107C6000F1EE10FA06DCF0EEE77AF5EEC07AF1EE0E
:107C700010FA02DD04A81DF035FAB7EE001A6B20E9
:107C8000FFEE000A9DED050A19F0DCFBB7EE001AC5
:107C9000FFEE000A6C2089ED000AB7EE008A9DED28
:107CA000040A19F0CFFB04A888ED000A1DF08AF938
:107CB000002852D00023C9F8003088ED008AD4EDA6
:107CC000067A67EEA77AF4EEC87AF1EE10FA4ADB8C
:107CD0000023336085ED008AB7EE001A7C20DFEDCB
:107CE0003E0A96ED000A19F0ADFBB7EE001A86EDDC
:107CF000000AFFEE000A7D2095ED000A19F0A2FBB4
:107D000085ED000AD4ED067A129BF1EE677ADFED7D
:107D1000336AC3ED007A96ED007AF0EEC77AF4EE9E
:107D2000E67AF1EE10FA2BD503AB02AA01A92046A0
:107D30001AF090F89DED018AB0EE480ABFF09CFC65
:107D400085ED000AB0EE480AC0F09CFA87ED000A03
:107D500007B0BDEC028BBDE8F08304A81DF01EF94E
:107D60000028A7D1ABE738EE670A19F08FFA86ED45
:107D7000000A94ED087AC7EE007AC5ED007AABE709
:107D800094ED076AC6EE077AC7ED007A96ED007AA1
:107D9000B0EEC77AB4EEE67AF1EE10FAC4D495EDFF
:107DA000007ADFED0F6AB0EEC76AB4EE666AF1EEF4
:107DB00010FAB9DCB4EE477AF1EE10FAB4D6B0EEB0
:107DC000E77AB4EE667AF1EE10FAADDCF4EE677A9B
:107DD000F1EE10FABCD7A7E7000000000000003465
:107DE000FFFF7F7F1FB500F51D7300F5187200F5CA
:107DF0004E71039300F51C73029300F51B730193FE
:107E000000F51A73009300F51973FFF711FF05B021
:107E10005DF804FB9FED196AD0ED846ADFED187AF6
:107E200066EE866A90ED860A20EE060A26EEA77AAE
:107E3000C0ED7E6A10B5BDEEC77A044680ED817A4A
:107E400090ED857A27EE067A67EE275A80ED7F7AE5
:107E500060EE277AFDEEE55AFDEEE77AC0ED825A34
:107E600017EE903A002BBCBF03F50C43A033C0F8CB
:107E70000C3219F043FA84ED800A10BDE02E654201
:107E80000000C8421FB50E4B04461B68B3B16846DC
:107E900003F05CFC69462046FFF710FC20B16A46FF
:107EA00000212046FDF71CFF94F89432DB0705D52E
:107EB00004F5217201212046FDF712FF04B010BD28
:107EC0002486003008B502F085FCBDE8084001F0CA
:107ED000D7BE00007FB518F04DFD90F80B1407B029
:107EE0005DF804EB17F056BD10B5044680F810138A
:107EF00076F0FCF8C4F8140310BD000010B590F83B
:107F00001033044653B176F0F1F8D4F81433C01AA4
:107F1000B0F57A7F84BF002384F8103394F81833C7
:107F200053B176F0E3F8D4F81C33C01AB0F57A7F79
:107F300084BF002384F8183310BD000000F5AA7038
:107F40000B4607C883E80700012070470023C0F8EC
:107F50009C30C0F89830C0F89430C0F8A830C0F811
:107F6000A430C0F8A030C0F8AC30704770470000B3
:107F7000024B0B604FF07C53136070470000484287
:107F80007047000000F5B47010B50C460FC884E8C7
:107F90000F00204603F0CEFB30B1FFF7BBFD00F52C
:107FA00021700FC884E80F00204603F0C3FB80F067
:107FB0000100C0B210BD000010B5044604F02CF85A
:107FC000204610BD10B5D0F8603104465BB176F0A4
:107FD0008DF8D4F86031C01A41F28833984294BFCA
:107FE0000020012010BD0120FCE7000013B5009324
:107FF00003680192DB6D98470446DDE9002128B94A
:108000000448054B0068C06A15F09CFD204602B08C
:1080100010BD00BF608200307C4A0F0813B50446D3
:10802000019101F0F1FC019A23680146DB6B08B174
:1080300090F84E11204602B0BDE8104018470000ED
:1080400090ED007ADFED0F7AB0EEC77AB4EEE77A02
:10805000F1EE10FA14D590ED017AB0EEC77AB4EED5
:10806000E77AF1EE10FA0BD590ED027AB0EEC77A0E
:10807000B4EEE77AF1EE10FA4CBF01200020704711
:10808000002070470000003410B501F0BDFC04462C
:1080900058B190F84E1101F087FC30B194F84E11B0
:1080A0002046BDE8104001F083BC002010BD000058
:1080B0002DE9F043002504462DED028B8FB00368B7
:1080C00002A99B6B03950495059506950295984723
:1080D000064638B1FFF7F6FEDDED027A27EE800A9C
:1080E0008DED020A0DF054FCFDF798FE0746002EB8
:1080F00050D0DDED027A0BA9D4ED646A204694EDF0
:10810000657A236827EE877A0B9567EEA67A0C9539
:108110000D9509AD8DED097ACDED0A7A5B6B984727
:108120000BA928461CF0B2FE012F8DED030ACDED00
:10813000040A40F2B3800DF02BFCB02590F8F43225
:10814000DFED5A7A05FB030090ED3C8A28EE278A82
:10815000B0EE480ABFF090FAF0EE408AB0EE480A5E
:10816000C0F090F88DED0C0ACDED0B8A0DF010FCEF
:1081700090F8F43205FB030009AD90ED3B0A0BA823
:108180001CF0A4FE05A88DED050ACDED060A96BBF0
:1081900003C885E00128CED89DED020AB5EEC00ADD
:1081A000F1EE10FA7FDD07AED4F89421D4F89031C7
:1081B0003046079208931CF0B3FE23680BA90B9579
:1081C00020460C950D955B6B9847DDED077A9DED8C
:1081D0000B7A09AB77EE877A9DED0C7ACDED077AB5
:1081E000DDED087A77EE877ACDED087A96E8030020
:1081F00083E8030049E02369B7EE008A04F5BC79FF
:1082000004F5C47693ED000A03AF04F5C07838EEA8
:10821000408A1CF05BFE8DED090A4846CDED0A0A46
:10822000B0EE480A1CF052FE0BA92846CDED0C0A10
:108230008DED0B0A1CF02AFE3146C4ED5F0A38466C
:1082400084ED5E0A1CF032FE8DED090AB0EE480A9C
:108250004046CDED0A0A1CF039FE0BA928468DEDEB
:108260000B0ACDED0C0A1CF011FE84ED600AC4ED82
:10827000610A97E8030086E80300494640461CF07F
:1082800005FE8DED090ACDED0A0A9DED090ADDED29
:108290000A0A0FB0BDEC028BBDE8F083DDE90301F3
:1082A00085E80300F1E709950A95EEE735FA8E3C7B
:1082B00010B590F84613044604F09CF87C23C0B235
:1082C00003FB0044D4F8A40010BD0000044B026F6F
:1082D0001B68DB6A5A60426F9A60826FDA6070478F
:1082E00060820030F0B58FB0044618F043FB0023E5
:1082F00002AA90F80A1402930546039304F1940726
:10830000049301AB17F01AFAD8B39DED010AB5EE4C
:10831000C00AF1EE10FA34DD04F1B00602A81CF038
:10832000FDFF394684ED2C0A3046C4ED2D0A84ED5C
:108330002E1A1DF003F804F17C0130461CF0B2FF48
:1083400004F1880105A88DED050ACDED060A8DED35
:10835000071A1CF0A7FF08A88DED080A9DED010A79
:10836000CDED090A8DED0A1A1CF0C8FF0BA904F126
:1083700028008DED0B0ACDED0C0A8DED0D1A19F0CC
:108380008BFD95F80A040C23394603FB005000F5D9
:1083900051701CF087FF84ED2C0AC4ED2D0A84ED8A
:1083A0002E1A0FB0F0BD00007B4B2DE9F0470025E1
:1083B0001F6804460E462DED028BC0F89C508AB013
:1083C000C0F8985004F12809C0F89450C0F88450BF
:1083D000C0F88050C567C0F89050C0F88C50C0F805
:1083E0008850C0F8B850C0F8B450C0F8B050F86A1F
:1083F00003685B68984700284CD075F077FE42F21E
:108400000F73984246D8FB6A484693ED010A84ED03
:108410001C0AD3ED020AC4ED1D0A93ED031A84ED84
:108420001E1A19F0B7FC53F085FADFED5C7A94ED73
:108430001E6A062194ED1C7A26EE276A584A27EE1A
:10844000277AB7EEC66A8DED046B94ED1D6A26EEB1
:10845000276AB7EEC77AB7EEC66A8DED007B8DED61
:10846000026B4DF065FB94ED1E8AB0EE480ABFF03A
:1084700003F984ED650AB0EE480ABFF003FF84ED0E
:10848000640A75F033FEC4F864010AB0BDEC028BD7
:10849000BDE8F087A6B194ED1C0AB4EE400AF1EEF7
:1084A00010FA0DD6D4ED1D0AF4EE600AF1EE10FAC2
:1084B00006D694ED1E1AB4EE411AF1EE10FA67D703
:1084C00018F058FA4FF00C0A90F80B34B2EE028A0A
:1084D000F2EE068A07460AFB030307AE4FF01508C3
:1084E00003F5077393E8070086E8070030461DF0A0
:1084F00023FBB4EEC80AF1EE10FA11D508F1FF38EB
:1085000018F0FF0815D130461DF016FBF1EE047A85
:10851000B4EEE70AF1EE10FA1CDC2567656731E07E
:1085200030461DF009FBB4EEE80AF1EE10FAE5DC86
:10853000E9E7384617F02CF8384617F073FA97F841
:108540000B340AFB037303F5077393E8070086E80F
:108550000700CBE7DDED098A9DED088A68EEA80AE1
:108560009DED070AE8EE080AF1EEE00AC0F05CF8BB
:1085700084ED1D0AF1EE680AB1EE480AC0F054F825
:1085800084ED1C0A9FED071AD4ED1D0A94ED1C0A18
:10859000484619F0FFFB66E760820030E02E654236
:1085A000844C0F08000000000021FFF7FDBE000012
:1085B00037B504460846154601911DF0BDFAB7EEE1
:1085C000007AB4F8D0300198C7EE007A94ED337A8F
:1085D0000133A4F8D03037EE277A84ED337AB0EE49
:1085E000007AF4EEC77AF1EE10FA06D5B6EE007A0C
:1085F000F4EEC77AF1EE10FA0DDC9FED0E7AF4EE90
:10860000C77AF1EE10FA13D59FED0B7AF4EEC77A24
:10861000F1EE10FA0CDDB0EE670A1CF06FFE0120DF
:10862000C5ED010A85ED000A85ED021A03B030BDE3
:108630000020FBE700247449BD37863570B500F192
:10864000280600F134050446294630462DED028BFC
:10865000B6EE008A8AB01CF0CDFE284620EE088ACD
:10866000B0EE480A1CF04AFE07A93046CDED080AD4
:108670008DED091A8DED070A1CF02AFE8DED010A19
:10868000B0EE480A3046CDED020A8DED031A1CF01B
:1086900035FE07A928468DED070ACDED080A8DEDB8
:1086A000091A1CF015FE04A901A88DED040ACDEDF0
:1086B000050A8DED061A1CF0B1FE324601A92046CE
:1086C0008DED070ACDED080A8DED091AFFF770FF51
:1086D00058B975F00BFD0121C4F860012046FFF781
:1086E00063FE0AB0BDEC028B70BD2A4604A9204689
:1086F000FFF75EFF0028ECD004F1400207A92046F6
:10870000FFF756FF0028E4D0EBE7000030B50D4638
:1087100004462DED028B284683B091F8461303F0F2
:1087200069FEC1B27C2000FB015104F128009431A4
:1087300019F0C8F968468DED000ACDED010A1CF06C
:108740005DFCDFED1C7AB4EEE70AF1EE10FA05D518
:108750009FED190A03B0BDEC028B30BD68461CF0DA
:10876000C1FC68461CF02EFC0028F1D194ED428A31
:10877000284603F0A7FFF0EE400AB0EE480A18F0D2
:1087800017FD80B9284603F09DFFB0EE408A84EDC6
:10879000420ABEF071FF84ED430AB0EE480ABFF012
:1087A00071FD84ED440A04F5867168461CF0E2FB15
:1087B000D0E700BF00000034000000009FED0C7AFD
:1087C000B4EEC70AF1EE10FA0BD4DFED0A7AB4EE7C
:1087D000E70AF1EE10FA07DCC0EE077AB0EE670A9E
:1087E0007047F7EE007AF9E7F2EE047AF6E700BF99
:1087F000F3665F3F58A00B411C3008B51CF0FEFB30
:10880000F1EE007AB4EEE70AF1EE10FA97BFF1EE5E
:10881000027A9FED050A37EEC00ADFED047A98BFB1
:1088200020EE270A08BD00BFCDCCCC3DCDCC4C3EC0
:1088300008B5836993F9000038B10DF0A9F8FDF788
:10884000EDFA012894BF0020012008BDF8B52DEDF8
:10885000028B054604F0A8F904F0A4F80446B8B366
:10886000FFF758F990F8213393B32846FFF7E0FF5C
:10887000064668B30DF08CF8B02790F8F432F0EEAD
:10888000087A07FB030090ED3B7AB4EEE77AF1EE4D
:1088900010FA1DD495ED1E8A0DF07AF890F8F43296
:1088A000DFED1E7A07FB030090ED3C0A98EE270AE5
:1088B00018F03AFDB0EEC00ADFED197AB4EEE70A1F
:1088C000F1EE10FA08DC344675F010FCC5F85001E2
:1088D0002046BDEC028BF8BD05F5AA701DF02CF901
:1088E000B0EE408A0DF054F890F8F4329FED0D7A16
:1088F00007FB0303D3ED3B7A67EE877AB4EEE78A92
:10890000F1EE10FADFD575F0F1FBD5F85041001B00
:10891000B0F5FA6F8CBF00240124D9E7E02E654240
:1089200000003442CDCC4C3F0A4B1B6810B5DB6ACB
:10893000044693F89C305BB975F0D8FBD4F86431E9
:10894000C01A44F61F6398428CBF0020012010BD5E
:108950000020FCE760820030F8B52DED068B044660
:108960000DF016F8054604F01FF9064606F07EFAEB
:10897000002840F0AB802046FFF768FF002800F099
:10898000A8803046FFF794FCD4F8DC30984200F021
:108990001A813046FFF78CFCD4F8DC30DFED8F7A9B
:1089A000C31A304608EE903AF8EE688A68EEA78A55
:1089B000FFF77EFC94F8BC30C4F8DC00F3B9304615
:1089C00004F002F8D0B104F1280796F846233046A7
:1089D000394603F07BFED4ED1D0AB0EE401A38464E
:1089E00094ED1C0A19F0D6F90023C4F89030C4F8AD
:1089F0008C30C4F88830012384F8BC3020463146DE
:108A0000FFF784FE95F8F402B0EE408A05EB0015FE
:108A1000D5F8A030C4F8E03004F1B000D4ED129ADB
:108A20001DF08AF86368DFED6E7A68EE299A93ED9F
:108A3000007AB0EE40AAB4EEE77AF1EE10FA01D572
:108A4000C3ED007A2046B0EE4A0AFFF7B7FE63682E
:108A500020EE299A93ED000A29EE009AFFF7CCFE4A
:108A6000204629EE009A84ED249AFFF75DFF38B185
:108A7000B2EE007AD4ED247A67EE877AC4ED247AD8
:108A8000F0EE007AF4EEE78AF1EE10FA10D5DFEDA1
:108A9000557AB4EEE7AAF1EE10FA09D5DFED527A75
:108AA00069EEA79AD4ED2A7AE9EEA87AC4ED2A7A7B
:108AB000B0EEC88A9FED4D0A94ED367ADFED4C7A20
:108AC00028EE008AA7EE278A84ED368ABDEC068B55
:108AD000F8BDFFF71FF890F82133002B73D0204624
:108AE000FFF7A6FE00286ED095F8F42205EB0213DE
:108AF000D3F8A010D4F8E0308B4264D0B026F0EE6A
:108B0000087A06FB025292ED3B7AB4EEE77AF1EE78
:108B100010FA58DBCB1AC4F8E0109FED361A08EEB5
:108B2000903A95F8F43294ED1E0A06FB0353F8EEE2
:108B3000688ADFED317AD3ED3C9A68EEA78A69EE58
:108B4000819A39EEC00A18F051FCB0EE409ABFF09D
:108B500099FB94F8BC30B0EE408AF3B1F3EE047A9E
:108B6000F4EEE78AF1EE10FA17DC95F8F402F2EE73
:108B7000027A06FB005595ED3B7AB4EEE77AF1EE0A
:108B800010FAFFF649AFB0EEC99ADFED1C7AB4EEE9
:108B9000E79AF1EE10FAFFF63FAFB0EE691AD4EDA6
:108BA0001D0A94ED1C0A04F1280019F0F3F89FED5A
:108BB000148A012384ED248A84ED238A84ED228A99
:108BC00084F8BC3028E7BDEC068B04F188009FEDEB
:108BD0000D0ABDE8F8401CF0E5BB00BFBD37863587
:108BE000CDCC4C3DC2B8B23E0AD7233CCDCC4C3E96
:108BF000CDCC4C3F35FA8E3C6F12833A1904863F38
:108C000000000000EC51783F0C2303FB010130B55C
:108C100001F1C0038BB0144604AD93E8070085E86A
:108C2000070094E8070083E807002846FFF708FAE2
:108C300007AB58B194E8070083E807009DED070AE9
:108C4000DDED080A9DED091A0BB030BD95E807006F
:108C5000F2E7000010B52DED028BDFED0E8AB0EECD
:108C6000408A044660EEA88AB0EE680ABEF004FDB1
:108C700020EE480A84ED550AB0EE680ABFF002FB08
:108C800020EE480A0023BDEC028B84ED560AC4F89E
:108C90005C3110BD35FA8E3CF0B52DED028BD0F86D
:108CA0001831044685B00D468B60D0F81C31CB607E
:108CB00001F090FD06460CF06BFEA369074693F9A0
:108CC0000030022B53D1FDF7A9F802284FD997F8AD
:108CD000F432B02202FB0373D3F8E01000222846DE
:108CE00002F038FD94ED4A1A94ED490A2846B7EE91
:108CF000C11AB7EEC00A03F00BF994F82C3183B314
:108D00009FED258A75F0F2F901AA97F8F41206464C
:108D100038468DED018A0BF085FDD4F82001F0EE88
:108D2000480A9FED1E0AB6EE001A361A40F23C4081
:108D300007EE906AF8EE677A27EE800A18F082FB59
:108D4000DDED017A04F1F00030EE270A8DED010A25
:108D50001CF0BCF82846B7EEE01AB7EEC00A03F0E4
:108D6000D7F894F82C0105B0BDEC028BF0BD707CF7
:108D7000502303FB006696ED0B8AFEF7CBFED0ED89
:108D8000A27A9FED077AF8EEE77AE8EE077AFDEE31
:108D9000E77A17EE901AA1E7000000006F12833AFD
:108DA0000000C84230B589B004460D46684602F05E
:108DB000CDFC69462046FFF7E5F818B900242046A7
:108DC00009B030BD04A802F0C1FC204604A9FFF799
:108DD00063FF04460028F1D004A9684602F0FEFEB5
:108DE00085ED000B85ED021B85ED042BE7E7000008
:108DF00010B586B0002200230C466946CDE9002359
:108E0000CDE90223CDE90423FFF7CCFF18B1DDE95A
:108E10000423C4E9002306B010BD000070B586B07D
:108E2000002200230C466D462946CDE90023CDE9FA
:108E30000223CDE90423FFF7B5FF064618B195E8F4
:108E40000F0084E80F00304606B070BDF8B52DED78
:108E5000028B06460F46154600F0D6FD0446A0B12B
:108E6000394600F0A1FD80B12046394600F0A0FD52
:108E7000044650B100F0C8FD394600F09BFD85ED79
:108E8000000A2046BDEC028BF8BDFEF743FE90F8C9
:108E90002033B7EE008A7BB13046FFF7C9FC0446A9
:108EA00050B1D6ED538AFFF70DF8C8EE007A67EEA1
:108EB000A87AC5ED007AE4E7D6ED538AFFF702F809
:108EC000C8EE007A002467EEA87AC5ED007AD8E7EC
:108ED00070B52DED048B1646FFF7B8FF054670B34D
:108EE000FEF718FE90F93C424CB30CF051FDFCF734
:108EF00095FF012823D9E4B207EE904AB8EE678ABD
:108F00000CF046FDB02290F8F43296ED009A02FB88
:108F10000300D0ED3B8AFEF7D5FF40F2654029EE15
:108F2000000A38EE281A78EEC80A18F08BFAB0EE6C
:108F3000408AFEF7C7FFC8EE007AC6ED007A2846E1
:108F4000BDEC048B70BD000038B50D460CF020FD63
:108F50000446FCF763FF022885BF94F8F402B023AF
:108F6000002003FB004081BF00F5827007C885E840
:108F70000700012038BD000030B585B000230D4644
:108F800001A9019302930393FFF7DEFF044620B18A
:108F9000039B2B60204605B030BD01F01BFC417CDB
:108FA00001F0C4F804460028F4D001F013FC00F0EE
:108FB0001BFFB1EE400A85ED000AEBE7F8B5036F41
:108FC00000F14C070C4605464B6001F11006436F5B
:108FD0008B60836FCB600FCF0FC60FCF0FC63B6880
:108FE00005F1280104F1340033601AF0B3FC234684
:108FF000012203F8442B05F1B00207CA83E80700F9
:1090000005F1940204F1500307CA83E8070005F153
:109010001C0204F15C0307CA83E8070004F1740131
:109020002846FFF791FF04F1840184F88000284668
:10903000FFF7A2FF04F18C0184F888002846FFF7AF
:109040002BFE84F89C00F8BD08B503F0ADFDBDE82B
:10905000084003F0A7BC000010B504461CF0FAF964
:1090600050B904F10C001CF0F5F928B904F118000E
:10907000BDE810401CF0EEB9012010BD38B500F17C
:10908000280504462846FFF7E7FF28B120460121BE
:10909000BDE83840FFF788B9B7EE007AD4ED107A12
:1090A000F4EEC77AF1EE10FA06D5BFEE007AF4EED0
:1090B000C77AF1EE10FA12DC2046FFF7BFFA284615
:1090C000FFF7CAFF0028E1D1D4ED107AB2EE047A9E
:1090D000F0EEE77AF4EEC77AF1EE10FAD6DC38BD9E
:1090E00010B504461CF028FD2046BDE810401CF0D9
:1090F0006DB900002DE9F04F2DED048B9FEDCB8A6B
:1091000095B0F0EE408A04468DED028A8DED038A1B
:109110008DED048AFFF720FC17F02CFC0023054698
:1091200095F80D22012AA8BF012293423FD20021C7
:10913000284616F085F901230028F1D008AB0BAAC8
:10914000002128468DED0B8A8DED0C8A8DED0D8A60
:1091500016F052FB9DED080AB5EEC00AF1EE10FACA
:1091600023DD0BA81CF0DAF811A904F128008DED1D
:10917000110ACDED120A8DED131A18F047FC8DED92
:109180000E0AB0EE680A0EA8CDED0F0A8DED101A8A
:109190001CF0B4F811A904F1E4008DED110ACDED35
:1091A000120A8DED131A1CF0C9F80123B8E70C233D
:1091B00095F80B1404F1280B03FB0151584601F5F7
:1091C000077118F023FC84ED070A94ED3F0AC4ED03
:1091D000080A70EE288A84ED091AC4ED3F8A0CF063
:1091E000D7FB0646FEF796FC90F821332046019304
:1091F000FFF71EFB80B13046FCF710FE02280BD9AA
:1092000096F8F422B023616903FB026391F9001020
:1092100093F80201884263DA94ED3F7ADFED847AB5
:10922000B4EEE77AF1EE10FA62D4D4ED538AFEF789
:109230002BFF58B100F0E8FB90F84E1100F0BAFB9C
:10924000F0EE408AFEF73EFE60EE288A236CB0EE18
:10925000680A626B11A8A16A1393129211911CF013
:109260004DF804F5AA7102A88DED020ACDED030AAE
:109270008DED041A1CF062F874F038FF00230746E5
:1092800084F814312046FFF7D3FA002867D096F807
:10929000F422B02101FB0262D2F8E430C4F81831A4
:1092A00096F8F43201FB0363D3F8E830C4F81C31BC
:1092B00074F01CFF0123C4F8200184ED498A84ED79
:1092C0004A8A84F82C31D4F80031002B5AD102ABF1
:1092D000C4F80071F03493E8070084E8070007E061
:1092E00006EB0212D2F8A070D4F80021BA4204D1E1
:1092F00015B0BDEC048BBDE8F08F03F582730DF162
:10930000080C93E8070094F814318CE807001BB9A7
:1093100004F1F00383E807000123604604F5AA7115
:1093200084F814311BF0D4FF11A904F14C008DED29
:10933000110ACDED120A8DED131A18F095FBB5EE5A
:10934000C00A8DED110ACDED120A8DED131AF1EE62
:1093500010FAD8BF9FED350A84ED530A92E794EDD9
:109360003F7AD4ED497ADDED026AE6EE877ADDEDEB
:10937000036AC4ED497AD4ED4A7AE7EE267AC4ED61
:109380004A7AA0E7D4ED3F7A254BF5EEC07A8DED11
:10939000058A8DED068A0793F1EE10FAA8D9214BC4
:1093A0009FED217A1B6867EE877ADB6AB7EE007A59
:1093B00093F89CA0C7EE279ABAF1000F4AD094F810
:1093C000143113B9019B002B42D0E36804F1F00182
:1093D00002A8D3ED008A1BF07BFF8DED110A11A8C6
:1093E00069EEA88ACDED120A8DED131AB0EE680A67
:1093F0001BF084FF0EA905A8CDED0F0A8DED0E0A16
:109400008DED101A1BF09AFF05A8FFF769FE05A85D
:109410001CF03AF8F0B174F069FEC4F8600167E737
:10942000000080BF608200300AE81C41000000009C
:10943000CDCC4C3ECDCC4C3FCDCC4C3D920A06BF62
:10944000920A063FC2B8B23E728A0E3C5B8218395D
:10945000DDF804A000234FF0FF325FED0C8A04F129
:10946000E4080092CDE90833CDE90A33CDE90C33A5
:1094700095F80D22012A1046A8BF0120834253D23D
:109480000123002AFAD095F82D140029F6D0B0EE69
:10949000690A40460DF12C091BF084FFBAF1000F58
:1094A0003DD0424600212046FFF7AEFB8DED0B0A72
:1094B000CDED0C0A8DED0D1A4846FEF7C1FD60BBDF
:1094C0004846FFF70DFE48461BF0DEFF28BB05A906
:1094D00048461BF0A3FF05A94846CDED090A8DEDCE
:1094E0000A1A8DED080A1BF085FF08A8B0EE409A15
:1094F0001CF022FB009B2BB9F4EEC08AF1EE10FAAF
:1095000030FE280AB5EEC09A0023F7EE008A0093D9
:10951000F1EE10FA58BFF0EE408A0123A8E798E870
:10952000070089E80700C7E7009B002B7FF473AFB3
:109530000023204684F80431FFF788F938B120462B
:10954000FFF776F9002840F025818DED0A8A95F81D
:109550000A3495F80C229A4240F233812B4493F856
:109560002C34002B00F02D8195F80B3495F80D224A
:109570009A4240F226812B4493F82D34002B00F0C0
:10958000208108A9584618F06FFA8DED080ACDED34
:10959000090A8DED0A1A08A81BF05CFF002840F0AC
:1095A000178108A81BF070FF002840F011815FEDC3
:1095B000607A04F1B00094ED357A68EEA78A5FED29
:1095C000637AE7EE278AC4ED358A1CF0B5FAA36802
:1095D0005FED677AF0EE408A93ED007AB4EEE77AB9
:1095E000F1EE10FA00F1F8802046B0EE680AFFF7BD
:1095F000E5F808A81BF082FEA3688DED110A11A8FA
:10960000CDED120A8DED131A93ED000A1BF076FED4
:10961000204684ED1F0AC4ED200A84ED211AFFF7CD
:1096200083F928B1B2EE000A04F17C001BF0BAFE07
:10963000019BB3B33046FCF7F1FB012831D996F812
:10964000F402B023F0EE087A03FB006696ED3B7A55
:10965000B4EEE77AF1EE10FA23D595F80B040C235B
:10966000F1EE0C7A03FB005595ED877AB4EEE77ABC
:10967000F1EE10FA15DBD4ED1D7A1FED907AF4EEC1
:10968000C77AF1EE10FA0CDD1FED937AF4EEC77A8B
:10969000F1EE10FA05D5B6EE000A04F17C001BF0DD
:1096A00081FE5FED987AF4EEE78AF1EE10FA22D5AA
:1096B0001FED9B0A08A81BF021FE0EA88DED0E0AD7
:1096C00094ED3F0ACDED0F0A8DED101A1BF016FE3A
:1096D00011A904F1A0008DED110ACDED120A8DED56
:1096E000131A1BF02BFED4ED2B7A94ED3F7A77EE14
:1096F000877AC4ED2B7AF1EE047A94ED2B7AB4EEEE
:10970000E77AF1EE10FA3BDB17F034F95FEDB17A4E
:1097100094ED2B1A40F2C93094ED280A21EE271A55
:10972000F1EE410A8DED011ACDED000A17F08AFE27
:1097300040F2CA309DED011ADDED000A84ED280AE1
:1097400094ED290A17F07EFE40F2CB309DED011A10
:10975000DDED000A84ED290A94ED2A0A17F072FE65
:1097600004F1A00104F1940084ED2A0A1BF0E6FD47
:1097700084ED2A8A84ED298A84ED288A84ED2B8A57
:10978000002384ED3F8AC4F8E430C4F8E830C4F81C
:10979000EC309CE5E368F7EE000A93ED000A17F061
:1097A00007FD00283FF4D1AE94ED1C0AB0EEC00ACC
:1097B000BEF068FDDDED0A7A27EE800A8DED0A0A1B
:1097C000C5E68DED0A8A8DED098A8DED088AE2E6FF
:1097D0002046FFF753FC1EE6C3ED007A04E700BF06
:1097E000F0B52DED108BA1B0044617F0C3F800F5CD
:1097F000836390ED868AD3ED007AF4EE487AF1EE39
:1098000010FA48BFB0EE678ADFED5C7AB4EEE78A03
:10981000F1EE10FA0DDD0023C4F8E430C4F8E830AE
:10982000C4F8EC300023C4F8FC3021B0BDEC108B40
:10983000F0BD204616ADFEF755FD2046FEF7FEFEB4
:10984000B0EE480A204604F14C06FFF753FC2046D0
:10985000FFF714FCFEF75EF904F1280100F53A72F7
:1098600016A818F051F90FCD0FC60FCD0FC62B68F3
:1098700004F1740204F1700104F14C00336004F14E
:10988000780318F0E7FA94ED1E8AB0EE480ABDF0AE
:10989000F3FE84ED650AB0EE480ABEF0F3FC204604
:1098A00084ED640AFEF712FDFEF734F904F5B47195
:1098B000FDF704FF74F01AFCD4F89831C31A632B37
:1098C000B3D9C4F8980146F05FFC054674F016FC65
:1098D000DFED2B7A94ED1E0A074694ED1C8A0E46A6
:1098E00094ED1D9A20EE270A28EE278A29EE279A62
:1098F00017F004FDD4ED53AAB0EE40AA94ED35BAAA
:10990000B7EEC88A94ED36CAB7EEC99A94ED55DA27
:10991000B7EECBBA94ED56EAB7EECCCA94ED57FA4F
:10992000FEF7D0FA8AEE807A164B174A2846019342
:10993000164B1749B7EECDDA0093B7EECEEA154BCA
:10994000B7EECFFAB7EECAAA8DED12FB8DED10EB94
:109950008DED0EDB8DED0CCB8DED0ABB8DED08ABE7
:10996000B7EEC77A8DED069B8DED147B8DED048BE4
:10997000CDE9027646F090F957E700BFCDCC4C3EDA
:10998000E02E6542DA210F08BB4C0F0830220F0889
:10999000784A0F08B04C0F0870470000002070474D
:1099A000704700000020704700207047002070477B
:1099B000002070479FED010A704700BF00000000C3
:1099C0009FED010A704700BF0000000070470000D3
:1099D000002070477047000010B50446143000F0B6
:1099E00019F804F12C0000F015F804F170008CF067
:1099F000E9FF04F1F4008CF0E5FF4FF0FF3320465F
:109A0000C4F8543110BD0000014B1868704700BF06
:109A10008482003070470000094A0123D2ED057AA4
:109A2000D8B2F4EEC07AF1EE10FA02DD0138C0B21D
:109A3000704701331432082BF0D10720704700BF64
:109A40009C4D0F080C4B1422DFED0C6AF0EE407AAF
:109A500002FB003090ED047A90ED010AB0EEC76A87
:109A6000B4EEE66AF1EE10FA5EBFD0ED006A77EE72
:109A7000E67AA7EE270A70479C4D0F0800000034D5
:109A800010B504463648F0EE407A012103462DED2C
:109A9000068B90ED077ACAB2F4EEC77AF1EE10FAAF
:109AA00023DD013AD2B2142101FB023393ED027A95
:109AB00087EE870ADFED2B7AB4EEE70AF1EE10FAB3
:109AC00019DA44F089FDA7224FF4801144F03CFDDF
:109AD000637C5022D4ED467A02FB034393ED0B0ADC
:109AE00030EE270ABDEC068B10BD01311430082979
:109AF000CFD10722D7E793ED049A93ED008AB0EE19
:109B0000C97AD3ED019ADFED188A9FED18AAB4EE59
:109B1000E77AF1EE10FA12D568EEE98ABEF0D6F8CF
:109B2000F0EE487A88EE8A7AE0EE077A9FED107AB6
:109B300067EE876A77EE677A86EEA70AD2E768EE65
:109B4000C98AC8EE8A0ABEF0DFF989EE897AF7EE93
:109B5000007A30EE670AF0EE487AE7EE007AE5E741
:109B60009C4D0F0800000034CB868F430AE81C414F
:109B70003CFEC14ADFED257A254920EE277A30EEFA
:109B8000270A08B587EE005A2DED028BB0EE450A84
:109B9000FFF742FF142303FB001140B2FFF752FF0F
:109BA000DFED1C7AD1ED045A91ED038AB0EEE57A2F
:109BB000B4EEE77ADFED187AF1EE10FA12D520EE66
:109BC000270A9FED167AC7EE007A91ED000A35EE6E
:109BD000400A27EE800ABDF0D5FF20EE080ABDEC52
:109BE000028B08BD65EEA75ADFED0D7AC7EEA50A18
:109BF000F7EE007A70EEA70AD1ED017A80EE270A1F
:109C0000F1EE600ABEF080F9E7E700BF3CFEC14A12
:109C10009C4D0F0800000034CB868F430AE81CC11E
:109C20000AE81C4108B5FFF7A5FFDFED087A9FEDB4
:109C3000087AB4EEE70ADFED077AF1EE10FA20FEBB
:109C4000270AC7EE007AB1EEE70A08BD000000342B
:109C5000CDCC9C3FBC77E93610B52DED028BF0EEF4
:109C6000608A0446FFF70CFFB0EE408A2046B0EE53
:109C7000680AFFF705FF30EE480ABDEC028B10BD05
:109C8000427C5021D0ED467A01FB020292ED0B0A94
:109C900030EE270AFFF7C6BF38B52DED088BB0EEC2
:109CA000409A0546F0EE609A1524B0EE408ADFED4A
:109CB0001DAA9FED1DAA9FED1DBA013CA4B25CB385
:109CC000F0EE490A2846B0EE480AFFF7C5FF70EEED
:109CD000698AF0EE490A284638EE2A0AFFF7BCFFE7
:109CE000B0EEE87A70EE697AB4EECA7A77EEE87A86
:109CF000F1EE10FA10D468EEAA8A40F26310B0EECA
:109D00004B1AF0EE4A0A88EEA70A38EE400A17F01E
:109D100099FBB0EE408AD0E7B0EE480ABDEC088B64
:109D200038BD00BFCDCCCC3D0AD7233C00247449BC
:109D3000002343608360C360036143618361C36147
:109D4000002380F82030704790F82020531C00EB4F
:109D50008202DBB2062B80F8203082ED010A84BF3C
:109D6000002380F82030704700228EF055B90000A3
:109D70004FF0FF3310B543610023044600F59670A1
:109D800040F8D03C40F8CC3C40F8C83C40F8803C1F
:109D900040F87C3C40F8783C40F8303C40F82C3CA3
:109DA00040F8283C0C4B0360002380F82030FFF77C
:109DB000BFFF0A4B04F5C870C4F82C3173F0ECFAFD
:109DC000074B204607491C6040F0A4FED4F814312C
:109DD0002046C4F8183110BD744F0F08844F0F0887
:109DE0008882003030500F0800F5967008B548F0B2
:109DF0004FFBDFED027A20EE270A08BD00007A440F
:109E000090ED5D0ADFED057AB0EEC07AB4EEE77A48
:109E1000F1EE10FA48BF90ED5E0A70470000003482
:109E200073B5D0F8283104460E4663B174F05EF97C
:109E3000D4F82831C01A42F20F73984203D894ED37
:109E4000490A02B070BD114B1D687DB195F84E11E5
:109E50002846FFF7ADFD48B101AA95F84E112846F6
:109E6000FFF79CFD10B19DED010AEAE75021DFEDFF
:109E7000087A01FB064494ED0A0AB4EEE70AF1EE13
:109E800010FA58BFB0EE670ADBE700BF84820030EB
:109E900000000C4208B561B10378022B02D90648D4
:109EA00074F0F6F85A1C027000EB83004160012048
:109EB00008BD0846FCE700BF3C4E0F082DE9F843FB
:109EC00005460E469146002400F13C082B7CA34237
:109ED00011DD00234A463146012013F09FFA50233A
:109EE00007460021634358F8030013F0A7FA87429E
:109EF00004D00134EAE70020BDE8F8830120FBE745
:109F000070B50B46064614469AB111469847054669
:109F100028B9236820465B68BDE8704018470146B1
:109F20003046FFF7B7FF20B92B6828465B68984793
:109F3000EFE770BDF0B50D4685B011461A460446F0
:109F4000CDE90213FFF7BAFF034698B90A48042780
:109F5000006840680668DDE90212CDE90037074B6A
:109F60003668B04702462946204605B0BDE8F040B5
:109F7000FFF7C6BF0022F6E760820030801A0600B5
:109F80001A4B1B682DE9F0470546D0F884915868B4
:109F90004FF0010A164C036804F1E4089B689847E7
:109FA00095F921310646002BA4BF01269E40236867
:109FB00019EA030F07D000270AFA07F3334206D144
:109FC0000137202FF8D10C344445F0D10BE0237A2F
:109FD000FAB261682846FFF7ADFF2B78032B02D059
:109FE0002B7C032BECD1BDE8F08700BF60820030F2
:109FF00050510F087FB5D0ED457A01239FED3F7A90
:10A000000446F0EEE77A0376F4EEC77AF1EE10FA42
:10A010000AD400F58A70002303A90190039341F04C
:10A0200053FD019840F03AFF00257623344920463D
:10A030002A46E563C4F88C50C4F8DC50FFF77AFF79
:10A040002378032B18D0237C032B15D076232A46A4
:10A050002C492046FFF76EFF2378032B0CD0237C7E
:10A06000032B09D094F92121AA4207DA2046FFF7F1
:10A0700087FF2378032B0ED104B070BD7723D2B2B3
:10A0800021492046FFF756FF2378032BF4D0237C89
:10A09000032BEBD1F0E7237C032BEDD0D4F88431F4
:10A0A000DA0403D5637E0BB9012363760025637E52
:10A0B000EAB2EB40DB070CD40135082DF7D1237849
:10A0C00023B1237C13B16368002BD5D10F4801F075
:10A0D00013FB3820019201F097FF064618B1019A50
:10A0E00021468FF027FA31462046FFF7D3FE23782A
:10A0F000032BC1D0237C032BDED1BDE7000000344D
:10A1000099730B0855980B08ED910B08584E0F08E2
:10A11000054B1B682BB141694A1C02D0184645F01B
:10A12000FDBF0020704700BF2486003002290BD8F5
:10A13000502303FB010191F8390030B191F83A0046
:10A1400018B191F83B007047002070472DE9F047A7
:10A15000044673F0CBFF42F210730027D4F87C6101
:10A160004FF0500942F2107A861B9E4288BFC4F815
:10A170007C01FDB2237CAB421CD929462046FFF767
:10A18000D5FF70B109FB0548D4ED460A204698ED8D
:10A190000D0AD8ED097A30EE270AFFF77DFD88ED2C
:10A1A0000C0A564504D909FB0540303040F076FED4
:10A1B0000137DEE7617C2046FFF732FE84ED5E0A60
:10A1C000BDE8F08770B504462DED028B86B073F0C4
:10A1D0008DFFD4F81C310546C31AB3F57A7F3FD3FF
:10A1E00094ED467A9FED3A8AF0EEC76A394BD4ED8A
:10A1F000457A1B68F4EEC86ADB6AF1EE10FA93F850
:10A200009C6022D5F0EEE76AF4EEC86AF1EE10FA2F
:10A210001BD502A801F09AFA16BBFDF77BFC02A938
:10A22000FDF74CFAE0B1DDED037A9FED2B7AF8EE05
:10A23000E77A67EE877AB0EEE77AB4EEC87AF1EEA5
:10A2400010FA11D4C4ED467A11E077EE676AB7EEE2
:10A25000006AF0EEE66AF4EEC66AF1EE10FA1CDC73
:10A2600006B0BDEC028B70BD1C4BC4F81831C4F8AD
:10A270001C51FDF74FFCFCF7FDFE2046FFF766FF83
:10A2800051F058FB94ED467A154A0621B7EEC77A8D
:10A290008DED007B4BF04CFCE2E7F0EEE76AF4EE6C
:10A2A000C86AF1EE10FADBD4002ECBD004F58A7028
:10A2B00084ED457A40F0F2FD51F03CFB094A012162
:10A2C00006B0BDEC028BBDE870404BF031BC00BF66
:10A2D00000000034608200300AD7233C6F12833ABA
:10A2E000A14E0F087C4E0F082DE9F0412DED048B97
:10A2F00084B0044640F2723200F5C87103A800250C
:10A3000013F02AFAD4ED437AD4ED446A50229FED3B
:10A31000806A37EEE67A637C02FB0343B0EEC77ACD
:10A32000B4EEC67AF1EE10FAC1BF9FED7A7A67EE0D
:10A33000877A9FED797AE6EE877AC4ED447A93F8CE
:10A340003970E9B223788B4206D904EB81030135D9
:10A35000586800F0ADFAF4E74FF000089FED6F9AEF
:10A36000DFED6F8ADFED6F9A5FFA88F5237CAB42F1
:10A3700071D9502303FB054393F83920002A3FD0BD
:10A38000D3ED0C7AF4EEC97AF1EE10FA0BDBF4EEB1
:10A39000677AF1EE10FA06D6F0EEE77AF4EE687A14
:10A3A000F1EE10FA04DD502303FB05435A6A1A63E9
:10A3B000502606FB054696ED098AD6ED0D0A96F85D
:10A3C000383038EE208AF3B9294620468FF084FBD6
:10A3D00078EE400A204696ED0C0AC6ED1A0AFFF701
:10A3E0003BFCD4ED467A30EE670AB4EE400AF1EE5B
:10A3F00010FA18D75023002203FB054383F83A20B4
:10A4000008F10108B0E7012B03BFD6ED0C0AD4ED2B
:10A410005C7A30EEC88A96ED0B0A04BF88EE297A82
:10A4200087EE270AE1E7F0EEC07A502101FB0545EF
:10A43000F4EE687AF1EE10FAD7BF0123002385F815
:10A440003A30D4ED447ACEBF85F83A3037EE800A00
:10A4500085ED0B0AD4E7627C20461146FFF766FEC5
:10A4600048B1502104F5967001FB0242D16992ED8A
:10A470000B0A47F0EFFF94F92011267C002907DB37
:10A48000B14205DACAB220461146FFF74FFE68B95D
:10A4900000226274D5B2AE4209D929462046013263
:10A4A000FFF744FE0028F5D0657400E06274204692
:10A4B000FFF788FE2046FFF72BFE10B120468EF0F6
:10A4C0003FFB637C502505FB034393F83930BB42C7
:10A4D00016D045F059FE4FF6FF7145F01FFE78B1DA
:10A4E000607C05FB004494F83930002B14BF002237
:10A4F0000422019245F048FE019A122145F0A0FD88
:10A5000003A813F04BF904B0BDEC048BBDE8F08157
:10A510000AD7233C0AD7A33C48E17A3F0000003425
:10A52000FFFF7F7F002019462DE9F04F04460F46BC
:10A5300087B0007C04F13A0300220121D5B25033E8
:10A54000A84205D9013203F84F1C03F8501CF5E767
:10A550006F4B1E68F06A03685B68984740B151F022
:10A56000E9F96C4A062107B0BDE8F04F4BF0E0BABC
:10A5700051F0E0F9684A06210A254BF0D9FA002388
:10A5800003A904F58670039341F09EFA73F0AEFDC3
:10A5900080462046FFF7A8FE73F0A8FDA0EB080058
:10A5A000B0F5FA7F02D95D4801F0A6F8B06A0A2139
:10A5B00003685B689847617C2046FFF7B7FD002879
:10A5C000E7D0B06A013D642103685B68984715F0E5
:10A5D000FF05DBD1524B05951B888DF80650ADF871
:10A5E0000430CDE90355052573F080FD80462046F3
:10A5F000FFF77AFE73F07AFDA0EB0800B0F5FA7F62
:10A60000D1D8617C2046FFF791FD0028EFD094F867
:10A6100010B00DF10C08A14601AA4FF0000A5FFA34
:10A620008AF18B4516D92046FFF780FD50B1D8ED51
:10A63000007A99ED097A137877EE877A0133C8EDBD
:10A64000007A13700AF1010A08F1040809F15009AF
:10A650000132E4E7B06A013D642103685B68984712
:10A6600015F0FF05C0D1A9464FF05008237C5FFAD2
:10A6700089F6B34226D906AB334413F8143C33B9F8
:10A6800008FB064686F83B3009F10109EEE7002F8A
:10A69000FAD006AA07EE903A2046D4ED460A02EB1D
:10A6A0008602F8EEE77A12ED030A80EE270AFFF73A
:10A6B000F3FA08FB064002A98DED020A303041F0A2
:10A6C00003FAE1E700264FF05008DFF85C902046DF
:10A6D000617CFFF7A5FB84ED5E0A237CF7B2BB42E9
:10A6E0000FD908FB074393F83B3043B1013551F0D4
:10A6F00021F97B1C4A46EDB206214BF019FA0136CE
:10A70000EBE70DB907484FE707B0BDE8F08F00BF92
:10A7100060820030BC4E0F08E74E0F08FD4E0F0858
:10A7200000F90E08394F0F08174F0F0808B5037CC2
:10A73000022B02D9034873F0ABFC5A1C0274184672
:10A7400008BD00BF584F0F0838B50246057C0024ED
:10A75000E1B28D4206D910460134FFF7E7FC00282C
:10A76000F6D138BD281E18BF0120FAE770B50D4696
:10A7700009780446072906D8027E437E22B90122C1
:10A780008A401343437670BD002BFCD0002622780C
:10A79000F3B29A42F7D904EB83032946013658688D
:10A7A0000368DB689847F2E737B50D460192FFF77B
:10A7B000CBFF0199044630B904482A46044B00688F
:10A7C000C06A13F0BFF9204603B030BD608200308C
:10A7D000AFB01008014B1868704700BF8882003086
:10A7E0007047000073B5436805460C461B7C8B42DE
:10A7F00042D900F10801212201A812F0ADFF73F047
:10A8000075FC6A68502303FB0423D969411AB1F52A
:10A81000FA7F33D2196A401AB0F5FA6F2ED2D3ED0F
:10A82000097A9FED177AF0EEE77AF4EEC77AF1EE47
:10A8300010FA54BF0120002050269FED127A06FB2B
:10A8400004F31A4482F8390069680B44D3ED0A7A9C
:10A85000F4EEC77AF1EE10FA06D49FED0B7AF4EE1F
:10A86000C77AF1EE10FA04DD06FB0411002381F82B
:10A87000393001A812F092FF02B070BD0020DBE772
:10A8800000000034000048C300004843044B10B5EA
:10A890000446C0E90031083072F07EFD204610BD4C
:10A8A0003C520F084368502000FB0131CA637047D7
:10A8B00013B50368044601919B6898472368019982
:10A8C00020461B6902B0BDE810401847F8B52DEDD1
:10A8D000028B4368F0EE408AB0EE608A05461B7C2E
:10A8E0000C468B421FD9502773F000FC6B68F0EECA
:10A8F000680A674306463B4493ED090A16F058FC84
:10A90000A0B96B68502202FB04331E6250216B68B1
:10A910004C432344C3ED098A6B68234483ED0A8AC0
:10A9200069680C44E661BDEC028BF8BD6B68F0EE23
:10A93000480A3B4493ED0A0A16F03AFC0028E0D09E
:10A94000E4E70000B0EEC07ADFED297AB4EE677A72
:10A95000F1EE10FA49DCB4EE400AF1EE10FA44D6FA
:10A96000436893F9803163B190ED087ADFED217A85
:10A97000F0EEC76AF4EEE76AF1EE10FA03D580ED67
:10A98000080A01232BE077EE407ADBB237EE006A4B
:10A99000F0EEE77AC7EE866A9FED176A07EE903A07
:10A9A000F8EE677A26EE866AB4EEE76A9FED136AE0
:10A9B000F1EE10FA15DDF2EE047A436A013366EE29
:10A9C000A76A43620023C6EE267AF7EE006A27EEF6
:10A9D000800A76EEE76AA7EE260A80ED080A184696
:10A9E0007047F0EE467A0123EFE70023F7E700BF58
:10A9F000FFFF7F7F0000003400004843CDCCCC3DFA
:10AA0000002070470020704700207047704700000A
:10AA10000020704790F836007047000090F83B0027
:10AA200070470000012070470020704702207047E7
:10AA30007047000010B5044601F0EEFA204610BD44
:10AA400090F8A835934207D902F5B07250F8220069
:10AA500010B103689B6A1847002070472DE9F34145
:10AA60006E46054604460F4600F5C87886E80C0099
:10AA7000114B45F8043B28462C3500F043FDA84512
:10AA8000F9D104F2AC53C4F8A47596E8030083E846
:10AA90000300089B20460949C4F8B43540F03AF851
:10AAA000074B1A6812B1074873F0F2FA20461C608F
:10AAB00002B0BDE8F08100BF80540F0848530F0872
:10AAC0008C82003050520F082DE9F04F2DED028B93
:10AAD00090F8A89585B00446B9F1000F6BD17F239B
:10AAE00004F5C87504F5B067261D80F8B835042351
:10AAF0009FEDAC8A0DF10F012A308DF80F3041F037
:10AB00001FF85FFA89FA1C22FF212846C0F032FCA8
:10AB100085F864A096F926B0ABF103031C2B2AD864
:10AB2000DFE813F01D001D00290029004E00290058
:10AB30009800A400B300C0005A0068008C007000A8
:10AB4000290029007F002900DA002900E700CD0054
:10AB5000F5002900020110011D0129001D004420FB
:10AB600001F052FA804620B133462A4621468FF042
:10AB7000EDF9C7F80080386850B1E96EC5F868B0E3
:10AB800031B1894B43F8291040F0BEF940F0B4F9D7
:10AB90000AF1010A57F8040B5FFA8AFA20B1036838
:10ABA0009B68984784F8A8A509F1010970352C36EF
:10ABB000B9F1090FA5D105B0BDEC028BBDE8F08F4E
:10ABC0007C2001F021FA80460028D2D033462A4664
:10ABD000214690F001FFCCE7482001F015FA8046AD
:10ABE0000028C6D0032300932A463346214691F01D
:10ABF00015F9BEE7482001F007FA80460028B8D0D2
:10AC00000623F0E77C2001F0FFF980460028B0D051
:10AC100033462A46214690F0DFFE644BC8F80030E8
:10AC2000A7E77C2001F0F0F980460028A1D0334648
:10AC30002A46214690F0D0FE5D4BEFE7442001F01C
:10AC4000E3F98046002894D033462A46214691F005
:10AC50006BF88EE7382001F0D7F98046002888D0BD
:10AC600033462A4621468FF03BFE82E7302001F032
:10AC7000CBF9804600283FF47CAF33462A46214674
:10AC8000CDF800A091F0A0FB73E7542001F0BCF9CF
:10AC9000804600283FF46DAF33462A4621468FF0A8
:10ACA000FDFE66E75C2001F0AFF9804600283FF426
:10ACB00060AF33462A46214690F046F859E75820BF
:10ACC00001F0A2F9804600283FF453AF33462A46EC
:10ACD00021468FF08DFF4CE7782001F095F98046F2
:10ACE00000283FF446AF33462A46214690F0CAF882
:10ACF0003FE72C2001F088F9804600283FF439AF67
:10AD000033462A4621468FF0C9FA2A4B86E7482067
:10AD100001F07AF9804600283FF42BAF33462A46EB
:10AD2000214691F0C3FB24E7282001F06DF980460D
:10AD300000283FF41EAF33462A4621468FF0AEFA74
:10AD40001D4B6BE75C2001F05FF9804600283FF463
:10AD500010AF33462A4621468EF0B0FF09E7A02007
:10AD600001F052F9804600283FF403AF33462A46EB
:10AD700021468FF093FA114B08F1880088ED1D8A67
:10AD8000C8F800304FF6FF7388ED1E8AA8F82E3001
:10AD9000A8F8703088ED1F8A88ED208A72F0FCFADE
:10ADA000E7E600BF0000C07F90820030F4520F0839
:10ADB000601A1108701C110864151108181B11087D
:10ADC00090F8A8358B4283BF702303FB010090F8F5
:10ADD000E10100207047000090F8A8358B4283BF46
:10ADE000702303FB010090ED6B0A9FED010A704791
:10ADF0000000000090F8A8358B4206D901F5B0712B
:10AE000050F8210008B18FF05BBA9FED010A70473E
:10AE10000000000010B490F8A8450A468C4214D9EE
:10AE200001F5B07450F824407CB1E468246A6406EB
:10AE300003D55DF8044BFFF7DDBF702101FB020372
:10AE400093ED6B0A5DF8044B70479FED010AF9E73B
:10AE50000000000090F8A8358B420BD901F5B071C5
:10AE600050F8210038B1C3681B6A1A4214BF012090
:10AE7000002070470020704770B590F8A835044650
:10AE80000E461546934201D8002070BD02F5B073FE
:10AE900050F823000028F7D003689B6998470028E2
:10AEA000F2D0702202FB0544D4F8B0313360ECE7F5
:10AEB00070B590F8A83504460E461546934201D861
:10AEC000002070BD02F5B07350F823000028F7D0C1
:10AED00003689B6998470028F2D0702202FB054462
:10AEE000D4ED6D7AF4EE677AF1EE10FAE8D6C6ED9D
:10AEF000007AE6E770B590F8A83504460E46154688
:10AF0000934201D8002070BD02F5B07350F82300C1
:10AF10000028F7D003685B6998470028F2D07022B8
:10AF200002FB0544D4F8B8313360ECE790F8A8355B
:10AF300093420ED902F5B07350F823305BB1702301
:10AF400003FB020292F8F00130B1D2F8EC310B6051
:10AF500070470020704718467047000008299DBFC1
:10AF60002C2303FB0100406800207047474B1B68FF
:10AF70002DE9F04F2DED028BDB6A87B0044693F884
:10AF80009C30002B7DD04FF00009DFF814A1DFF8D2
:10AF900014B19FED3F8A5FFA89F594F8A835AB426A
:10AFA0006FD905F5B07354F82300002853D0036817
:10AFB0005B6B98477023074603FB054393F8E0312A
:10AFC000834248D2032857D8DFE800F04502484FB3
:10AFD000304E4FF0000850F0ADFC94F8A8256B1CE3
:10AFE0000421AA4289BF7022B0EE487A02FB0542D2
:10AFF00092ED6B7A702202FB0545B7EEC77A524696
:10B0000095ED6D6A0096B7EEC66A8DED027B8DED0B
:10B01000046B4AF08DFD012384F8B9358BF80B30B1
:10B0200085F8E071D4F8B4354BB3002255B25957C6
:10B03000481C03D0414502F10102F7D194F9B8351B
:10B04000AB4208DBD4F8B03542463146D4F8AC0503
:10B05000984784F8B85509F101099CE72C230E4E56
:10B0600003FB054393F92D80B5E72C230B4E03FB1F
:10B07000054393F92E80AEE70026B046ABE71D46A8
:10B08000DCE707B0BDEC028BBDE8F08F60820030DA
:10B09000000000007D520F080615110874520F08B9
:10B0A0008C520F080D8300300020704790F8A835AF
:10B0B0008B4207D901F5B07150F8210010B1036837
:10B0C000DB6918470020704708299CBF702303FBE9
:10B0D000010000F5C8707047F8B504460E461546E5
:10B0E0001F46FFF7E3FFD0B10D2D19D8082E9CBFE6
:10B0F000702101FB06444FF6FD7104F5C87434F865
:10B100001520531E9BB28B420AD807EE902A9FED62
:10B11000057AF8EEE77A67EE877AC7ED007AF8BD30
:10B120000020FCE76F12833A90F8A835934207D9C4
:10B1300002F5B07250F8220010B103685B6A18473C
:10B14000002070470B46114690F8A8259A4207D96F
:10B1500003F5B07350F8230010B10368DB6A184799
:10B16000002070472DE9F04F002493B005460E46AD
:10B17000174621462F2206A8059405F5B069C0F0B0
:10B18000F9F805F12A0A4FF02C0B05F5FC730BFBBF
:10B1900004F259F8040BE5B21AF9021030B951B9AA
:10B1A0000134092CF3D14FF0010813E070226243FF
:10B1B0009A58914212D001351448154B4FF00008AF
:10B1C0000068EDB20193324600953946114BC06AD2
:10B1D00012F0B8FC404613B0BDE8F08F05A9332249
:10B1E00003938FF04DF905A98046039B0028D7D122
:10B1F0000135064801913246EDB20068054B3946EB
:10B200000095C06A12F09EFCE4E700BF6082003047
:10B210008D5E0F08B4520F082DE9F04F06468DB031
:10B220000027DFF87C90DFF87CA0DFF87CB096F890
:10B23000A835FCB2A3422ED9702505FB046595F80C
:10B24000E83133B395F8E91119BB4FF0010820221A
:10B2500004A8444489F81980C0F08CF84AF21043DD
:10B2600007EE904A03AA4C215046F8EEE77AADF873
:10B2700028302423CDED037A4AF050FA50F05AFBDF
:10B280009BF80030054A042100944AF051FC85F8EF
:10B29000E9810137CBE70DB0BDE8F08FC4520F084C
:10B2A0000D83003014870030BD260030304B2DE96F
:10B2B000F04F1E6885B0044646B1D0F8A41530465C
:10B2C00044F02CFF10B1304643F0A4FD4FF00008CD
:10B2D0004FF02C0A4FF0700B72F008FF01905FFAEC
:10B2E00088F594F8A835AB4239D904EB8507D7F82F
:10B2F000800588B30AFB05430BFB054993F92A2017
:10B30000D9F8F8118A4227D132B30268D26890473F
:10B31000D7F880050268126B904799F8E12112B1C5
:10B32000019BC9F8E431BEB1D4F8A415304644F00D
:10B33000F5FE88B172F0E2FE02460B46CDE902103E
:10B340002946D7F8800590F0C5F82946D7F880053A
:10B35000DDE9023290F034F908F10108BFE7204638
:10B36000FFF704FE204605B0BDE8F04FFFF754BFDD
:10B37000248600302DE9F0474FF000080446894646
:10B38000012647464FF0700A2DED028BB0EE408A41
:10B3900094F8A8355FFA88F5AB421AD929FA05F373
:10B3A000DB070AD505F5B07354F8230078B10368BC
:10B3B000B0EE480A9B6B984706400AFB054508F12A
:10B3C000010895F8E0319F4238BF1F46E0E7064686
:10B3D000F3E727B97F23A4F8B835034BDF72304673
:10B3E000BDEC028BBDE8F0870D83003090F8A835E6
:10B3F0008B4207D901F5B07150F8210010B10368F4
:10B40000DB6B1847002070470B46114690F8A825C3
:10B410009A4207D903F5B07350F8230010B10368BE
:10B420001B6C18477047000070B504460E46002597
:10B43000E9B294F8A8358B4205D932462046013549
:10B44000FFF7E2FFF4E770BD2DE9F843024690F8FC
:10B45000A855002400F12A062C2700F5FC784FF0AF
:10B460007009E1B28D420FD907FB04F309FB04F028
:10B47000F35658F80000834209D11BB11046FFF77C
:10B480009FFC10B10134ECE70120BDE8F8830020F7
:10B49000FBE7000010B590F8A82504468A4217D9AA
:10B4A000702202FB010393F8E031022B03D004D990
:10B4B000032B18BF0023184610BDFFF797FF48B9AC
:10B4C0002046FFF7C1FF00280CBF06230123F2E747
:10B4D0000023F0E70623EEE70B46114690F8A82577
:10B4E0009A4207D903F5B07350F8230010B10368EE
:10B4F0005B6C184700207047014B1868704700BF0D
:10B500008C82003010B5044602493FF003FB204610
:10B5100010BD00BF08550F0810B5044620305EF07E
:10B52000A7FB044B204604491C603FF0F3FA204679
:10B5300010BD00BFB4820030A0560F082DE9F341C2
:10B540000546B7EE000A002202213EF0EDFE284635
:10B5500091F0A4F85EF022FD234B04461E68F06AC9
:10B5600003685B6A98470B46022102462046009119
:10B570005EF094FBB5F94A70002F13DDD6F82C80ED
:10B58000BCB2D8F8003040465B68984728B198F8BC
:10B590004D3013B1C92FA8BFC824B06A2146036833
:10B5A0005B6898472022002195F9490015F0B2FF09
:10B5B000C4B25FF037FE5FF07DFD70B9B06A013450
:10B5C00005210368E4B25B689847072CF1D9074866
:10B5D00002B0BDE8F04171F06DBF072CF7D885F8D7
:10B5E000494002B0BDE8F0816082003008560F0883
:10B5F00010B5044691F008F82046BDE8104091F0DF
:10B6000033B800002DE980481446284B012293B03E
:10B6100005460E464FF00008DFF89490DFF894A03E
:10B62000DFF894B01A7072F061FDD9F80030A0EB29
:10B6300008020746039341F287339A421FD90398C1
:10B640005346342205A9B846CDE90056C06A12F027
:10B6500079FA214605A8049471F01CFF03985B4613
:10B66000342205A9CDE90056C06A12F06BFA0494A1
:10B6700050F060F9049B05AA02214AF041FA50F00B
:10B6800059F94FF027FE50F055F952F05FF90A21B1
:10B6900005A812F047F8039B0521986A03685B68C8
:10B6A000984705A812F04AF8BDE700BFB8820030FD
:10B6B000608200302DE00F08653311080FB400B52B
:10B6C00095B0002116AA05A8049152F8043B0392F4
:10B6D0003C220193BFF04EFE054A4021019B04A885
:10B6E00071F080FE039A04A90248FFF78BFF00BFA8
:10B6F00020560F0836560F080FB407B504AA0348A2
:10B7000052F8041B0192FFF77DFF00BF48560F0857
:10B7100038B504460025E289ABB2A0689A4205D943
:10B7200050F823000135B9F071FEF4E7B9F06EFE70
:10B73000204638BD1022044908B5BFF0C1FDB0FA5B
:10B7400080F0400908BD00BFBC82003010220021FB
:10B75000BFF010BE0378022A416023F00D0303708E
:10B7600008D0032A0AD0012A03D1DBB243F0010337
:10B7700003707047037843F00803F9E7037823F078
:10B78000050343F00503F3E773B504460E4615467B
:10B790000193FFF7DBFF2046069A0199C4E9026591
:10B7A000FFF7D8FF02B070BD4B68436003780A789A
:10B7B00062F3000303700B780278C3F3800363F332
:10B7C00082020270D2B20B78C3F3C00363F3C302E8
:10B7D000027070470078420704D4030704D400F0D5
:10B7E000010070470320704702207047F0B587B012
:10B7F00004461546FFF7EEFF88420F46064605D180
:10B8000063682B600126304607B0F0BD0023032893
:10B81000019301D0032913D141F0EAFF08B90026B2
:10B82000F1E7012301AA214641F04AFD0028F6D0A4
:10B83000DDED017A9FED337A67EE877ACDED017AFF
:10B84000032E32D8DFE806F0020916246468032FBD
:10B85000E5D8DFE807F02C2E3C49FCF75BF990F8BF
:10B860009432DB07DBD56468FCF754F9D0F88832F2
:10B870001C44ECE702A8FFF769FFFCF74BF902A9AB
:10B88000FBF71CFF06460028BDD06468039BEFE76A
:10B89000D4ED017A9DED017AF8EEE77A77EE877ABA
:10B8A000FDEEE77A17EE904AD1E70024CFE72C604F
:10B8B000A8E7FCF72FF990F8946216F00106AED0D5
:10B8C000FCF728F9D0F88832E41A2C609BE702A82C
:10B8D000FFF73CFFFCF71EF902A9FBF7EFFE064657
:10B8E000002890D0039BEFE707EE904A9DED017A88
:10B8F000F8EEE77A77EEC77AFDEEE77AC5ED007AE3
:10B9000080E700BF0000C84273B501AA05460E4695
:10B91000FFF76CFF044620B1324601992846FFF735
:10B9200019FF204602B070BD13B5144601AAFFF7F7
:10B930005DFF48B1DDED017A9FED047AF8EEE77A1C
:10B9400067EE877AC4ED007A02B010BD0AD7233CB7
:10B9500007EE900A9FED0C0AF8EEE77A08B527EE9D
:10B96000800ABBF089FEDFED097AB4EEE70AF1EE5A
:10B9700010FA02DDB7EEC00A08BD9FED010BFBE730
:10B9800000000040E17A843F50E0EF300AD7233CCA
:10B9900010B50446806815F0EBFF20B1E068BDE803
:10B9A000104015F0F9BF10BD73B5856804460E460A
:10B9B0001DBBC36823B98B6801258360CB68C36056
:10B9C000636873B92378DB070BD52046FFF702FFC6
:10B9D00001AA01463046FFF709FF10B1019B054659
:10B9E00063602046FFF7D4FF20B9B3680125A36048
:10B9F000F368E360284602B070BD0025E0E7000070
:10BA00000D4B83424FF000038B4106DA00F12550C5
:10BA100000F5311000F5E0507047084B98424FF0A8
:10BA2000FF3371EB0303BEBF00F1564000F5130076
:10BA300000F52440704700BF00D2496B002EB69439
:10BA400090EA010F01D4401A7047C317401A63EB04
:10BA5000E1710D4B83424FF000038B4106DA00F198
:10BA6000255000F5311000F5E0507047074B984223
:10BA70004FF0FF3371EB0303BEBF00F1564000F5FA
:10BA8000130000F52440704700D2496B002EB69495
:10BA900070B52DED028B84B004460D466846FFF765
:10BAA00055FEFCF737F86946FBF708FE064628B353
:10BAB000A368029ADFED148A9B1A039907EE903A65
:10BAC000F8EEE77A67EEA87AC5ED007AE068FFF74E
:10BAD000B7FF08EE100AA068B8EEC88A024428EE44
:10BAE000288A02EBD2725010B7EEC88AFFF730FFF7
:10BAF00028EE000BB7EEC00B85ED010A304604B00E
:10BB0000BDEC028B70BD00BFF67C8E3F002337B5C5
:10BB10000C4601AA022105460193FFF767FE10B902
:10BB2000002003B030BD21462846FFF7B1FF0028B2
:10BB3000F6D0DDED017AF8EEE77AC4ED027AF0E7AF
:10BB400008B5FFF7E3FF08BD38B50D46FFF7DEFF88
:10BB5000044620B19FED030A284619F023FC204635
:10BB600038BD00BF0AD7233CF0B50D4606462DED83
:10BB7000028B8C6889B0D0E90271E868FFF760FF3A
:10BB800008EE100AE019E41B00EBD0704010FFF73C
:10BB9000DFFEB8EEC86ADFED0F4A736826EE246A4E
:10BBA0006A689FED0D1A9B1AB7EEC66A07EE903AC7
:10BBB00026EE006BB8EEE75A07EE904AF8EEE75A29
:10BBC000F7EEC60B25EE011A25EEA40A09B0BDEC6E
:10BBD000028BF0BD8262363C0AD7233CF0B50D469D
:10BBE00006462DED028B8C688DB0D0E90271E868B5
:10BBF000FFF726FF08EE100AE01900EBD0704010A6
:10BC0000FFF7A6FE73686A68B8EEC87ADFED107AAF
:10BC1000B0EE401B9B1A02EE103AE31BB8EEC22AAC
:10BC200000EE103AB8EEC00A22EE272ADFED097ABC
:10BC300027EE277A20EE270AB7EEC22AB7EEC77A98
:10BC4000B7EEC00A27EE011B0DB0BDEC028BF0BDB4
:10BC50000AD7233C8262363CF0B52DED028B8BB0C7
:10BC60000D460021074605AA0691FFF7BFFD0021FA
:10BC700090BB0023CDE90533D7E90261AC68E868E1
:10BC8000FFF7DEFE08EE100AA019A41B00EBD0702F
:10BC90004010FFF75DFEB8EEC86ADFED134A9FED76
:10BCA000131A26EE246ADDE90532B7EEC66A9B1A3E
:10BCB00007EE903A26EE006BB8EEE75A07EE904A90
:10BCC000F8EEE75AF7EEC60B25EE011A25EEA40AA8
:10BCD0000BB0BDEC028BF0BD06AA2846FFF786FD2F
:10BCE0000028C6D0C8E700BF8262363C0AD7233C92
:10BCF00038B50C4602462DED028BC168E068FFF7AF
:10BD00009FFE9568A46808EE100A6019641B00EB9A
:10BD1000D0704010FFF71CFE07EE904AB8EEC81B2B
:10BD2000B8EEE77B87EE006BBDEEC60B10EE103A67
:10BD30005B4200EE103AB8EEC00BBCF0DDFB9FEDAD
:10BD4000087B30EE070BB5EEC00BF1EE10FA03D511
:10BD50009FED057B30EE070BBDEC028B38BD00BFBD
:10BD600000000060FB21F93F00000060FB2119404A
:10BD70000B4630B52DED028B8C6885B0D0E90251B1
:10BD8000D868FFF75DFE08EE100A6019641B00EB2F
:10BD9000D0704010FFF7DCFDB8EEC86A9FED095A7D
:10BDA00007EE904A26EE056AF8EEE75AB7EEC66A45
:10BDB00026EE006B25EE850AF7EEC60B05B0BDEC4E
:10BDC000028B30BD8262363C0B4630B52DED028BC6
:10BDD0008C6889B0D0E90251D868FFF731FE08EECF
:10BDE000100A6019641B00EBD0704010FFF7B0FD23
:10BDF00007EE904AB0EE401BB8EEE76BB8EEC87B9A
:10BE00009FED050B27EE007B26EE000B27EE011BB6
:10BE100009B0BDEC028B30BD0000004050CC863F25
:10BE200084B004B0FFF7D0BF10B52DED048B84684B
:10BE30000B468A68111B224409EE101AC168D868A3
:10BE400002EBD272FFF7FCFD08EE100A5010B8EEBC
:10BE5000C99BB8EEC88BFFF77BFD28EE000B20EEE8
:10BE6000000BA9EE090BBDEC048BB1EEC06B9FED8E
:10BE7000020B26EE000B10BD0000004050CC863FA8
:10BE8000094B984206DDC0F1D64000F5930000F55D
:10BE9000A4407047054B9842BEBFC0F1144000F566
:10BEA000360000F53850704700E9A43500175BCA2A
:10BEB000F8B52DED048B9FED149BB0EE418B076818
:10BEC00006460D4620EE090B28EE098BFDEEC07BE1
:10BED00017EE904A04EBD47007EB6000FFF738FDD3
:10BEE00088EE007B3819FFF7CBFF306051EC170B61
:10BEF000F4F782FD2B68C01841EBE371FFF780FD7A
:10BF00002860BDEC048BF8BD000000404075564031
:10BF100000F10C010830FFF7CBBF000000B52DED9C
:10BF2000068B9FED109B83B0B0EE418B20EE099BFA
:10BF30000190B0EE490BBBF0CDFCB0EE40ABB0EEE3
:10BF4000490BBBF007FD20EE081B01982AEE080BF9
:10BF500003B0BDEC068B5DF804EBFFF7D9BF00BF63
:10BF6000AFF30080000000A046DF913F10B52DED3B
:10BF70000A8B9FED1ECBB0EE409B0446B0EE42AB69
:10BF800021EE0CBB29EE0C9BB0EE4B0BBBF0A2FCE0
:10BF9000B0EE408BB0EE490BBBF09CFCB0EE40CB5A
:10BFA000B0EE490BBBF0D6FC28EE001B204628EE75
:10BFB0000C8B21EE0A1B28EE0A0BFFF7A9FFB0EE4F
:10BFC0004B0BBBF0C7FC20EE0A0B63689FED092BFF
:10BFD000BDEC0A8B20EE020BBDEEC00B10EE102A5A
:10BFE0001344636010BD00BFAFF30080000000A0E9
:10BFF00046DF913F00000000000059400148FFF774
:10C00000A5BB00BFBC8200300121884238BF084672
:10C01000B9F0F8B9FFF7F8BF08B1B9F0F7B9704750
:10C02000FFF7FABFF8B506460F46144622B9254673
:10C03000B9F0ECF92846F8BD10461EB9BDE8F84045
:10C04000B9F0A0B9B9F09EF905460028F2D0BC427B
:10C050002246314628BF3A46BFF042F93046B9F091
:10C06000D5F9E7E737B5089D0446084611461A4654
:10C07000036801959DF81C5000951D68069BA84714
:10C080002060204603B030BD00214FF0FF33002276
:10C0900010B54363044600F14003016041608160D4
:10C0A000C16080F8291000F50C70D9707C3343F81A
:10C0B000742C43F8702C43F86C2C43F8682C43F82C
:10C0C000642C43F8602C43F85C2C43F8582C43F85C
:10C0D000542C43F8402C43F83C2C43F8382C43F8BC
:10C0E000342C43F8302C43F82C2C43F8282C43F8FC
:10C0F000242C43F8202C43F8102C43F80C2C43F844
:10C10000082C9842D1D1214604F5177007F030FB76
:10C11000044B1A6822B9044920461C603EF0FAFC20
:10C12000204610BDCC82003000590F0873B5D0F8FE
:10C13000403204460191994213D0D0F844329942DA
:10C1400018D0D0F848328B4216D102200AE0D4F839
:10C15000383253B3D4F83C324BB34FF0030002B043
:10C1600070BD002094F826308342F8D8431C84F830
:10C170002630F4E70120F5E7D0F83462002EE6D14E
:10C1800094F845233546B6009AB1A319C3F8341282
:10C19000A319019A2846C3F8402294F82630AB42EE
:10C1A0009CBF6B1C84F82630D9E70126E8E70226FD
:10C1B000E6E704F50D7001A930443FF093FDE7E791
:10C1C00038B504460D463FF003FD291D201D3FF004
:10C1D000FFFC05F1080104F108003FF0D3FD05F173
:10C1E000140104F114003FF0CDFD05F1200104F12C
:10C1F00020003FF0C7FD05F12C0104F12C003FF0B9
:10C200007BFC05F1300104F130003FF083FD05F1C6
:10C210003C0104F13C003FF0B5FDAB6BA3636B6BDD
:10C22000636338BD2DE9F04300F14007A1B000235E
:10C230000025064600F51078B9468DF8075003939F
:10C240000493059306930793089309930A930B931A
:10C2500010931193129313931493159316931793AA
:10C2600018931C931D931E9358F8043BF3B1326F3F
:10C27000934222D0D6F8EC20934220D0D6F8682101
:10C28000934213D10221EBB299420FD0C1EB41117D
:10C2900001A809EB81042146FFF792FF39462046A9
:10C2A000FFF78EFF01A93846FFF78AFF01357C377B
:10C2B000032DD9D121B0BDE8F0830021E3E70121AE
:10C2C000E1E700002DE9F04704460E46154680469A
:10C2D00007464FF0000A31462046FFF727FFBA6FA6
:10C2E0005FFA8AF9B2420ED1C3B2022B0BD87C227C
:10C2F00002FB0A44012084F8433084F8420085F8A8
:10C300000090BDE8F0870AF1010A7C37BAF1030F0B
:10C31000E1D1002731462046FFF708FFD8F870200A
:10C320005FFA87F912B9C3B2022B19D9013708F1A4
:10C330007C08032FEED131462046FFF7F7FEC2B24C
:10C34000C2EB421304EB830393F8427067B9022AED
:10C350000BD8012083F8432083F842002A70D0E7ED
:10C360007C2000FB0744C5E700274FF07C0904F15F
:10C37000420A31462046FFF7D9FE034609FB07F083
:10C380005FFA87F81AF8002012B9DBB2022B09D93C
:10C390000137032FEDD194F8271004290BD9144845
:10C3A00071F076FE0444012084F8433084F84200A2
:10C3B00085F80080A5E704F54477002057F8043B92
:10C3C000C2B2B34208D1914202D8531C84F827303C
:10C3D00003322A70002094E733B9481CC43184F832
:10C3E000270044F82160F3E701300528E6D1F1E7A2
:10C3F00040570F08C9B200EB8101D1F8403253B168
:10C40000426F93420AD0D0F8F020934208D0D0F87F
:10C410006C21934206D04FF0030070470020704714
:10C4200001207047022070472DE9F8430F469146DE
:10C43000044600F5BA7894F8425035B97C34444546
:10C44000F9D100252846BDE8F88300234A4639463D
:10C45000012010F0E3FF06460021206F10F0EEFFF0
:10C460008642EBD1EEE70000012303FA01F1D0F898
:10C470000C3319420AD14AB190F82430032B1FBF64
:10C48000591C063380F8241040F823207047000020
:10C490002DE9F043044685B000F5107600257C2791
:10C4A000DFF87080B14656F80C3CE9B20436D9F892
:10C4B0000020934219D1C3B12046FFF79BFFC0B2C1
:10C4C00007FB004090F842307BB903A9A9F10C00AA
:10C4D00003933FF007FC4FF02DFA56F8043C424618
:10C4E000012100932B4649F023FB0135032DD9D1BF
:10C4F00004F1700504F5F274296821B9AB6813B131
:10C5000028463DF00FFC7C35A542F5D105B0BDE8CD
:10C51000F08300BF5C570F0838B504461546FFF797
:10C5200069FFC0B2022808D87C23294603FB0040DB
:10C53000BDE8384054303FF015BC38BD38B504462E
:10C540001546FFF757FFC0B2022808D87C232946BA
:10C5500003FB0040BDE8384060303FF003BC38BD0D
:10C5600037B50D4604468DED010AFFF743FF022D56
:10C5700007D8C0B27C2301A903FB00406C303FF018
:10C58000A3FA03B030BD000038B50546FFF732FF0F
:10C59000C4B2022C13D8C4EB441440350021A400CB
:10C5A00004F1080028443DF0BDFB04F1340104F11E
:10C5B000300029442844BDE838403FF093BB38BDE3
:10C5C00070B505460E461446FFF714FFC3B2022BA2
:10C5D0000DD87C2000FB035394E80700483383E820
:10C5E000070031462846BDE87040FFF7CDBF70BD5B
:10C5F00037B504461546FFF7FDFEC0B2022809D83C
:10C600007C230DF107018DF8075003FB00404430F7
:10C610003FF0DEFA03B030BD1FB590F9303004466C
:10C6200023B390F925300BB36846FFF78FF8FBF77B
:10C6300071FA6946FAF7A0FFC0B1DDED037A012374
:10C640009FED0B0AF8EEE70ADDED027A84F841333C
:10C65000F8EEE77AC0EE800A87EE800A07F0DEFA8D
:10C66000DFED047A20EE270A84ED0B0A04B010BD3A
:10C670008096184B35FA8E3C024690F9250058B149
:10C6800092F8440340B1114491F9300220B192F97B
:10C690002800033818BF01207047000038B590F813
:10C6A000263005465BB100242346E1B22846FFF759
:10C6B000E3FF08B10133DBB20134032CF5D1184696
:10C6C00038BD000090ED0B0A7047000038B50C46ED
:10C6D000D1ED066A11460546FFF78CFED4ED087AC7
:10C6E000C3B27C2094ED076AB7EE007A00FB0353D7
:10C6F000D3ED270AA6EEE67AD3ED265A26EE600A97
:10C7000093ED255A67EEA00AA5EEA70AF0EE607A2F
:10C71000E5EE867AB1EE400A67EEE60AE5EE070A34
:10C72000BBF082FF40F658009FED061ADFED060AC7
:10C7300014F088FED5ED0B7ABDE8384030EE270ABC
:10C7400014F054BEDB0F4940DB0F49C02DE9F04126
:10C7500090F8263004460D468B4202D20020BDE8F8
:10C76000F081FFF747FE04F14006C0B2C0EB401075
:10C7700006EB8000083019F0DFF9B0EEC00ADFEDFB
:10C78000147AB4EEE70AF1EE10FAE7D4294620460F
:10C79000FFF730FEC5B27C2000FB05477B6F002B06
:10C7A000DCD0032DDAD000FB0560D7F87080303084
:10C7B0003EF07CFAD7E91C32934201D1984505D06E
:10C7C0007C2000FB0544C4F87080C7E70120C6E761
:10C7D000000000342DE9F74F04460E46174600F5D9
:10C7E000107A4FF0000B5AF8049B5FFA8BF8B9F1FE
:10C7F000000F26D041462046FFF73EFF08B34146D2
:10C800002046FFF7F7FD7C23C0B203FB004090F801
:10C8100042505DB908F101031B4A39463046DBB28C
:10C8200070F0E0FD284603B0BDE8F08F5AF8102CF8
:10C83000914506D0154A39463046002570F0D2FDA4
:10C84000F0E70BF1010BBBF1030FCCD14FF0000867
:10C850005FFA88F194F826308B420DD92046019179
:10C86000FFF774FF054620B901992046FFF704FF42
:10C8700020B908F10108EBE70125D3E7044A39465E
:10C88000304670F0AFFDCDE784570F0899570F0879
:10C89000BE570F082DE9F04106464FF000082DED78
:10C8A000048B82B090F84613FFF7A4FD06F1400711
:10C8B000C5B27C209FED2F8A00FB0575DFED2E8A27
:10C8C0009FED2E9A54355FFA88F396F826209A4207
:10C8D0004DD919463046FFF7CFFE10B908F10108CF
:10C8E000F1E719463046FFF785FDC4B27C2000FB16
:10C8F0000474D4ED157A5434F0EEE77AF4EEC87A85
:10C90000F1EE10FA0ED5D4ED017AF0EEE77AF4EEFE
:10C91000C87AF1EE10FA05D5002002B0BDEC048B08
:10C92000BDE8F0812946204619F016F9B4EEE80A70
:10C93000F1EE10FAF0DC2946204618F06BFBB4EE5D
:10C94000C90AF1EE10FAE7DC2146284618F0AEFAE3
:10C9500068468DED000ACDED010A18F04FFBDFEDC2
:10C96000087AB4EEE70AF1EE10FAB7DDD4E7012059
:10C97000D3E700BF00000034DB0FC93F920A863FB7
:10C9800000004843022910B5044608D8FFF732FDDD
:10C990007C23C0B203FB004494F8410010BD00208A
:10C9A000FCE7000013B590F8461304460191FFF729
:10C9B000E9FF30B10199204602B0BDE81040FFF711
:10C9C0005BBE02B010BD0000F7B590F925500446DB
:10C9D000002D73D090F84453002D6FD090F846137B
:10C9E000FFF7D0FF94F84133064613B92046FFF70E
:10C9F00013FE002594F82420EBB29A4207D906339F
:10CA0000013554F8230003689B689847F2E771F0FA
:10CA10006DFB0027224604F5BA7140F2F315D2F8F7
:10CA2000A0307C32C31AAB428CBF0023012302F832
:10CA30003B3C914247EA0307F1D194F92830032B9C
:10CA400007D194F84033002B3BD0D4F83C030028A6
:10CA500049D167B1636B013309D043F095FB616B3A
:10CA600043F05CFB18B143F08FFB42F023FB94F9D9
:10CA70003032002B3AD194F93132CBBB94F93232B7
:10CA800013B1022384F8463394F846132046FFF787
:10CA900079FF8642054611D043F076FB4FF6FF71D1
:10CAA00043F03CFB50B1002D14BF00220422019240
:10CAB00043F06AFB019A032143F0C2FA284603B00F
:10CAC000F0BD0123042084F84033FFF79DFA0546AA
:10CAD00010B1214606F0FCFE94F92830C4F83C530E
:10CAE000032BB2D0B5E706F001FFB2E70023C9E798
:10CAF0000123C7E738B590F925300446D3B190F843
:10CB00004453BDB1FFF776FCC0B2022812D87C2393
:10CB10009FED0A7A03FB0044D4ED1B7AF4EEC77A4A
:10CB2000F1EE10FA06D4B7EE087AF4EEC77AF1EE19
:10CB300010FA00DD0025284638BD00BFABAA2A3F09
:10CB400070B5D0F80C5304460E4615F400350DD1DF
:10CB500090F844335BB90A78072A07D8012303FA0F
:10CB600002F290F84333134380F8433370BD94F8D6
:10CB70002420EBB29A42F9D906333146013554F8F4
:10CB800023000368DB689847F1E7000038B50546E5
:10CB900070242B591BB1002128193DF0C3F87C34B7
:10CBA000B4F5F27FF5D138BD014B1868704700BF6E
:10CBB000CC82003010B50446006810B103685B6891
:10CBC0009847204610BD000010B50446006810B11B
:10CBD00003685B689847204610BD000010B5044606
:10CBE000006810B103685B689847204610BD0000DC
:10CBF0002DE9F04FD0F80C538DB004460F4615F4D4
:10CC0000807B164698469DF858909DF85CA060D1B0
:10CC1000FFF70AFC054600283FD0CDE906BB069B7E
:10CC20004FF0000B4246394620460493CDE905BB40
:10CC3000FFF7FAFB064600283DD0CDE90ABB0A9A69
:10CC4000002308A904A808924A46CDE909335346AF
:10CC500000F0D4FF074608A8FFF7C0FF09A8FFF7B8
:10CC6000BDFF0AA8FFF7B0FF16B10BA8FFF7ACFF96
:10CC700004A8FFF7B3FF05A8FFF7B0FF06A8FFF76A
:10CC8000A3FF15B107A8FFF79FFF3A4608212046EA
:10CC90000DB0BDE8F04FFFF7E7BB04230E493A465D
:10CCA0000968CDE901030D4B06A800933346496896
:10CCB000FFF7D8F9B3E7042307493A460968CDE9F5
:10CCC0000103064B0AA8009343464968FFF7CAF9D7
:10CCD000B5E70DB0BDE8F08F60820030801A060025
:10CCE0002DE9F04F01249146D0F80C238BB08C40F5
:10CCF000984606460F4614409DF850309DF854A0C3
:10CD00009DF858B035D11A4641460593FFF78CFB84
:10CD1000059B054600B3CDE90844089A0023514617
:10CD200006A806925A46CDE90733C847044606A826
:10CD3000FFF754FF07A8FFF751FF08A8FFF744FFCC
:10CD400015B109A8FFF740FF2246394630460BB01F
:10CD5000BDE8F04FFFF788BB04220749CDE9010287
:10CD6000096808A8054A009242464968FFF77AF91F
:10CD7000D3E70BB0BDE8F08F60820030801A060068
:10CD8000B34B2DE9F04F1D68044689B00026686852
:10CD90004FF001084FF0080ADFF8BC9203689B6867
:10CDA0009847074608FA06F33B4240F07A8201367C
:10CDB000202EF7D1686800264FF001094FF00608D1
:10CDC0000368DFF894A2DB689847074609FA06F380
:10CDD0003B4240F078820136202EF7D16868002669
:10CDE0004FF001084FF0080A0368DFF870929B6863
:10CDF0009847074608FA06F33B4240F07582013631
:10CE0000202EF7D1686800264FF001084FF0080A7D
:10CE10000368DFF84C929B689847074608FA06F3C8
:10CE20003B4240F071820136202EF7D1686800261F
:10CE300001274FF01A0903689B689847804607FA54
:10CE400006F313EA080F40F06F820136202EF6D168
:10CE5000686800264FF0010A4FF01A090368B046CF
:10CE6000DB68984707460AFA06F33B4240F07782B0
:10CE70000136202EF7D1686800264FF0010ADFF84E
:10CE8000E4910368B046DB68984707460AFA06F360
:10CE90003B4240F07F820136202EF7D168680026A1
:10CEA0004FF0010ADFF8BC910368B046DB68984791
:10CEB00007460AFA06F33B4240F07C820136202EF8
:10CEC000F7D1686800264FF001084FF0020A0368A6
:10CED000DFF890919B689847074608FA06F33B42B3
:10CEE00040F078820136202EF7D1686800264FF096
:10CEF00001084FF0020A0368DFF868919B689847C1
:10CF0000074608FA06F33B4240F080820136202EA5
:10CF1000F7D1686800264FF00108DFF84C910368EC
:10CF2000B2469B689847074608FA06F33B4240F032
:10CF30007D820136202EF7D1686800264FF0010A65
:10CF4000DFF824910368B046DB68984707460AFA81
:10CF500006F33B4240F07A820136202EF7D1686812
:10CF600000264FF001084FF0060A0368DFF8FC9036
:10CF70009B689847074608FA06F33B4240F07682E2
:10CF80000136202EF7D1686800264FF0010ADFF83D
:10CF9000DC900368B046DB68984707460AFA06F358
:10CFA0003B4240F073820136202EF7D1294B07AF68
:10CFB0000426DFF8BC904FF00C0A079368684FF026
:10CFC00000084FF0010B03689B68984705900BFA27
:10CFD00008F3059A134240F0698208F10108B8F19C
:10CFE000200FF4D168684FF000084FF0010B036880
:10CFF000DB68984705900BFA08F3059A134240F056
:10D00000668208F10108B8F1200FF4D1013E013722
:10D0100016F0FF06D2D168684FF00108B146DFF87C
:10D0200054A003689B689847074608FA06F33B42FA
:10D0300040F060820136202EF7D1686800264FF05C
:10D040000109DFF830A00368B046DB6814E000BFD8
:10D05000608200300C0D0E0FE9FE02084116030835
:10D0600069180308750803084106030889DB0208EC
:10D07000350403084D0103089847074609FA06F3EB
:10D080003B4240F047820136202EF7D168680026E7
:10D090004FF00108DFF868A30368B1469B68984722
:10D0A000074608FA06F33B4240F044820136202E40
:10D0B000F7D1686800264FF00109DFF844A3036840
:10D0C000B046DB689847074609FA06F33B4240F052
:10D0D00041820136202EF7D1686800264FF0010802
:10D0E000DFF820A30368B1469B689847074608FA13
:10D0F00006F33B4240F03E820136202EF7D1BD4B75
:10D10000002668684FF00109079303689B689847F9
:10D11000B94A804609FA06F313EA080F1AD00DF14E
:10D120001C0A0427F3B24FF0000B1AF8011B20462B
:10D13000059300911021CDE9019BFFF7D1FD94F8F3
:10D140002710052900F0BC80013FAB4A059B17F072
:10D15000FF07EAD10136202EDCD1686800264FF0A7
:10D16000010B0368DB689847A34A80460BFA06F375
:10D1700013EA080F1AD00DF11C090427F3B24FF07F
:10D18000000A19F8011B2046059300911021CDE9F2
:10D1900001AAFFF7A5FD94F82710052900F090805B
:10D1A000013F954A059B17F0FF07EAD10136202E73
:10D1B000DCD1686800274FF00109DFF84CA2036852
:10D1C0009B689847804609FA07F313EA080F15D0C1
:10D1D0001026FBB24FF0000B52460321204600966A
:10D1E0000593CDE9019BFFF77BFD94F82720052AE5
:10D1F00066D00136059BF6B2142EEDD10137202FF3
:10D20000E1D1686800274FF00109DFF8F0A1036859
:10D210009B689847804609FA07F313EA080F15D070
:10D220001426FBB24FF0000B524615212046009603
:10D230000593CDE9019BFFF753FD94F82720052ABC
:10D240003ED00136059BF6B2182EEDD10137202FC6
:10D25000E1D1686800274FF0010A684E0368DB6877
:10D26000984780460AFA07F313EA080F15D01425E9
:10D270005FFA87FB4FF000095B46324615212046D6
:10D280000095CDE90199FFF72BFD94F82730052B88
:10D2900016D00135EDB2182DEED10137202FE1D196
:10D2A0000EE01E234A46002120460093F3B2CDE94A
:10D2B000018AFFF715FD94F82730052B7FF477AD31
:10D2C00009B0BDE8F08F1E23002152462046CDF85C
:10D2D0000880CDE90031F3B2FFF702FD94F8273062
:10D2E000052B7FF478ADEBE70D234A460C21204651
:10D2F0000093F3B2CDE9018AFFF7F2FC94F82730EE
:10D30000052B7FF47CADDBE72C234A461421204615
:10D310000093F3B2CDE9018AFFF7E2FC94F82730DD
:10D32000052B7FF480ADCBE7F1B269230C222046B8
:10D330000591CDE90079FFF75BFC94F82730052BC8
:10D34000BED068230C2205992046CDE90079FFF76D
:10D350004FFC94F82730052B7FF477ADB0E7F1B29E
:10D3600069230C2220460591CDE90089FFF740FC96
:10D3700094F82730052BA3D068230C22059920466A
:10D38000CDE90089FFF734FC94F82730052B7FF4B2
:10D390006FAD95E71C234A46052120460093F3B262
:10D3A000CDE90188FFF79CFC94F82730052B7FF42A
:10D3B00072AD85E71E234A46052120460093F3B24D
:10D3C000CDE90188FFF78CFC94F82730052B7FF41A
:10D3D00075AD75E71C234A46052120460093F3B23C
:10D3E000CDE9018AFFF77CFC94F82730052B7FF408
:10D3F00079AD65E720212223BD1B0308A9E80208B7
:10D40000E90D030815130308CDE002081E234A4660
:10D41000052120460093F3B2CDE9018AFFF760FCB5
:10D4200094F82730052B7FF471AD49E71E234A4657
:10D43000172120460093F3B2CDE9018AFFF750FC93
:10D4400094F82730052B7FF474AD39E71E234A4644
:10D45000172120460093F3B2CDE90188FFF740FC85
:10D4600094F82730052B7FF477AD29E70C234A4643
:10D47000062120460093F3B2CDE9018AFFF730FC84
:10D4800094F82730052B7FF47BAD19E70C234A462F
:10D49000062120460093F3B2CDE90188FFF720FC76
:10D4A00094F82730052B7FF47EAD09E7CDE901BA6A
:10D4B0003B784A460721204600935FFA88F3FFF73E
:10D4C0000FFC94F82730052B7FF487ADF8E6002396
:10D4D000CDF808A04A460721019320463B780093E7
:10D4E0005FFA88F3FFF7FCFB94F82730052B7FF4F5
:10D4F00088ADE5E60C2352460F2120460093F3B297
:10D50000CDE90189FFF7ECFB94F82730052B7FF478
:10D5100091ADD5E60C2352460F2120460093F3B27D
:10D52000CDE90188FFF7DCFB94F82730052B7FF469
:10D53000AAADC5E630235246092120460093F3B236
:10D54000CDE90189FFF7CCFB94F82730052B7FF458
:10D55000ADADB5E630235246092120460093F3B223
:10D56000CDE90188FFF7BCFB94F82730052B7FF449
:10D57000B0ADA5E630235246132120460093F3B206
:10D58000CDE90189FFF7ACFB94F82730052B7FF438
:10D59000B3AD95E670B50446FFF7F2FB94F827307B
:10D5A000052B29D0002594F84333E8B2EB40DB0784
:10D5B00015D40135082DF6D194F82730052B1BD052
:10D5C00094F8243013B194F82630ABB90B4B0C49C6
:10D5D0001B6898690368BDE870401B68184703F032
:10D5E00021FF02460028E4D011212046FEF73CFF2F
:10D5F00094F82730052BDCD170BD00BF608200306D
:10D60000D8570F082DE9F04F90F9253089B004461E
:10D61000002B00F00481012300F50D75024600F592
:10D62000107180F845332E462B46106F002859D0D4
:10D63000002384F8453394F94430642B5BD094F98B
:10D64000C030642B00F08D8094F93C31642B00F0E5
:10D650008A80D4F834722FBB01A920463CF046FBE7
:10D6600000B30C230697694604A805930123049789
:10D670008DF818306F4B8DF800700793BDF80430AB
:10D68000ADF810303CF0B2FC9DF9001051B1022908
:10D6900008DC38B1C9B27C23284603FB0141703154
:10D6A0003EF038FB94F845B3BBF1000F5DD0236F1B
:10D6B0000021A367D4F8EC30C4F8F430D4F8683112
:10D6C000C4F8703194F8273003F1C40204EB8202ED
:10D6D000042B7CD852F8040B01331061DBB242F802
:10D6E000041CF5E753F8040B0028A1D18B4202F18A
:10D6F0007C029AD19FE70020662304A98DF81030A0
:10D700007C2303FB004044303EF048FA04A9204645
:10D710003CF0ECFA00289CD004238DF8183000234C
:10D72000CDE90133039331230593694604A83CF006
:10D730005DFC059B28B108AA009902EB830242F820
:10D74000E01C0133332B0593EFD96DF091FF9DED74
:10D75000031ADDED020A66219DED010A6DF046FF18
:10D7600077E70120C8E70220C6E70127A94655F858
:10D77000043B23B1AB600137042FF7D197E7AA46EA
:10D78000B8465FFA88F3022BF5D8DAF8002055F88E
:10D79000043C9A4205D104A95046CDF810B03EF0A1
:10D7A000B9FA5AF8043B08F101020BB99046E8E7D0
:10D7B00004A906EB88000193CDF810B03EF0AAFA58
:10D7C000019B01A94846AB603EF0A4FAD3E794F868
:10D7D000453313B92046FEF725FD94F826300BB3E8
:10D7E000154B64211B68986A03685B68984720465C
:10D7F000FFF7EAF894F8423003B9236794F8BE3093
:10D800000BB9C4F8EC3094F83A310BB9C4F868316C
:10D81000FAF780F9FAF7EAF90123A4F8443309B0DA
:10D82000BDE8F08F2046FFF7B5FE94F82630002BB8
:10D83000E0D0D5E7C01A10086082003070470000C1
:10D8400001207047012070474368986870470000C6
:10D85000054B10B504460360C06A10B103685B68ED
:10D860009847204610BD00BF945C0F0840680368CD
:10D870009B6A184733B46C46406884E80C00036820
:10D88000DD6A94E80C00AC4602B030BC6047000092
:10D8900010B50446FFF7DCFF2046FEF7BDFB20462F
:10D8A00010BD000040680FF0F9BC00000123406883
:10D8B0000FF0F4BC40680FF0CDBC00000A224068B5
:10D8C0000FF072BC40680FF087BC000090F8313058
:10D8D00013B1002101F028B97047000040680FF033
:10D8E00001BD000073B5044605250026E06A0DF170
:10D8F00007028DF8076001210368DB68984778B15B
:10D900009DF807300C2B09D0102B05D0092B07D11F
:10D9100084F8333002B070BD1523F9E71423F7E71C
:10D92000013DE3D12846F5E710B4C06A0822312151
:10D9300003681C690123A4465DF8044B604700009E
:10D9400010B4C06A0122322103681C690023A44676
:10D950005DF8044B60470000F7B50446C06A0368F1
:10D960005B6998470546002871D0E06A03685B69E7
:10D97000984703689B689847E06A03689B699847E3
:10D9800060B9344B34491B68986903681B68984731
:10D990002B6828460026DB68984755E02046FFF7AD
:10D9A000CFFF0028F4D02046FFF79CFF0028EFD0DF
:10D9B000E06A01210368DB6A98472046FFF7B4FF5D
:10D9C00030B9244B25491B68986903681B68DEE75A
:10D9D000E06A0368DB69984730B91E4B20491B6831
:10D9E000986903681B68D2E7E06A012794F833104E
:10D9F00084F8317003685B6A9847E06A03689B6A41
:10DA000098470146204601F0F1F806460028BFD0AD
:10DA100094F830301BB13946204601F0F7F894F8FD
:10DA20003210204601F018F92B682846DB68984729
:10DA3000E06A009442F2107103681D6A094B019379
:10DA400002AB13E90C00A847304603B0F0BD064610
:10DA5000FAE700BF60820030005C0F08265C0F0808
:10DA6000455C0F0859DB020870B5002386B000251D
:10DA70000446C06A6A468DF8085010210593039346
:10DA80000493CDE9005503689E680923B047A0B10F
:10DA90009DF8003013F0010615D194F834300133AD
:10DAA000DBB2052B84F8343007D12046FFF748FF5E
:10DAB0002046FFF739FF84F83460E06A03681B6B87
:10DAC000984706B070BD9DF8083084F834501B07A5
:10DAD000F3D4BDF901309FED1E6A06EE903ABDF910
:10DAE0000330F8EEE66A07EE103ABDF90530B8EEFD
:10DAF000C77ACDED036AF0EEE66A07EE903A8DED57
:10DB0000047AF4EEC66AF8EEE77AF1EE10FACDED9B
:10DB1000057A0DD5B0EEC77AB4EEC67AF1EE10FAFA
:10DB200006D5F0EEE77AF4EEC67AF1EE10FAC4D438
:10DB30009FED080A03A817F035FCB2EE040A03A80B
:10DB400017F030FC0A2203A9204601F0E9F8B4E7F7
:10DB5000000000349A99193EFFF786BF044B10B5B8
:10DB6000044640F8043BFFF739F8204610BD00BFDB
:10DB7000AC5C0F0810B50446FFF7F0FF2046FEF737
:10DB80004BFA204610BD0000F7B503680F46164655
:10DB90001BB90024204603B0F0BD002401930460AB
:10DBA0000820FEF731FA054620B1124B0360019BB5
:10DBB0000194436001A8FFF711F8002DE9D0382047
:10DBC000FEF722FA04460028E3D000F0ADFE0A4B2F
:10DBD000E5622046236084F8307084F83260FFF7F5
:10DBE000BBFE05460028D5D1236820462C465B683D
:10DBF0009847CFE7AC5C0F08945C0F082DE9F74F0E
:10DC0000046806460D4690469946002C6CD00B6879
:10DC1000002B49D0236820469B6A984703689B687D
:10DC200098470123002128680DEB03020FF036FB13
:10DC300098B39DF80130EA2B2FD14FF0060ADFF898
:10DC4000ECB000238022062128680FF003FB20B3EC
:10DC5000DBF800700A21B86A03685B689847002304
:10DC6000062128681A460FF0F5FAB0B1B86A0A2101
:10DC700003685B6898470123062128680DEB0302BF
:10DC80000FF00CFB48B19DF8014014F040042FD078
:10DC90000AF1FF3A1AF0FF0AD3D1306803689B6A91
:10DCA00098470368DB68984700241DE0022223465A
:10DCB0000F2128680FF0CEFAB86A012103685B686B
:10DCC0009847306803689B6A98470368DB68984701
:10DCD00033684A463460414601A80193FFF754FF78
:10DCE000044601A8FEF77AFF204603B0BDE8F08F96
:10DCF000224623460F2128680FF0ACFAB86A0121AA
:10DD000003685B6898470223214630680DEB0302E5
:10DD10000FF0C4FA04460028C8D0B8690249036865
:10DD20001B689847B9E700BF6C5C0F086082003041
:10DD3000002100F0F9BE000070B504468CB0042646
:10DD4000013E76B2731C4AD015236A465D21E06A13
:10DD50000FF0A4FA0028F3D0152306AA5D21E06A8B
:10DD60000FF09CFA05460028EAD0152206A968465D
:10DD7000BDF0A6FA0028E3D19DF800309DF81020F0
:10DD800084F830309DF8073084F832309DF8143034
:10DD900084F83C309DF8133084F83D309DF80F3006
:10DDA00043EA02239DF80C20E3879DF8013084F8B4
:10DDB00031309DF8083084F83330039BC3F30F23D0
:10DDC000A3869DF80B3043EA0223E386049BC3F34A
:10DDD0000F232387019BC3F30F23638707E0054BC2
:10DDE000002505491B68986903681B689847284601
:10DDF0000CB070BD60820030E05C0F082DE9FF417F
:10DE000004460023C06A04258DF807300368DFF854
:10DE100050819B6A984703689B689847E06A0A218B
:10DE20000368DB6C98470A220421E06A0FF0BCF912
:10DE3000013D6DB26B1C32D000234B218222E06A7F
:10DE40000FF008FAD8F8006007460221B06A0368AC
:10DE50005B689847002FEBD001234B21E06A1A46FC
